:020000021000EC
:10F000000000012039F5010061F5010063F5010000
:10F0100065F5010067F5010069F5010000000000D9
:10F020000000000000000000000000006BF501007F
:10F030006DF50100000000006FF50100A917040044
:10F04000014D020073F501003D500200614D0200C8
:10F05000B54D0200D5600200A951020073F5010010
:10F0600073F50100ED17040073F5010073F501005D
:10F0700073F50100115B020073F5010073F50100E7
:10F08000E9170400C928020073F5010073F50100B7
:10F09000D129020075D20300C519020073F50100E1
:10F0A00073F5010073F5010073F50100356302008B
:10F0B00073F5010073F5010000000000000000007E
:10F0C00073F5010073F5010073F5010073F501009C
:10F0D00073F50100DD5C020073F501000000000023
:10F0E0000000000000000000000000000000000020
:10F0F0000000000000000000000000000000000010
:10F1000000000000000000000000000000000000FF
:10F1100000000000000000000000000000000000EF
:10F4000010B5054C237833B9044B13B10448AFF35E
:10F4100000800123237010BD402D0020000000005B
:10F42000E088060008B5034B1BB103490348AFF35E
:10F43000008008BD00000000442D0020E088060088
:10F44000154B002B08BF134B9D46A3F5803A0021B6
:10F450008B460F461348144A121A00F063F80F4BFC
:10F46000002B00D098470E4B002B00D0984700206F
:10F47000002104000D000D48002802D00C48AFF315
:10F48000008000F02BF82000290024F0E9FB00F0B8
:10F4900011F800BF0000080000000120000000007B
:10F4A00000000000402D002050E10020000000007E
:10F4B0000000000008B5074B044613B10021AFF36C
:10F4C0000080054B1868836A03B19847204600F016
:10F4D00031F800BF00000000BCD2050070B50D4D32
:10F4E0000D4C641BA4100026A64209D10B4D0C4CF8
:10F4F0003DF0D8FE641BA4100026A64205D170BDC5
:10F5000055F8043B98470136EEE755F8043B984719
:10F510000136F2E7182D0020182D0020182D0020AC
:10F520001C2D002002440346934200D1704703F88B
:10F53000011BF9E7FEE700BF0649074A074B9B1A84
:10F5400003DD043BC858D050FBDC06F0C7FCFFF7D6
:10F5500077FF0000EC880600402C0020402D0020A2
:10F56000FEE7FEE7FEE7FEE7FEE7FEE7FEE7FEE773
:10F57000FEE7FEE71FB501238DF80030054B8DF83F
:10F58000080001916846D3E90012904705B05DF884
:10F5900004FB00BF78CA002061DF704748DF704776
:10F5A00010B50388012B11D8094A02EB03124388D6
:10F5B0005189CC1A032C09D4C3F57F43FD330B4486
:10F5C0005381002303804380184610BD0420FCE7CC
:10F5D00080CF002010B5124A0B6802EB0010426881
:10F5E00073B15888033003EB800302F580524FF665
:10F5F000FF749A4202D91868013004D1002009E052
:10F6000002F10803F1E79888A04204D0188810B1ED
:10F610000B60012010BD5888033003EB8003E8E73E
:10F6200080CF002073B5436804460D4613B31E4ACD
:10F6300011688B421ED3526893421BD813F003000B
:10F6400018D11A4A21891289914213D121689A68E6
:10F6500091420FD1164A5268934201D80A2004E021
:10F6600002F580529342F9D22880B0FA80F0400926
:10F6700002B070BD00232B801E46019601A9288888
:10F68000FFF7A8FF30B92B8801339BB22B80002BEA
:10F69000F3D0EDE7019B226899689142EED1636057
:10F6A000024B1B892381E3E7202D00203CCC002066
:10F6B00080CF0020033083B240F2FD32934230B558
:10F6C0000ED909200BE0228965892A441A4492B296
:10F6D000B2F5806F08D2088062891344638130BD1F
:10F6E000024C20780028EED00720F8E780CF0020D9
:10F6F00010B50A494A788C78531CDBB29C4208BF8B
:10F7000000230C789C421FBF0370486802EB420242
:10F7100000EBC20008BF002010BD00BFFCCE0020DF
:10F72000AADF7047A9DF7047A7DF704785DF704702
:10F730007FDF70477EDF7047084A30B500230C2416
:10F7400004FB03F18D5A854202D10A44508830BD32
:10F750000133082BF4D14FF6FF70F8E7A6CB002059
:10F760006EDF704758B1CB0801F00701C25C01237E
:10F7700003FA01F10A4214BF184600207047012025
:10F780007047000070B50A4E3468054654B1706881
:10F7900060B1FF2D08D02946FFF7E4FF30B1F368D0
:10F7A00003FB0544204670BD0024FBE70446F9E74F
:10F7B00004D10020012804D0043804288CBF002084
:10F7C000012070478378013B072B07D8DFE803F05F
:10F7D0000706060606070409142303807047012361
:10F7E000FBE743689B8809339B08F6E770B5054D36
:10F7F0000646002455F8043B304601349847052C52
:10F80000F8D170BDF8D40500114BF0B500221426D4
:10F810001D4606FB02F4E75A874212D12344142600
:10F8200000249A788A420AD001342246072A0BD84B
:10F8300006FB02F3EF5A874208D1EB18F1D11846C4
:10F84000F0BD0132082AE4D10023F8E70132EDE7E8
:10F8500014D1002030B5072185B0FFF7D5FF04464D
:10F8600000283AD04568002D39D1007CFFF78AFF87
:10F870000721CDE902558DF80A1040B3E3680390E3
:10F8800003EB83031B019BB29B0802A8ADF8083071
:10F89000FFF798FF9DF80A00FFF78CFFD8B1114BD6
:10F8A0001B789B0715D5BDF808500DF106012846B9
:10F8B000FFF700FF48B9BDF80630A380E5800A4B8A
:10F8C000185C092803D005B030BD0928F7D90320FA
:10F8D000F9E70220F3E70846F5E70520F3E7002003
:10F8E000F1E700BF39CC0020D8D2050038B54FF67B
:10F8F000FF73984218BF01300D4614BF84B2002434
:10F90000FF2C03D94FF6FF74204638BD2146284608
:10F91000FFF728FF0028F7D10134A4B2F0E7000078
:10F92000F8B5074D074E074600243378A34200DCA4
:10F93000F8BD55F8043B384698470134F5E700BF59
:10F9400018CC0020C9CD00207DDF704779DF7047DB
:10F950006DDF704738B5074C051E04F1080318BF6A
:10F960001C4623682BB11A6822605B6828469847BA
:10F97000F7E738BD50CB002040DF70473FDF7047CE
:10F9800037B5D0F818350A7DDBB28DF807300B7F1C
:10F990009A4282BF0A699DF80740D4540B7F0D7BC1
:10F9A0000133DBB25A1C95420B7705D98B689B5CFF
:10F9B000C0F81C3501200AE00C7D944201D9CB7EB1
:10F9C000F6E7AB42F6D3A3422CBF0020012003B0E0
:10F9D00030BD0023435082B043580193019B02B0D5
:10F9E00070472DE9F0470D789DF820609DF824A020
:10F9F00004460F469946002D60D1D0F8243192F884
:10FA000000809BB14FF49271FFF7E3FF0123636124
:10FA10003B70B04550D1D4F80431002B4CD04FF49A
:10FA200082712046FFF7D5FF00251DE0D0F81C317C
:10FA3000FBB14FF48E71FFF7CCFFD0F824311BB12E
:10FA40004FF492712046DFE713789E4207D919F8E8
:10FA50000330C0F81C35137801331370D9E7012344
:10FA6000BAF1000F03D0C3612846BDE8F0874361B7
:10FA7000CFE7D0F80831002BCBD04FF48471FFF7DB
:10FA8000A8FFD0F82431002BDAD113789E42C0D9D8
:10FA9000D0F8181509F8031013780133DBB213708E
:10FAA000721E934205D10223C0F800320123236263
:10FAB000AFE79E42FAD1ACE70125D5E74FF492714A
:10FAC000FFF787FF4FF48E71FFF783FF4FF48471C8
:10FAD000FFF77FFF9FE72DE9F3470C4605464FF4FC
:10FAE000827120461F469046FFF773FF4FF49271D4
:10FAF000FFF76FFF4FF48E71FFF76BFF4FF48471C8
:10FB0000FFF767FF0023012F85F8263085F82330A3
:10FB100008BF02224FF001030CBFC4F80022C4F852
:10FB20000032236223602E6846BB05F1260A05F1E8
:10FB30002309CDE900764346524649462046FFF761
:10FB400050FF0028F5D195F82330EBB1D4F8C43438
:10FB5000C4F8C434C3B113F0010F14BF4FF4024012
:10FB6000032048F2012213F0020F18BF104613F0D1
:10FB7000040F48F2022318BF184606E040F286231D
:10FB8000AB60AB68C4F80433002002B0BDE8F08776
:10FB90002DE9F3470C4605464FF4827120461F4677
:10FBA00016469DF82880FFF714FF4FF49271FFF777
:10FBB00010FF4FF48E71FFF70CFF4FF48471FFF7C5
:10FBC00008FF0023C4F8003285F8263085F823307A
:10FBD00001232362A36095F82620974232D9B35CB3
:10FBE000C4F81C3595F82630013385F826302B688B
:10FBF0007BBB05F1260A05F12309CDE900783346E0
:10FC0000524649462046FFF7ECFE0028F5D195F80C
:10FC1000233023B3D4F8C434C4F8C434FBB113F094
:10FC2000010F14BF4FF40240032048F2012213F0E9
:10FC3000020F18BF104613F0040F48F2022318BF3A
:10FC400018460DE0B8F1000F01D0E361CFE7636122
:10FC5000CDE740F28623AB60AB68C4F804330020E4
:10FC600002B0BDE8F0872DE9F04793F9005090B05D
:10FC70000024013D6E46AD002746A446A0465FF035
:10FC8000000E03E05FEA080EBEEB050EB8EB0E09AE
:10FC900052F809A051F80E90A9FB0A9A14EB090436
:10FCA00057EB0A075CF1000C1EF1040EAE4501DCB7
:10FCB000C645EBDD46F808403C4667465FF0000C61
:10FCC00018F10408A845DADDB8EB450FDADD46F88F
:10FCD0000840D3F8B0303146984710B0BDE8F087FF
:10FCE00013460A46FFF7BFBFF0B5154689B01C465C
:10FCF00007460E461A4629466846FFF7F1FF234697
:10FD00006A4639463846FFF7AEFF23462A4669461B
:10FD10006846FFF7A8FF23466A4631463046FFF79C
:10FD2000A2FF09B0F0BD00EB81010023884200D39F
:10FD3000704751F8042D43EA52030B60D307F5E7EF
:10FD400010B5013A52B2130601D5002010BD50F88B
:10FD5000224051F822309C4205D802F1FF32F2D203
:10FD60004FF0FF30F2E70120F0E710B500235CB25E
:10FD7000A24200DC10BD51F8234040F8234001337B
:10FD8000F5E7013910B549B2041D0A06CBB204D417
:10FD9000013954F82120002AF7D001335BB273B146
:10FDA00003F18042013A50F82220002022B9013BA1
:10FDB00000EB431318B210BD52080130F6E71846A5
:10FDC000F9E7002310B51C465AB2914200DC10BD81
:10FDD00040F823400133F7E7000000000000000076
:10FDE000C3F10803DB0070B50133002403A500BF95
:10FDF0005B1920C940CAAD1B20C0184720C940CAA2
:10FE0000B54120C020C940CAB54120C020C940CA60
:10FE1000B54120C020C940CAB54120C020C940CA50
:10FE2000B54120C020C940CAB54120C020C940CA40
:10FE3000B54120C06441B4FA84F0400970BD00BFF0
:10FE4000C3F10803DB0070B50133002403A500BF34
:10FE50005B1920C940CAAD1920C0184720C940CA43
:10FE6000754120C020C940CA754120C020C940CA80
:10FE7000754120C020C940CA754120C020C940CA70
:10FE8000754120C020C940CA754120C020C940CA60
:10FE9000754120C06441204670BD00BFF0B5082206
:10FEA00089B00C460646FFF760FFCB6A03930B6BE5
:10FEB00004934B6B05938B6B0693CB6B07930027D7
:10FEC00008236A4669466846CDE901770097FFF73F
:10FED000B7FF082305466A4631463046FFF7B0FFB4
:10FEE000236B0393636B0493A36B0593E36B05444C
:10FEF000CDE906376A46082369466846FFF7A0FF42
:10FF0000082305446A4631463046FFF799FF236AC5
:10FF10000093636A0193A36A0293A36B0693E36B56
:10FF20000793054408236A4631463046CDE90477F5
:10FF30000397FFF785FF636A0093A36AA26B01939F
:10FF4000E36A02930492636BE26B0393CDE90523AA
:10FF5000236A0793054408236A4631463046FFF773
:10FF60006FFFE36A0093236B0193636B0293236A31
:10FF70000693A36A0793054408236A463146304630
:10FF8000CDE904770397FFF72BFF236B0093636B97
:10FF90000193A36B0293E36B0393636A0693E36A93
:10FFA00007932D1A08236A4631463046CDE9047777
:10FFB000FFF716FF636B0093A36B0193E36B029350
:10FFC000236A0393636A0493A36ACDE90537236B1D
:10FFD00007932D1A08236A4631463046FFF700FF83
:10FFE000A36B0093E36BCDE90137636A0393A36AC4
:10FFF0000493E36ACDE90537636B07932D1A082351
:020000022000DC
:100000006A4631463046FFF7EBFE2D1A0D4C0FD4F1
:1000100035B9082231462046FFF792FE01280FD05D
:100020000823224631463046FFF7DAFE2D1AEFE765
:100030000823224631463046FFF702FF2D18F7D439
:1000400009B0F0BDF4D205002DE9F04391B00F46A0
:100050001C220021804609A8FFF764FA01251C2212
:10006000002101A80895FFF75DFA394608AA11F9A1
:10007000046B009533461046FFF7E2FE314608A8B0
:10008000FFF77FFE013804B2012C07DC32466946D7
:100090004046FFF76AFE11B0BDE8F0833A46684675
:1000A0006946FFF71DFE10AB601103EB80001FFADD
:1000B00084F909F01F0350F8202C05FA03F31342CA
:1000C00005D03B46424669466846FFF7CCFD09F13C
:1000D000FF3424B2D8E770B5036813F00105064673
:1000E000144605D013460A460146FFF7A9FE054609
:1000F00021463046FFF717FE45B104F18042013A30
:1001000056F8223043F0004346F8223070BD70B5F7
:100110009DF910401E4623460546FFF761FE38B1A3
:100120002346324629462846BDE87040FFF788BE80
:1001300070BD2DE9F0438BB01446129D15F9046B88
:1001400000961F46804689462B460246214602A855
:10015000FFF7DDFF02A9129A0846FFF7C1FD129BC7
:1001600002AA41464046FFF77EFD129B02AA2146A5
:100170002046FFF778FD2B464A463946384600961A
:10018000FFF7C5FF129A394602A8FFF7A9FD02A999
:100190002B46424608460096FFF7B9FF02A92B46B8
:1001A000224608460096FFF7B2FF2B4642462146FC
:1001B00020460096FFF7ABFF129B22464946484671
:1001C000FFF751FD2B4602AA414620460096FFF755
:1001D0009EFF129B224639463846FFF744FD2B46C8
:1001E0004A46394638460096FFF791FF324602A943
:1001F0002046FFF7BAFD0BB0BDE8F08370B59DF95E
:1002000010401E4623460546FFF71AFE30B9224627
:1002100029463046FFF794FD012807D02346324691
:1002200029462846BDE87040FFF7DABD70BD2DE9CC
:10023000F0439BB01646229C14F9045B0095984647
:100240000746894623460246314612A8FFF75FFF5C
:1002500012A9229A0846FFF743FD229B12AA3946AB
:100260003846FFF700FD229B12AA31463046FFF7C1
:10027000FAFC23464A46414612A80095FFF7BEFF06
:1002800023464A46414640460095FFF740FF234635
:100290003A4631460AA80095FFF739FF229B0AAA81
:1002A00049464846FFF7DFFC2346324639460AA84E
:1002B0000095FFF7A3FF229A41463046FFF710FD55
:1002C00023460AAA314630460095FFF720FF234611
:1002D0003246394602A80095FFF719FF229B02AA71
:1002E00041464046FFF7BFFC23464A46414640464A
:1002F0000095FFF70CFF229A12A902A8FFF7F0FC65
:1003000002A923460AAA08460095FFF700FF2346E4
:100310003A4602A90AA80095FFF7F9FE0AA9229B0E
:1003200012AA0846FFF79FFC23464A460AA94846F8
:100330000095FFF7ECFE2A4602A93846FFF715FDA7
:100340001BB0BDE8F0832DE9F04115468AB00446A4
:1003500088461C22002103A8FFF7E4F82E1D95F91A
:10036000007003232A46414620460293FFF7B8FC5B
:10037000334602AA214620460097FFF7C8FE2B46C7
:10038000424621462046FFF76EFC0097334605F1B2
:10039000840221462046FFF731FF0AB0BDE8F08114
:1003A0000C4B1B78062B10D10B4B1B681A070CD17A
:1003B0000A4B186800F0F003302B08D000F0E00082
:1003C000A0F1400358425841704700207047012077
:1003D000704700BFE00F00F0E40F00F0E80F00F0FE
:1003E000094B1B78062B0CD1084B1B681A0708D148
:1003F000074B186800F0F000A0F130035842584154
:1004000070470020704700BFE00F00F0E40F00F0DD
:10041000E80F00F010B9024B01221A60704700BFCC
:100420000050004010B50C494A6E042A044611D011
:100430000B6E1344032B02F101024A6688BF043B92
:10044000182202FB031318460021FFF76BF8206007
:10045000012010BD0020FCE720D0002010B504468C
:1004600086B01422002101A8FFF75CF86088ADF87F
:100470000800FFF761F92378ADF80600092B0CD8C6
:10048000DFE803F005051014161B1D0E1F210723BE
:100490008DF8043008238DF80C3001A8FFF740FADE
:1004A00006B010BD0D238DF80430F6E70E23FAE7F1
:1004B00007238DF804300523EDE70F23F3E710231E
:1004C000F1E70523EFE706238DF80430A3680393D3
:1004D000A388ADF80630E0E708B5134644F2010200
:1004E000904203BF5A681988986800221AF05CF994
:1004F00030B50B4B1B68012293F8641021338A42FC
:1005000004DB405CB0FA80F0400930BD13F8014BC9
:10051000855CA54201D10132F1E70020F5E700BF7B
:10052000CCC9002070B5244B0022C3F80025234A13
:10053000516831B12249C3F8081322490420C1F897
:100540008000D3F80C55D3F81445D3F80815D3F828
:1005500010054FF0FF36B542C3F8146518BF05F516
:10056000E075C3F80C65C3F80865C3F810651EBFD5
:100570004FF0A043022643F82560651C1FBF4FF0D3
:10058000A04304F5E074022543F82450441C1FBF27
:1005900000F5E0704FF0A043022443F820404B1CCC
:1005A0001FBF4FF0A04301F5E071022043F8210086
:1005B0000023D376536070BD0020004078CA00202D
:1005C0008402020000E100E02DE9F04F85B08A4688
:1005D0000390039C2578284632F032FA0746D8B9B2
:1005E0002D2D1CD10134012303940193DDF80CB0AF
:1005F000BAF1000F01D0CAF800B00022114603A8DA
:1006000032F0C6F98046002835D1614D00242046DD
:10061000294605B0BDE8F08F01340394D9E72B2DAE
:1006200004BF013403940190E0E71846029332F0CE
:100630009AF9B0F10009029B20DBC8451EDD404657
:100640003CF05AF822462B463CF0C0F804460D46D2
:1006500048463CF051F822462B463BF001FF01365C
:1006600004460D460396039E3378002BDDD1B8F186
:100670000A0F37D113E000240025F4E7B8F10A0F80
:1006800030D12E2B0BD10FF20019D9E90089013698
:100690000396039E30783038C3B2092B39D9039BB7
:1006A0001A7802F0DF02452A1CD15A1C03925A78AC
:1006B0002D2A01D02B2A05D12D3A574203F10203EE
:1006C000574103934FF000080A20039A1378303BF8
:1006D000D9B2092936D9002F39D12E4F0026B8F1C9
:1006E000000F46D1039BBAF1000F01D0CAF80030C9
:1006F0009B458AD09BF800202E2A03D10BF1010BD9
:100700005B4582D0019B002B81D005F100431D4643
:100710007DE73BF0F1FF42464B463CF057F802467E
:100720000B46204629463BF09BFE002204460D4620
:1007300040464946174B3CF073F9013680468946DE
:100740000396A6E7013200FB08380392BDE7114F7C
:10075000C8F100080026B8F1000FC3D02046294692
:1007600032463B463CF05CF908F1010804460D4670
:10077000F1E72046294632463B463CF027F808F18F
:10078000FF3804460D46AAE79A9999999999B93F75
:100790000000F87F0000244070B58AB00C46014686
:1007A00068461D4632F0E4FE0022214605A832F0DC
:1007B000DFFE684632F088FC044605A832F084FC6F
:1007C0008442064621D0039850B1C389A3F5007333
:1007D0009BB2C381C38903F4F0530BB937F0C6FE53
:1007E000089850B1C389A3F500739BB2C381C38934
:1007F00003F4F0530BB937F0B9FE002C01DB002EE7
:1008000000DAF5B9A01B0AB070BD002C1BDA039802
:1008100050B1C389A3F500739BB2C381C38903F4AC
:10082000F0530BB937F0A2FE089850B1C389A3F575
:1008300000739BB2C381C48914F4F05401D137F022
:1008400095FE0020DFE7684632F0A8FA05A832F0EE
:10085000A5FAAEE7044A138A9BB223F0410343F0A2
:1008600040031382704700BF682D002030B587B069
:100870000A46014601A832F07BFE0025DDE901327F
:10088000934205F1010401D2013514D1049850B10D
:10089000C389A3F500739BB2C381C38903F4F053EA
:1008A0000BB937F063FE20202CF0BCFB14F1FF34B1
:1008B0000DD207B030BD059810B1C05C0A28E5D054
:1008C0002CF0B0FB01A8254632F068FAD6E70820E4
:1008D000EAE730B587B00D46019009B100230B60FF
:1008E0000021102202A8FEF71DFE02A9019838F08F
:1008F000AFF9E0B10024029B039A23F07F43033356
:1009000023F00303013203F110030AD11C44002237
:1009100002A901A838F0D6F90028ECD1204607B08A
:1009200030BD002DF3D02A6813442B60EFE7044656
:10093000F4E730B587B04FF4D8240021102202A884
:100940000194FEF7EFFD02A9204638F081F970B15D
:10095000002202A901A8DDE9015438F0B3F900280A
:10096000F6D124F07F4413352C4424F00304C4F55D
:10097000EC2007B030BD2DE9F04F89B0D51C0193B4
:1009800025F00305002382468B4617461035039356
:10099000984604AC039E86B3304638F05DF9804635
:1009A000039838F07FF9064678B1039BC21A954246
:1009B0000BD9FB1A0344984507D9B5F5007F04D23B
:1009C000214638F045F900B90396019B039947EA9F
:1009D000036710224FF0FF33204605930497CDE9BB
:1009E00006AB1AF021FE129B23B194E80F00129C73
:1009F00084E80F00039E103638E04FF4D8230393A9
:100A0000B1462146039838F023F978B1059B0133AC
:100A100006D1DDE906235B4504BF5245DDF80C90A5
:100A20000122214603A838F04DF9EEE7039838F08B
:100A300013F985421ED9039838F034F90123039045
:100A40000398C8B9B9F1000F0BD02146484638F0D9
:100A5000FFF80422002309EB020105A805931AF010
:100A6000E3FD039878B9B8F1000F11D0304609B012
:100A7000BDE8F08F0023E3E7002BC2D138F0ECF89B
:100A80008542BED8DEE738F0E7F88742EBD881E749
:100A900038F03EFA80460028E8D00023039379E737
:100AA0002DE9F04F8DB002AFB3F10009C7E90201A3
:100AB00092463E6D4FF0000519DBAE4217DB07F1A1
:100AC000100110463D6133F050FC804600BB50469B
:100AD00035F0C4FA0446386131F0F0FD04F5807356
:100AE000834209D95A49012034F078FE002528466E
:100AF0002C37BD46BDE8F08FE31D23F00703ADEBB7
:100B0000030D0DF1080822464146504635F096FA8D
:100B100006B93E6907F1180B5A46D7E9020138F0C9
:100B2000FCF8044620B9B9F1000F2FD04949DAE7A3
:100B3000B9F1000F35D1BB691A0E05D1B34203D10B
:100B4000314638F043F960BBBD6925F07F439E42D2
:100B50001CD12D0E1AD1D7F810A0564516D1331F2F
:100B600010E062597A619D428CBFAAEB0502042213
:100B700008EB050107F114007B603CF02DFB28B960
:100B80007B680435AA45ECD80125B0E7CDF800B064
:100B900000233246D7E90201FFF7EDFE04460028A4
:100BA000C4D03969BB6909EB010223F07F439A4243
:100BB00001D9294997E74C44204638F007F9054602
:100BC00020B92649012034F009FE90E714F0030013
:100BD0001FD0A4EB0009C0F10406D9F800307B61F6
:100BE0003B699E4228BF1E4607F114031844324653
:100BF00041463CF0FFFA0422494607F114001AF07E
:100C000013FD3B69B3427FF672AFB04434449E1B80
:100C10003E613A6902F00306921B3A611AB121461D
:100C200040461AF001FD002E3FF461AF39690C44D3
:100C3000324623687B61414407F114003CF0DAFA44
:100C40000422214607F114001AF0EEFC4FE700BF22
:100C5000B1D30500D8D30500F6D3050012D40500A2
:100C60000C4A002330B41146184640F6C41401EB78
:100C700003151032E8819D1C0133A34222F80C5C5D
:100C8000F5D149F634430122C852034B1A8030BCD7
:100C900037F038BB882D0020862D002070B586B037
:100CA00015460C460022014601A832F061FC2E4692
:100CB000DDE901239A4210D3049850B1C389A3F50A
:100CC00000739BB2C381C38903F4F0530BB937F0AF
:100CD0004DFC00232370AD1B0DE07EB9049850B18C
:100CE000C389A3F500739BB2C381C38903F4F05396
:100CF0000BB937F03BFC284606B070BD059B03B12D
:100D00009B5C04F8013B01A832F048F8013ECFE7B4
:100D100037B50123009300231A460A49044633F0ED
:100D200013FA05465CB1E389A3F500739BB2E38136
:100D3000E38903F4F05313B9204637F017FC284633
:100D400003B030BDEDD40500F8B5858907460C46E3
:100D500095B31A4B013D03EB05152846EB8903F5C6
:100D600000739BB2EB8133F0DBFBEB89A3F50073DF
:100D70009BB2EB81EB8903F4F053461C13B9284670
:100D800037F0F4FB304636F0E3FF214637F088FCBD
:100D9000044680B10146384633F05EFCE389A3F592
:100DA00000739BB2E381E38903F4F05313B9204647
:100DB00037F0DCFB701CF8BD0126E3E7882D00202E
:100DC00038B5074C25780023EDB20246194623704A
:100DD00035F05CFD25700348BDE838402CF010B9B3
:100DE000842D00205151060070B5044637F0A1FB58
:100DF0000546B0B120460022184934F071FF044680
:100E000037F0E2F978B900255CB1E389A3F5007306
:100E10009BB2E381E38903F4F05313B9204637F022
:100E2000A5FB284670BD00220D49204634F058FF2E
:100E300006460028E7D00B492DF04EF8F389A3F5BC
:100E400000739BB2F381F38903F4F0530546002B42
:100E5000DAD1304637F08AFBD6E700BFDCD4050094
:100E60005D180600E6D40500002370B50B6005464A
:100E70000E4637F027F8044610B90025284670BD05
:100E8000294636F0B7FF054668B9E389A3F5007334
:100E90009BB2E381E38903F4F053002BEDD12046AC
:100EA00037F064FBEAE7204632F05AFB3060E38912
:100EB000A3F500739BB2E381E38903F4F053002BA5
:100EC000DCD1ECE72DE9F341002400F47F671546FF
:100ED0001470A7F54072502A0E4600F4704312D8E1
:100EE000484A11F0100F484908BF1146002B79D02D
:100EF000B3F5805F78D0B3F5005F444C18BF002491
:100F00004FF440784BE0A7F50072202A0DD8002B53
:100F10006CD0B3F5805F6BD0B3F5005F3C4C18BF6D
:100F200000244FF400783B4939E0A7F52072302ABD
:100F30000AD8002B5ED0B3F5805F374C18BF002471
:100F40004FF4207835492AE0B7F5C07F09D1002B4E
:100F500052D0B3F5805F324C18BF0024B8463149F7
:100F60001DE0A7F11002B2F5887F47D844F643028E
:100F7000ADF80020C3F302321B0402F1310248BF76
:100F80004E2329494CBF8DF804408DF803408DF85D
:100F9000022048BF8DF803306C464FF01008F00770
:100FA00003D50F2228463CF067F9B2070BD5284637
:100FB0003CF05AF9A7EB08073F11012229180A2330
:100FC000B81831F0AFFC54B1330708D528463CF0CF
:100FD0004BF92146C0F10F0228463CF04DF902B012
:100FE000BDE8F081114C8BE7114C89E7114C98E773
:100FF000114C96E7114CA3E7114CAFE7A0461149FD
:10100000CDE700BF42D405003BD40500511A0600CD
:1010100061D40500AC1306006DD4050069D4050049
:101020004CD4050050D4050048D40500F112060048
:1010300054D4050057D405005CD4050065D40500E0
:1010400071D4050052510600F0B54FF080530220D4
:10105000D3F85014D3F85424284BC3F80403284879
:10106000C3F80403274B93F800E093F801C09F787E
:10107000DE781D795C7998794EEA0C033B43334363
:101080002B4323430343204B2AD083F800E083F80B
:1010900001C09F701E715D719C71D8711D789C7824
:1010A0005A785E79586885EA0401514081F08801D8
:1010B000D970197971409E797140DE797140197249
:1010C00012020321597242EA05420C4B2243C3F833
:1010D000942500BA4422C3F89005C3F8A025F0BDBA
:1010E000080A1970090C9970110A1A715971110CBA
:1010F000120E58709971DA71D0E700BF00500040AD
:1011000080000800F4CE0020DFCE002038B5002299
:10111000054634F0E5FD044698B100231A46014621
:1011200028462AF07DF8E389A3F500739BB2E3819A
:10113000E38903F4F05323B92046BDE8384037F083
:1011400015BA38BD70B5EFF3108672B60D4A9468C3
:101150000123A4B993600C4B0C4DD3F880102940A7
:101160001160C3F88050D3F8841051604FF0FF3203
:10117000C3F88420047006B962B6002070BD037005
:10118000F9E700BFBCD1002000E100E0FC06FFBC95
:1011900010B588B012788DF80C20CDE90001FF223F
:1011A000002102918DF80D2001214FF6FF72104CA5
:1011B0008DF81C10ADF80E208DF8103029F00CF9C8
:1011C00070B131F073FA58B914F1FF34F6D209490D
:1011D000042034F003FB684629F00EF908B010BD76
:1011E000002CF4D031F062FA0028F0D1F3E700BF10
:1011F00080841E00C3D405002DE9F341314C637E89
:101200000546002B5BD123680BB10123637695E87B
:101210000F002D4E86E80F00A27E637F2B4E23F039
:101220000303FF2A63771EBF012393404FF0A042C0
:101230004FF0000118BFC2F80C35254B217704226E
:10124000C3F808233160316800910099297939B3D6
:101250002A681278C3F81C252A79012A22D92A681B
:101260005278C3F81C2525680DBB194FDFF8548050
:10127000D7F80831002BFBD0356033680193414625
:101280003846019BFEF77CFB0028F1D1A27EFF2AA5
:1012900012D0012393404FF0A042C2F808350BE072
:1012A000E27ED7E72A7B012ADDD9E27ED9E7084B27
:1012B0000422C3F80423002002B0BDE8F08111200D
:1012C000FAE700BFBCCA0020C4CA002008310040B1
:1012D0000030004037B50B015BB249B2044643EA27
:1012E00001008DF804001A4D50B20343120152B2AE
:1012F0008DF805302B78114302438DF806108DF8D8
:10130000072013B302AB03EB941302AA13F8040CE7
:10131000C4F30113134413F8043C43EA002019F00A
:10132000F3FF2B788BB102AAC4F3810304F003040A
:101330001344144413F8040C14F8043C43EA00204A
:1013400003B0BDE8304019F0DFBF03B030BD00BFCF
:10135000CAD10020C30914BF13020B0270B510F0EC
:10136000400F0D460CBF2946114619430646122070
:1013700014461AF04FFAB1064CBF23022B0216F0A6
:10138000100F14BF21462946194312201AF042FAC1
:1013900032074CBF23022B0216F0040F14BF214664
:1013A0002946194312201AF035FAB3074CBF21021F
:1013B000290216F0010F08BF2C4621431220BDE878
:1013C00070401AF027BA00002DE9F047FF270546C4
:1013D0003C4604264FF6FF78296911B9002E61D0EA
:1013E00051E0286826F0A0FD064600284BD1686928
:1013F0000378002B5ED0C27AE52B02F03F0247D083
:1014000022F02001082943D00F2A46D159063DD5A4
:1014100003F0BF04EB88477B2B84437BBB4237D16F
:101420000378EE69DFF890E003F03F03013B0D2203
:1014300053434FF0010C00211EF8019B00EB090201
:1014400092F801A010F8092042EA0A22BCF1000F2C
:1014500020D03E2B1CD826F81320944601330131AE
:101460000D29E9D10278520604D53E2B10D800226E
:1014700026F81320013CE4B20021284627F044F866
:1014800006460028A8D000232B610CE0A342C4D05C
:10149000FF24F1E74245E2D0FAE73CB926F0D4FC5C
:1014A000B84203D100263046BDE8F0874FF6FF73FF
:1014B0002B84F8E70426E6E7E2D2050010B5074AD8
:1014C000002332F8024B8C4203D1184100F0010096
:1014D00010BD0133082BF4D10020F9E7D4C9002056
:1014E000F0B5224B9F7C1C4600221D46D6B2B74267
:1014F0000ED895F878701D4C0022D6B2B74216D897
:1015000095F8DE500022D4B2A54220D800200DE08C
:10151000B4F814C0844502F1010204F10A04E5D1D3
:1015200042F64D2301200B808870CE70F0BDB4F8D8
:101530007AC0604502F1010204F10A04DDD142F6ED
:101540004D230B8002238B70CE700120EEE7B3F8A1
:10155000E060B04202F1010203F10A03D3D142F686
:101560004D230B8003238B70CC70EEE748CC00201A
:1015700010B50C4C226886B0034682B104208DF869
:1015800004000868D989ADF80C10123333F8021C36
:101590000290ADF80E10049301A92046904706B0C2
:1015A00010BD00BF48CC00207FB54B89022B0FD166
:1015B000094A136863B1097B0068029011F0010FBA
:1015C00014BF022103218DF80410104601A9984789
:1015D00007B05DF804FB00BF48CC002070B50D4D8E
:1015E000002435F8026B964210D10122A240D2B2FB
:1015F000D543EDB2014410F8014B2BB1144388429E
:1016000000F8014CF7D170BD2C40F8E70134082CEC
:10161000E7D1F8E7D4C9002070B50023084C1A467A
:1016200041FA02F5ED0706D504EB420600EB43054F
:10163000B688AE8001330132082AF1D1036070BD53
:10164000D0C9002010B586B004460022684616F0C6
:1016500095FB2046009916F03BF9204606B010BDD8
:1016600038B501230B7004460D4636F0ADFD88B148
:1016700000220B49204634F033FB10B133F00FFE4B
:10168000287020460022074934F02AFBBDE8384084
:1016900033F084BC2046BDE8384032F041BF00BF83
:1016A000A4D30500A9D30500084B5A6E013A5A6627
:1016B00022B907490A7822F002020A701A6E013232
:1016C000042A08BF00221A66704700BF20D00020FD
:1016D0003ACC002030B5044685B00D4610220021DA
:1016E0006846FDF71FFF237A012B0AD0022B0ED08C
:1016F00063680193236829469B686846984705B04C
:1017000030BD23690293A38AADF80C30F0E70123C2
:10171000A2898DF80030E389ADF80A20D31AADF81C
:101720000830E5E728DF704729DF704738B51C4BE4
:101730005A6E19465AB31C6E182202FB04331A7AE9
:10174000012A07D0022A23D018460921BDE83840D3
:10175000FFF7C0BF1825D88A9A8A05FB0414D4E97C
:101760000314121AB2F5806F4FEA80000144B4BF2F
:1017700092B24FF480622044FFF7D6FF11280BD1BC
:10178000084A137823F0020343F00403137038BDB2
:101790009889FFF7C7FFF1E70028F8D0D4E700BF2A
:1017A00020D000203ACC0020054A137813F0060F11
:1017B00004D143F002031370FFF7B8BF704700BFB6
:1017C0003ACC00202DE9F3411F4B1B781746DA076E
:1017D000064688462BD51D4D1D4B9D4229D31D4BDA
:1017E0009D4226D239B330B341EA00039B0724D18E
:1017F0002B68984223D36A6800EB87039A421ED372
:10180000FFB101A8FEF70EFE78B1019B0024C3E9E9
:101810000054019B01221A72C3E903869F82FFF7DD
:10182000C3FF204602B0BDE8F0810720FAE701209F
:10183000F8E70220F6E70320F4E70620F2E70520A8
:10184000F0E70420EEE700BF3ACC0020202D002076
:10185000202D0020302D002038B5074B074A59684D
:10186000948810684A880332032592B200EB840002
:101870001D70FFF7A7FF38BD3CCC0020C4D000206E
:1018800010B501220C460649FFF79CFF28B905490F
:1018900001EB041101238B7310BD0E20FCE700BF88
:1018A0000CD5050080CF002008B502220149FFF7C2
:1018B00089FF08BD10D5050008B5034B034918681A
:1018C0000222FFF77FFF08BDC4D0002018D5050015
:1018D00073B51B4B1B78DB0705462BD5194E1A4BEE
:1018E0009E4229D3194B9E4226D238B3C0F30B0433
:1018F000D4B93368984219D3726800F580539A427C
:1019000014D301A8FEF78EFD90B1019BC3E90064DA
:10191000019B02221A722D0B01229D811A82FFF770
:1019200043FF204602B070BD0620FBE70520F9E723
:101930000720F7E70120F5E70220F3E70320F1E7AE
:101940003ACC0020202D0020202D0020302D00201A
:1019500010B50B4C0B4B628803EB02139A892AB922
:101960005868FFF7B5FF0423237010BD05232370CB
:10197000054B022218689A80FFF7AAFFF5E700BF1F
:101980003CCC002080CF0020C4D0002008B5074BFD
:10199000191D5888FDF71EFE18B1BDE80840FFF775
:1019A0005BBFBDE80840FFF7D3BF00BF3CCC0020C1
:1019B00060DF704710DF7047002208B5114618F04D
:1019C000F3FE00002DE9F347254B1B681BB1984738
:1019D00030B3FFF7F1FF234B1B7803F0FF07FBB198
:1019E000214D224E2C68DFF88C90B4FA84F46409FF
:1019F000B0463378A3B901A8FDF7D0FD052812D071
:101A00000028E6D1019B0BB9FDF7A4FF184B1B681A
:101A10000BB1019898474CB10124EAE7002CFBD0A8
:101A200002B0BDE8F087002CFAD13C46DFF848A0B0
:101A300098F80030002BF3D1B9F80030ADF804303D
:101A4000DAF8003001A91846FDF7A6FD0528E5D013
:101A50000028BED12A6818469047002CE8D1C8E774
:101A600028CC0020C1D0002008CA0020C2D000200D
:101A7000CCD0002004CA0020B4D1002010B5084BFF
:101A80009A685AB150B9EFF3108172B6054A1C68D2
:101A900014605C685460986001B962B6002010BDA3
:101AA000BCD1002000E100E02DE9F3411D4F7B682F
:101AB00006460D469BB304292FD943697BB3437C6B
:101AC0000024012B0DF107000CBF8846A0468DF8BD
:101AD0000740FFF737FB0DF10600FDF709FED0B117
:101AE00001230370104B4660D3F80435C0E9048429
:101AF000C0E902359DF806307B709DF80700FFF7BE
:101B0000BDFF24B9094B4FF48012C3F800212046D1
:101B100002B0BDE8F0810424EFE70724F7E70824CA
:101B2000F5E700BFFCCE00200010014000E100E01E
:101B30002DE9F341CE0801F007044FF0010808FA3F
:101B400004F4855DE4B22540074613D10DF107008A
:101B50008DF80750FFF7F6FABB5D9DF807001C42B1
:101B600002BF1C43BC554546FFF788FF284602B01C
:101B7000BDE8F0810025F9E72DE9F347814600270C
:101B800001261FFA87F84FEAD80A08F0070406FA78
:101B900004F419F80A50E4B2254008D00137B7F52B
:101BA000807FEED1B846404602B0BDE8F0870DF127
:101BB00007008DF80750FFF7C5FA19F80A309DF8AD
:101BC00007001C4202BF1C4309F80A400125FFF729
:101BD00055FF002DE2D0E6E773B50546B8B1C1F375
:101BE000C70401F0070301269E40035D33420ED077
:101BF00000230DF107008DF80730FFF7A3FA2B5DE6
:101C00009DF8070023EA06062E55FFF737FF02B0BE
:101C100070BD000038B50A4B1A687AB15D686DB1C5
:101C2000FF280BD084B221462846FDF79BFD28B142
:101C300021462846BDE83840FFF7CEBF38BD00BF7B
:101C400004D100202DE9F74F9846531E072B8146FB
:101C50000F46154600F2BB80FF2800F2B88001460F
:101C60005E48FDF77FFD0646002800F0B08039464B
:101C70004846FDF7C9FD044600283ED0C3689D4292
:101C800047D805D25FFA85F9E368207C994543D3AC
:101C900094F81090B9F1FF0F40F09780504B1A68FC
:101CA0009B46002A41D14FF6FF732380A370002387
:101CB000C4E90133E360238A03F4784343F0FF036C
:101CC0002382112084E0237C1844C0B2FFF7A2FFD6
:101CD000E3685FFA8AF083420AF1010AF3D84FF60B
:101CE000FF732380A3700023C4E90133E360238AD8
:101CF00003F4784343F0FF032382FF214FF6FF7084
:101D0000FDF782FD04460028DBD0A0F80090877024
:101D1000BEE74FF0000ADBE74844C0B209F1010911
:101D2000FFF778FF5FFA89F9AEE75B68002BBAD05E
:101D30000023DBF808205FFA83FA924502D34FF0C4
:101D4000FF0912E0DBF8040060B351460193FFF78E
:101D5000EFFE019B30B3B9F1FF0F08BFD146AAEBEC
:101D6000090A0AF1010AAA4521D1B9F1FF0F84F845
:101D7000109098D0E560207CFDF704FD58B305EB8A
:101D800085052D01ADB2AD0888F80270C8F80400D1
:101D9000A8F8005026B1082F02D1AD00063D85807D
:101DA000002015E0B9F1FF0F0CD14FF0FF0901330E
:101DB000BFE74846019309F10109FFF72BFF019B9B
:101DC0005FFA89F9D145F4D3EFE70026D2E707207F
:101DD00003B0BDE8F08F0320FAE700BFD8CF0020A2
:101DE00004D1002038B504460025E368AB420ED884
:101DF0004FF6FF732380A3700023C4E90133E3602F
:101E0000238A03F4784343F0FF03238238BD207C08
:101E10002844C0B2FFF7FEFE0135E6E737B5FDF70F
:101E2000F3FC0546A0B144682CB10A4B01941B7821
:101E30009B0706D403242846FFF7D4FF204603B0AF
:101E400030BD01A8FDF7ACFB04460028F3D0F1E754
:101E50000524F3E739CC0020FF2810B5044609D843
:101E600001460548FFF7B8FE21460448BDE810408A
:101E7000FFF7B2BE10BD00BFD8CF0020F8CF0020C2
:101E800013B50DF106010446FDF7CCFB70B1BDF8AA
:101E90000620084B03EB02139A894AB1A17A39B1A3
:101EA000013A00209A81A07202B010BD0A20FBE71F
:101EB0000620F9E780CF002037B50D460DF1060169
:101EC0000446FDF7AFFB88B1BDF80620084B6168FA
:101ED00003EB021300209A8901329A81296063681A
:101EE0000C336B600123A37203B030BD0A20FBE703
:101EF00080CF00202DE9F043DFF88480D8F874E02B
:101F0000BEF1030F0F46944635D81C4E756CC1F1D7
:101F100008039D422FD8D8F8704074441C2304F065
:101F20000304814603FB0484B9E80F000FC499E859
:101F300007000EF1010384E80700C8F87430C7B148
:101F4000336C2B4403F0070306EBC303002206F1B6
:101F500038040CEBC20103C9A34202F1010283E879
:101F6000030014BF0833054B9742F2D1736C1F4432
:101F70007764012000E00020BDE8F08300CB002062
:101F800004CF00202DE9F0411C46184B1B789B071D
:101F900006460F46154627D5DFF85880A3880BB1B3
:101FA0000A201FE098F800302BB92146A088FDF7E1
:101FB00011FB20B92060A3880133A380EEE72368DA
:101FC0001EB1998832889142EFD11FB119883A88A1
:101FD0009142EAD19B682B6023686B60044B1B899C
:101FE0002B810020BDE8F0810220FBE739CC0020E6
:101FF0003CCC002080CF002030B587B04CF20703E6
:1020000005460C46ADF8043003AA0F4B01A9002089
:10201000FFF7B8FF10B1002007B030BD01A903A839
:10202000FFF74AFF0028F6D10723A370019B5A88C7
:102030002280029A62609B8803F580432B8003A86C
:10204000FFF71EFF0120E7E72CCC00201FB500237F
:10205000A0F58040A1F58041CDE90233ADF8040040
:10206000ADF8061002AB0DF1060101A8FFF78AFFDB
:10207000002818BF052005B05DF804FB2DE9F041EC
:1020800002230B80164B00251C6800F5805E2F464E
:1020900008304FF6FF7870450AD305B11C6002B1D5
:1020A0001770BDE8F08101270EE0344601250BE0F2
:1020B00006680136F1D086884645F4D00688002EA1
:1020C000F1D08668A642F0D8468806F1030C00EBF2
:1020D0008C00B1F800C00CF1030C66440E80DAE706
:1020E000C4CD002070B5064D0646002455F8043BCB
:1020F0000BB1304698470134082CF7D170BD00BFB2
:10210000DCCA00202DE9F047AA4C266F1C2707FBEC
:1021100006F586B0635D013B8046052B00F22A81FF
:10212000DFE813F00600640064001D011D017E015C
:1021300030B1A14A137823F00103137001201FE08E
:1021400025442B79032B15D8DFE803F002072C3444
:10215000FFF7B2FB01232B7109E0984D2B78022B7E
:1021600040F03C826868FFF79FFB00232B7000283B
:1021700000F0F080904A137823F0010313700E20D2
:102180001C237343E218E35C0290023B012B00F234
:1021900032818B4B907D196C5A6C0144121A196470
:1021A0005A6428E1874F3868FFF792FB0223BB800F
:1021B0000023D0E7834FDFF804823868FFF774FB11
:1021C000814BD7F800E05B88B7F804C01B0108EB2F
:1021D00003025168A2F808C0C2F804E00222BA80E3
:1021E0000022396008F803202A71C0E707FB064780
:1021F000724BB7F812A04FEA0A1A03EB0A0299468B
:10220000118960B1FB8803F103088844C3F57F435B
:102210005189A2F80880FD330B4453818EE753683F
:1022200003EB81083B7C062B00F29780DFE803F08C
:102230002D733C4D1F84040041F61D501C2303FBED
:102240000643D144DB88B9F80810DA1C0A44A9F81F
:102250000820C3F57F43B9F80A20FD331344A9F8D9
:102260000A3041F61D53984200F0C38088E7574872
:102270005749002343601C2303FB06439B6903600B
:10228000FDF7D0F9002800F04C81291D01222144DE
:102290004046FFF797FA1C2303FB064302221A74F9
:1022A000002857D00E20C9E705F10C010122214476
:1022B00008F10800FFF786FA1C2303FB06439A7D0A
:1022C000002A14BF03220122E9E73D4B5A6C002A81
:1022D00000F08C81196C1C2505FB0645481C00F09C
:1022E000070003EBC1071864A88A53F83110013ABC
:1022F0005A6408EB8000BA88FFF764FAAB8ABA88A0
:102300001344AB82AB7D013BDBB2AB75002BC7D175
:1023100001232B74C4E705F108010122214408F1CF
:102320000400FFF74FFA1C237343E25C032A0CBF3F
:10233000052206222344B2E7254B1988234B58680F
:10234000FFF79EFA1C2303FB064306221A7400289B
:102350007FF474AF06B0BDE8F0870F206EE7002869
:102360007FF4ECAE07FB06473B79012B32D01BB163
:10237000022B3ED00F2003E7CDE90200FB6801935A
:102380000DF1020101A8FDF74DF980B10298BDF8E9
:1023900002108388FB8003883B81FFF771FA1C23BE
:1023A00003FB064302221A710028D3D059E70A2002
:1023B000F5E700BF04CF002039CC002080CF0020FB
:1023C00000CB0020C4D000203CCC00205C2D00209D
:1023D000C8D10020864FA81D3B4601AA4146204493
:1023E000FFF7D0FDB8B9B9880298FFF749FA0A2873
:1023F000DAD1002302931C2303FB06F2A25C013A0C
:10240000052A00F2B580DFE812F08E009200A000ED
:10241000CB00D500E1000A28C7E90088E9D020E711
:1024200000287FF48BAE734BDA7AAAB1D8721A788F
:10243000013A062A9ED801A151F822F0ED240200AB
:10244000E7240200FD240200032502007523020098
:1024500009250200192502001A78072AE7D801A1E8
:1024600051F822F0852402002F2402002F240200BC
:10247000A1240200B5240200D3240200D3240200C8
:102480009D2402001A8901321A8100225A80DA72D0
:10249000594A1278B2FA82F252099A72012207E07E
:1024A000564958688A884088033202448A8002224A
:1024B0001A70BCE75D88504A504902EB0512086863
:1024C000556850608888108102228A800D6006223B
:1024D000EEE70722ECE7484900229A728A8942B95E
:1024E000897B31B15A80FFF751FA5DE79A7A002A69
:1024F000F1D100221A705A805A607AE7FFF7ACF9DE
:1025000052E7FFF725FA4FE75A883B4B03EB0213DC
:102510005868FFF7C9F947E700225A60FFF7CCF97E
:1025200042E70A202CE600238DF8043020E003FB6C
:10253000064301228DF804201A89ADF810209A88EC
:10254000ADF81220DB68039312E003FB064302227E
:102550008DF804201A89ADF810209A88ADF8122061
:10256000DA681B7C03929A1F534253418DF8143052
:1025700001A8FFF7B7FD206F1C22002102FB0040DD
:10258000FCF7D0FF636F1BB3226F013202F003022E
:10259000013B22676367DBB10020FFF7B3FDD9E69B
:1025A00003FB064303228DF80420DA88ADF81020DF
:1025B0001A89C5E703FB06430422DB88ADF8103017
:1025C00000238DF80420ADF81230D1E70523ABE7E6
:1025D0000B4A137823F004031370BBE6084A137800
:1025E00043F0020323F00103137002E71368FFDED8
:1025F000D0D100203CCC002080CF0020C4D00020CF
:1026000039CC00200846FFF77DBD0000054A13784D
:1026100013F0040004D143F004031370FFF772BDFC
:10262000704700BF39CC0020F0B51C463D4B1B78ED
:102630009E0789B007460D466FD509884FF6FF7390
:1026400099426CD06B88002B69D06968B5F808C0D6
:1026500000239C4503D8BAB9164604310AE051F864
:102660003300800757D10133F3E731F832003044AB
:1026700086B201329445F8D80DF102013046FDF7DB
:1026800019F828B109B0F0BD13885688ADF80230AA
:1026900000238DF81430BDF80230ADF81630032356
:1026A000ADF81830204B8DF804401A6829898DF850
:1026B0001A1001321A602B88ADF80C30032C6B888D
:1026C000ADF8083004BF04238DF81430049208BF1D
:1026D0003B686A6808BF0793002401A8ADF80A6048
:1026E000ADF80E40FFF706FC50B9BDF802200F4BC5
:1026F00003EB021358890338801B58810820C1E777
:10270000049B3B600A4B7C601B89BC723B81FFF7DA
:102710007DFF2046B6E70320B4E70220B2E704209D
:10272000B0E700BF39CC0020C4CD002080CF00200E
:102730003CCC002030B58BB0FF28044601921D46EA
:1027400045D88B781846FDF735F800283FD04A6801
:1027500002920A88ADF80C20A4F58042ADF81C2046
:10276000A3F58042ADF81E2002AA08920122ADF81E
:102770002420194604AA2046FFF768FC0528019A80
:102780000ED1022352B907A904A8FFF74DFF07286D
:102790001FD010D8B0B103200BB030BD01AAF2E7B2
:1027A00032B10E4B1B789B0702D501A8FCF7F8FE4F
:1027B00003230022E7E708280DD00E280CBF1120C4
:1027C0000320E9E7002DE7D0049B2B60E4E7072016
:1027D000E2E78620E0E71120DEE700BF39CC0020E9
:1027E0001F4B204A1B6800BF00BF00BF00BF00BFD7
:1027F00000BF00BF00BF93422FD000BF00BF00BF8B
:1028000000BF00BF00BF00BF00BF00BF00BF00BFD0
:1028100000BF00BF00BF00BF00BF00BF00BF00BFC0
:1028200000BF00BF00BF00BF00BF00BF00BF00BFB0
:1028300000BF00BF00BF00BF00BF00BF00BF00BFA0
:1028400000BF00BF00BF00BF00BF00BF00BF00BF90
:1028500000BF00BF00BF00BF00BF0138C3D1704739
:10286000A42C00200024F40073B5154E73680546AF
:102870001BB343690BB3002404740DF107008DF8FA
:102880000740FEF75FFC0DF10600FCF731FF90B149
:10289000022303709DF80630456073709DF80700B1
:1028A000FFF7ECF824B9074B4FF48012C3F800216E
:1028B000204602B070BD0424F0E70824F8E700BF0A
:1028C000FCCE002000E100E02DE9F8432649274B2B
:1028D0000025C1F84051C1F84451C1F84851C1F830
:1028E0004C51C1F80051C1F804511B68002B39D07C
:1028F000D1F804451E49DFF88C800968641A24F079
:102900007F442F461A68A24217D8A41A15441A7C8D
:10291000DE6982B1D8F800901F74D3E90521B9F1BE
:10292000000F06D01046C84728B1FFF745F83346D8
:10293000E8E708469047002EF9D10E4A0E4B117871
:102940001B788B4205D10133DBB2022B08BF002379
:1029500013701278094B43F82250094B4FF4801240
:10296000C3F80021BDE8F88300100140B8D1002071
:10297000DCD00020D9D00020D8D00020D0D000203A
:1029800000E100E024CC00200D4B0E494FF4003252
:1029900010B5C3F8802001244FF48033C1F84833C8
:1029A0002F20C1F808334C60FFF71AFF064B8C60EC
:1029B0002F2000211960FFF713FF044B197010BD81
:1029C00000E100E000100140DCD00020B9D0002080
:1029D0002DE9F04FB64AB74913780978B64D85B05E
:1029E0009942D5F80080019500F095800133DBB263
:1029F000022B08BF002313701278B04B53F82260EB
:102A0000019A08EB060323F07F4313600127AC4BC8
:102A1000AC4A18680290AC48117890F800904FF0DA
:102A2000000CE2465078884278D1BCF1000F02D009
:102A3000A54981F80090002F40F0BB801F680299E3
:102A40007F1A18BF01270020196802919E4903913F
:102A500091F800E000244FF00108002840F0AD801C
:102A600092F80190D2F804C092F802A0117849457A
:102A700040F0C1801B68029A9A4201D1002F44D0D5
:102A8000002B00F01281D3F80090904C019BD4F8F9
:102A9000046519688E4F751A3B7825F07F4503351C
:102AA000A3B94FF48033C4F84433C4F80433894BDA
:102AB0004FF400324FF00108C3F880212F201A6034
:102AC000C4F80080FFF78CFE87F80080A9452CBF72
:102AD0004944491921F07F41C4F84015D4F8043520
:102AE0009B1B23F07F43891B033321F07F418B42E3
:102AF0000BD9D4F80435C4F840352F20FFF770FE09
:102B0000744B4FF40032C3F80021039A0023137072
:102B100005B0BDE8F08F0026374678E701EB4104A9
:102B2000506892F802B000EBC40E013110F8344046
:102B30001868C9B28B4508BF0021022C04D0032CB1
:102B40007FF470AF002410E0DEF804B0044686463F
:102B5000002C3FF467AFA34500F0C080A646E469AF
:102B6000F6E780F810A0C06901240028F9D1002CF4
:102B70003FF458AF186055E7D4F80C90C4F800E063
:102B8000761A8C44E1691960B9F1000F07D008EB9F
:102B90000C0121F07F41C4E90119E06120461C6865
:102BA000002C3FF451AF2168B142E5D98E1B26605D
:102BB0004AE7002084468646F1E70146C069019D48
:102BC000D1F804A02E68444DD1F80890AAEB060C69
:102BD0002CF07F4CAC4535D80CEB09060E60D3F8D1
:102BE00000C081F81080C1E90144CC61BCF1000F44
:102BF00033D1196031E701EB410B0131C9B25145C5
:102C000014BF117014701CF83B1001290CEBCB069B
:102C10007FF42CAF716891F810B0BBF1000F7FF416
:102C200025AFD6F808C0C1F804C0F5688D603569D5
:102C3000CD6076698E61BEF1000F0CBF66465E46C0
:102C40004E60BCE7A6EB0A0626F07F464E4502D250
:102C5000A9EB0606C2E70C60C1E7D1F80090DCF8EA
:102C60000060B1451FD8A6EB0906CCF80060C1F89A
:102C70001CC0BEE7A9EB0A09D6F81CA0B446BAF1FD
:102C8000000F0AD05646D6F800A0CA45F2D3AAEBE8
:102C9000090AC6F800A0B2466646C1F80090C1F81D
:102CA0001CA0F161D9E66646EDE7FFF76DFE2CE763
:102CB000D8D00020D9D00020DCD00020D0D00020F7
:102CC000B8D10020FCCE0020B8D000200010014078
:102CD000B9D0002000E100E0FEFF7F0074450FD175
:102CE000D0F81CB0C3F800B0BBF1000F08D10A4DFA
:102CF0000120A86001984FF0010CC0F800B0E14637
:102D00002068E469CEF81C40002C3FF48BAE2568A7
:102D10002844206086E600BF0010014037B5074B0D
:102D2000054693E803006C46002384E803001A4636
:102D300021462846FFF7FEFC03B030BDC0D2050097
:102D4000FDF78CBB10B54FF6FF7304469C42084656
:102D500009D1FEF711FFB0F5807F044601D14FF68F
:102D6000FF74204610BDFF2CF9D82146FEF7E0FE87
:102D70000028F6D1F3E710B5044601F0EFFC204639
:102D8000BDE8104000F02EBF1FB5037893B902795B
:102D9000072A0FD1448803932046CDE901338DF8EB
:102DA0000420FCF7C9FCADF8060001A8ADF8084006
:102DB000FFF7E1FF04B010BD1FB50023CDE90133DB
:102DC0000393ADF80600022301A88DF804308DF8B6
:102DD0000810FFF7D0FF05B05DF804FB86DF7047F1
:102DE00038B504884CB9821C00F10A0512F8013B81
:102DF0001BB99542FAD100200AE00B88A342FAD110
:102E00000822023102303AF0E7F9B0FA80F04009C6
:102E100038BD08B570B171B103780A78534013F02A
:102E2000FE0F08D10622013101303AF0D5F9B0FA8F
:102E300080F0400908BD0020FCE710B5044600F012
:102E4000BDFF2046BDE8104000F04ABF43DF704799
:102E50006FDF7047024B0022C3E90022704700BFBA
:102E60002CCC0020F0B5FF2887B004460E4615464E
:102E70001F4629D80846FCF79DFC28B303AA204624
:102E8000FFF7E4F818B10524204607B0F0BD01A90A
:102E900003A8FFF711F804460028F4D1019BAE7097
:102EA0005A882A805FB13B6892009A420AD30299FD
:102EB00068683AF09FF903A8FEF7E2FFE4E7029B97
:102EC0006B60F8E70424DFE70724DDE72DE9F04134
:102ED000CEB020AE502380460CADB8220021304643
:102EE00001930395FCF71EFB0DF1970305930DF17C
:102EF000AE0306930DF1C503079337AB08930DF1AD
:102F0000F30309930DF585730A931C4F04960DF294
:102F100021130B930024444507D1E2B2002104A8F9
:102F2000FFF796FF4EB0BDE8F08150220021284601
:102F3000FCF7F8FA01AB02AA072137F8020BFFF7FA
:102F400091FF20F002000528ECD06B7C032B12D8F7
:102F500017230DF1310203FB04630DF1450152F813
:102F6000040B43F8040B8A42F9D111881980927836
:102F70009A700134CFE743F20220D3E7E2D0002079
:102F80002DE9F04110220546A6B000212D48FCF79E
:102F9000C9FA35B929462846FCF7E2FB26B0BDE858
:102FA000F0816A0028492748DFF89C8004AE3AF097
:102FB00021F9382200213046FCF7B4FA00245023CE
:102FC000CDE9013412AF0397502200213846FCF7B7
:102FD000A9FA01AB02AA072138F8020BFFF742FF5A
:102FE00020F002000528D9D09DF85930032B26D8AF
:102FF000C4EBC402B318DDF85910B1500134BDF868
:103000005D209A80A5429DF85F209A71DCD10DF178
:10301000170313930DF11E0314930DF1250315935C
:103020000BAB16930DF1330317930DF13A0318937D
:103030000DF1410312961993E9B23846ACE743F219
:103040000220ABE7F2D00020E2D000202DE9F043CF
:10305000037889B00546002B3FD1017907293CD17F
:1030600004AA4088FFF7FEFEB8BBFFF7F3FE02A9F3
:103070000DF10600FEF7C0FF78B36E88BDF806704C
:10308000BE42F4D0059C631C1846113413F8012B82
:1030900012B9A342FAD1EAE7DDF80C80102208F158
:1030A00001013AF099F808F1110181462046FFF735
:1030B000B0FEB9F1000F01D00028D8D03046FCF79F
:1030C0003BFB0023ADF81A0006A88DF81830ADF8C8
:1030D0001C60ADF81E70FFF7B0FE09B0BDE8F083CC
:1030E000CA1F012A73B5064654D80025CDE90055FC
:1030F0008DF80210FCF788FB044600284CD0437C76
:10310000DB074BD4007CFCF73DFB10B9032002B079
:1031100070BDE368019003EB83031B019BB29B0826
:103120006846ADF80030FCF74DFB626804F1080317
:1031300069463046FFF7FEFA637C03F00603062B70
:1031400001BF174A136803F1FF33136030B9637C82
:1031500023F0070343F001036374D8E711280BD170
:103160000F4A136801331360637C23F0060343F0B6
:10317000040363740020CAE7862809D1084A13684B
:1031800001331360637C23F0060343F00203E3E79B
:103190000728BBD10720BAE70520B8E72846B6E7DD
:1031A000CCCD00202DE9FF410546102200216846C4
:1031B000FCF7B8F968882979ADF802008DF8041099
:1031C000FCF722FB2B78454E092B5ED8DFE803F095
:1031D0000505684D4D6C7173757D00283FD0437CAB
:1031E000DC073CD5FEF7FEFD2B78581E43424341D9
:1031F000002468468DF800408DF80830FCF7F6FA98
:1032000033684BB3364E002537464FF0140808FBA1
:1032100005735B7C5A0703D49B0759D5002C57D004
:10322000B1783088FFF75CFF002851D014235D434C
:103230007B1986289B788DF804307A5B16BF029044
:10324000082309236846ADF802200CBF8DF8003032
:103250008DF80030FCF7CAFA04B0BDE8F081012314
:103260008DF80030AB68029316E080B18268AB68DD
:103270009A420CD1437CD90709D5326823F0050363
:10328000013243F00403326043740024B8E70223A0
:103290008DF80030EB6803936846FCF7A7FAF4E773
:1032A00003238DF80030F7E704238DF80030EB6836
:1032B000D9E70523F5E70623F7E7072368468DF8E6
:1032C00000300124FCF792FA9AE7EB680293DCE7FE
:1032D0000135082D06F1140699D1BDE7CCCD0020AB
:1032E00014D1002070B500238CB02D492C4E4FF620
:1032F000FF70CDE90033FCF7F9FA4FF6FF7504468D
:10330000AC420BD0A4F58043ADF8143002AA6B4652
:10331000002105A8FEF736FE0A2822D0214B1A7894
:103320001846E2B94FF6FF718C4218D01E4E36781F
:1033300001251D70B607A4F580439BB21DD58B42B5
:103340002CD005218DF8141005A811468DF81850C1
:10335000ADF81A30FEF7CEFD60B1FFF757F90CB0AB
:1033600070BD2046FEF778FD20463146FCF7BEFAD8
:103370000446C5E70D4B1D70F1E702230022092129
:1033800002708DF8141005A8FF21ADF816408DF8D5
:103390001810CDE90723FFF705FFE0E70423EDE769
:1033A000F8CF002091CF002039CC002092CF002010
:1033B000F0B5426805783D4C85B0B2FA82F1490912
:1033C0000391691E0346042924D8DFE801F00303B2
:1033D00030496A009989DE8901F5804189B243F656
:1033E000FE77B94204D906F5804080B2B84211D8C0
:1033F000012DADF802108DF8046013D1002A14BF1E
:10340000032100218DF8001003929B680293684607
:10341000FFF7C8FE23781BB100232370FFF762FF7C
:1034200005B0F0BD002A14BF04210121EAE7998903
:10343000DD8901F5804189B243F6FE76B14204D9B7
:1034400005F5804080B2B042E4D8002A0CBF0222C9
:103450000522ADF802108DF804508DF80020D4E755
:10346000988900F5804080B243F6FE718842D1D839
:10347000DB89002BCED1FF23ADF802008DF804309C
:103480005AB906238DF80030FEF7E6FC084A0023FF
:1034900023701370FFF726FFB9E707238DF800307C
:1034A000F4E708238DF80030B1E700BF92CF002089
:1034B00091CF0020F8B50D490D4DFCF717FA4FF6E6
:1034C000FF760446A5F12007B44201D12046F8BD9D
:1034D000FF2CFBD821462846FCF744F90028F5D0FC
:1034E00020463946FCF702FA0446EDE7D8CF002023
:1034F000F8CF002073B5104B104C93E803006D46D5
:10350000002385E803001A4629462088FFF712F9B0
:103510004FF6FF762388B34201D0112801D102B0C3
:1035200070BD1846FFF7C6FF00231A4629462080C3
:10353000FFF700F9EEE700BFC8D2050014CC002069
:103540001FB50378012B044615D10179012912D149
:10355000002302AA4088FFF785FC60B902238DF89A
:1035600000306388ADF80230039B68461B788DF805
:10357000043000F0B5FD054B1A884FF6FF739A42F0
:1035800001D0FFF7B7FF04B010BD00BF14CC00207E
:1035900070B504468AB0142200216846FBF7C2FFCA
:1035A0006588ADF804502846FCF7C6F82378ADF8D6
:1035B0000200092B15D8DFE803F005163048525EEB
:1035C0008614A1A507238DF8003023798DF80830E3
:1035D0009DF80A3043F001038DF80A306846FCF785
:1035E0009FF90AB070BD07238DF8003023798DF85C
:1035F00008309DF80A30444AA168039143F0010362
:103600008DF80A301368002BE8D09942E6D10023E8
:1036100013603E4A03931580E0E708238DF80030DD
:1036200023798DF80830E3680493374BA1681A6852
:103630000391002AD2D09142D0D1354900221A609C
:103640000B680392013B0B60C8E707238DF800303D
:1036500023798DF8083001238DF80930BEE708235F
:103660008DF8003023798DF8083001238DF809306A
:10367000A3680493B2E7274D09238DF800302B7817
:10368000002BABD04FF6FF70FFF714FF4FF6FF7320
:1036900098420646A2D12049FCF728F9B0420446D8
:1036A0009CD1142200210DEB02002970FBF73AFF98
:1036B0000B238DF81430ADF81840ADF8164005A86E
:1036C000FCF72EF98AE70A238DF80030114BA46825
:1036D0001A780294002A81D0142200210DEB0200F6
:1036E0001970FBF71FFF0C238DF814304FF6FF7392
:1036F000ADF81830ADF816300794E0E705238DF8E3
:1037000000306BE70623FAE7D4CF0020C0CD0020BD
:1037100010CC002016CC0020F8CF00202DE9F04777
:10372000474B1B788AB00546002B00F08780454B3D
:10373000454F93E803003C7803AE86E80300BCB92C
:103740004FF6FF70FFF7B6FE0123ADF8143001AB62
:1037500006930423029305AA02AB06218046019436
:10376000ADF81640FFF77EFB07284AD101233B70D6
:10377000364B1C689846002C5AD1354A354F128872
:103780003B68AA4241D1002B3FD0142221460DEBC9
:103790000200FBF7C7FE072328468DF81430FBF71D
:1037A000CBFF0623ADF8160005A8ADF818508DF82C
:1037B0001C30FCF7B5F820460AB0BDE8F087CDF81C
:1037C00004A0019B4046A34224BFC1461C46FFF70C
:1037D00071FEBDF814309B00029305AA02AB0621CE
:1037E0008046FFF73FFB0028EBD00528E7D04FF6D7
:1037F000FF7398451CD1164BA3F80090154B1C6025
:10380000B4E74FF6FF79A246EDE701333B600022B3
:103810000E4B31462846FEF78DFF0028CCD0002302
:10382000C8F800303B68112803F1FF333B6001D139
:103830001120C1E7862818BF0320BDE70820BBE799
:10384000C8CD0020D0D20500D3CF0020D4CF002097
:10385000C0CD002010CC002063DF7047A6DF70478A
:10386000A2DF70472DE9F04391B0984611238DF8FF
:10387000043013788DF805300024164601254FF0EA
:10388000000365F34203074689461C22214609A826
:103890008DF80630FBF746FEB3788DF80930C3F398
:1038A0000302A24214BF1A2212228DF8242001AA78
:1038B0000E9203AB72788DF808200493224602AB77
:1038C00065F34202059308238DF80A20CDE90644EA
:1038D00004AAADF81C3009A9434638888DF80E506B
:1038E000ADF80C900894FFF7BBFF11B0BDE8F08372
:1038F000A0DF7047044A0123116883400B401ABFC0
:103900001218507E18467047D0C9002070B4094D77
:10391000134601262A6806FA01F4144207D001F181
:10392000190402463146281970BCFDF757BE70BC19
:10393000704700BFD0C900201FB50023CDE9013377
:1039400003938DF80A201A46074BADF80810062499
:103950001978ADF806008DF80440FFF7D7FF01A8ED
:10396000FFF709FA04B010BDAF2C002010B4084ACC
:10397000012314688B40234006D00A445DF8044BB1
:103980000146507EFDF79ABD18465DF8044B70471E
:10399000D0C9002010B50A4B19780446FFF7E6FF9E
:1039A00058B1084B00205A88A24201D1C0B210BDC4
:1039B0000130082803F10C03F5D1FF20F7E700BF21
:1039C000A4CB0020A6CB00202DE9F8430546FBF749
:1039D000B3FE234B074600221420984600FB02F159
:1039E000CC5AAC422AD10B44002634464FF014097D
:1039F0005BB199782846FEF711FA10B1052818BF77
:103A0000032401363246072A1DD9A4B9FF2D24D834
:103A1000144928464FF6FF75FFF794F9FFF762FC4B
:103A2000AF4208D03846FFF7B5FFFF2803D00C237C
:103A300043430D4AD5522046BDE8F8830132082A97
:103A4000CCD10023D0E709FB02F338F80310A942D8
:103A500001D14344CCE70132D5E70724EBE700BFAF
:103A600014D10020F8CF0020A6CB00202DE9F04192
:103A70001F46154B9DF818400E469046197805468E
:103A8000FFF744FFB8F1000F17D0104B3A461978F2
:103A90002846FFF73BFF0E4B224619782846FFF7D2
:103AA00035FF44B12846FFF775FFFF2803D00C23EC
:103AB0004343084AD652BDE8F081002CFBD0304683
:103AC000BDE8F041FFF780BFAF2C0020B12C0020F3
:103AD000B02C0020A6CB002008B5FFF75BFFFF2825
:103AE0001DBF0C234343034A4FF6FF7018BFD05A43
:103AF00008BD00BFA6CB00202DE9F04385B00546E8
:103B0000FFF7EAFF4FF6FF739842074641D00122C4
:103B10004FF0030901AB0821384602F10108FEF716
:103B200091F81FFA88F8064648BB02990A46032313
:103B300042F8049B06312846FBF7F2FD044660B9C3
:103B400008213846FFF7CCFA0446112C3FD01AD88A
:103B50000CB30C2C2FD107231EE00C280DD0052808
:103B600000D1344608213846FEF758F9002818BF1E
:103B700003244246002ECDD1E7E70126F2E70728CD
:103B8000E9D00446E1E7862C13D043F202039C42BD
:103B900011D100221CE0012328468DF80430ADF835
:103BA0000850FFF799FFADF8060001A8FFF7C8F825
:103BB000EFE70823F0E7092328468DF80430FFF7E4
:103BC0008BFFADF80850ADF806000394EDE7012235
:103BD000034B28461978FFF799FE05B0BDE8F0833E
:103BE00036CC00200378072B02D14088FFF784BF32
:103BF000704700002DE9F0434FF6FF75A84285B0ED
:103C0000044668D0FFF768FFA84227D100260327A3
:103C1000B0464FF001093B46324641462046FBF78D
:103C200081FD042805464DD0082847D00B282DD10A
:103C300017F002031FD1B8F1000F20D11EBB0323E0
:103C400020468DF80430FFF747FFADF80840ADF887
:103C5000060001A8FFF774F8002237E0002301AA4C
:103C60000821FFF7FFF80028D0D1029B03F10608D6
:103C70009E881F68CDE701274FF00009CBE7032797
:103C80001E469846F8E703274646F5E7B9F1000FC8
:103C9000D5D0112819D043F202039842DCD008B9DC
:103CA0000223CDE7092320468DF80430FFF714FFE7
:103CB000ADF80840ADF806000395CAE7B9F1000F6A
:103CC000EED1BCE7B9F1000FB9D00122034B204679
:103CD0001978FFF71BFE05B0BDE8F08335CC002056
:103CE00037B50578012D044614D14088FFF782FFCF
:103CF0006088FFF7F1FE00236A462946FFF7B2F815
:103D000040B9019B1B782BB1034B608819782A4678
:103D1000FFF7FCFD03B030BD37CC0020F0B587B015
:103D200004460E461746FFF7D7FE4FF6FF7398423C
:103D3000054624D01E4B20461978FFF717FE80B3A6
:103D40000023CDE90033029304238DF80030194B92
:103D5000ADF802401978ADF8046020468DF8067081
:103D6000FFF704FE68B12846FFF72EFE124B2046EF
:103D700000221978FFF7CAFD6846FEF7FCFF07B07E
:103D8000F0BD07212846FEF749F80528EED10923A2
:103D9000049003A88DF80C30ADF80E40FEF7EBFF51
:103DA000E4E73A4631462046FFF7C6FDE7E700BFA5
:103DB000B12C0020B02C0020AF2C002010B50278D0
:103DC00086B004461AB1012A09D006B010BD0E4BC8
:103DD0001B78002BF9D0C088FFF7F6FDF5E70B4BF9
:103DE00040881978FFF792FD1422002101A8FBF703
:103DF00099FB6088ADF80600FFF76EFEADF808008D
:103E000001A8FBF78DFDE0E7C8CD00200CCA00201B
:103E100070B5044686B01422002101A8FBF782FB8E
:103E200023786088ADF80600013B0B2B00F29080F0
:103E3000DFE803F02106233A4E585C68747A7C8CE4
:103E40002679444B321C19784FF0010518BF012226
:103E50008DF80450FFF75AFD731B5A425A413E4BEE
:103E600060881978FFF752FD6088FFF735FEADF8DE
:103E70000800002D42D106B070BD02238DF8043039
:103E80002379002B14BF012302238DF80C30314B12
:103E900001221978FFF73AFD2F4B227919786088B3
:103EA000FFF734FD0125DFE703238DF804302A4BAB
:103EB0001978FFF75BFD002814BF012302238DF85A
:103EC0000C30A3798DF81030A388ADF80E30E9E7F7
:103ED000204B1978FFF74AFD0028CCD102238DF83A
:103EE0000430DFE703238DF80430EAE70723A288D4
:103EF0008DF80430ADF808208DF80C3001A8FBF7E0
:103F00000FFDB8E708238DF80430A388ADF808301A
:103F100007238DF80C30A3680593EFE706238DF88F
:103F2000043063680393BDE70523D8E703238DF8C6
:103F30000430094B1978FFF719FD002814BF01233D
:103F400002238DF80C3041F20113BEE70423C6E7CB
:103F5000002589E790CF00200CCA00201FB50D294D
:103F60004FF0000301930393ADF80600029108D1CE
:103F70000B2301A88DF80430FFF74AFF05B05DF868
:103F800004FB86290CBF0A230923F2E730B5084950
:103F90000A680023012505FA03F42242D8B202D1AF
:103FA00022430A6030BD0133182BF4D11846F9E7DB
:103FB000D0C9002010B50378182B044602D1FFF7B2
:103FC000E5FF207010BD000010B5024B197DFDF714
:103FD00023FB10BDD0C900202DE9F04F3D4D89B025
:103FE0002878FFF787FC60B103A8FFF7EDFFDFF843
:103FF000E8A0DFF8E8B00DF110090027039B9F420D
:1040000002D309B0BDE8F08F39F8024B2978204679
:10401000FFF7ACFC064678B39AF800102046FFF78D
:10402000A5FC804640BBBBF800304FF6FF72194636
:104030002046FBF779FB43F20302904229D101337A
:10404000ABF80030EFE7052320468DF80030FFF78E
:1040500043FDADF802006846ADF80440FEF770FE7F
:10406000B046324629782046FFF750FC42469AF87F
:1040700000102046FFF74AFC0137BFE72046FFF754
:104080002BFDFEF74BFE0026EBE72046FFF7B2FDC7
:10409000E7E70828F2D012D80028D4D00628EDD0BF
:1040A0000923029020468DF80030ADF80440FFF758
:1040B00013FDADF802006846FEF742FED1E743F279
:1040C00002039842CDD043F201439842DDD011283B
:1040D000E6D1C6E737CC002038CC0020CCD1002078
:1040E0001FB5044640882378ADF80600012B10D098
:1040F0005AB21AB1022B15D004B010BD01A88DF828
:104100000420FEF71DFE6088FBF716FBFFF772FD2B
:10411000F2E78DF8043001A8A388ADF80830FEF767
:104120000FFEE9E72379002BE6D0FBF705FB4FF6FE
:10413000FF739842E0D0044B01221978FFF7E6FBA9
:10414000FFF74AFFD8E700BF37CC002038B5074C4F
:104150000146207DFDF7B2F930B1A07DFDF7AEF943
:10416000002814BF0220012038BD00BFD0C90020A4
:104170002DE9F0478CB0894616468046FFF7E6FFEA
:1041800020228246002104A8FBF7CCF9BAF1000FE7
:1041900046D0B9F1000F17D099F8005015F001057D
:1041A0004FF6FF7415D04046FFF796FCA042074635
:1041B00039D14048FDF7E0FCB0F5807F01D0B8422E
:1041C00075D10025032470E04D4685264FF6FF7714
:1041D0005FE02E4627465CE04A4631464046FBF704
:1041E000A7FA0446B9F1000F5DD000285DD199F817
:1041F000003013F0010F14BF012102214046FEF7E9
:10420000DBFDB6F1850218BF0122002400950123D1
:1042100039464046FFF72AFC20460CB0BDE8F0873F
:1042200043F20204F8E7002502AB012207213846D9
:10423000FDF708FD0446002837D121465022039897
:10424000FBF770F9039B83F800A0039C079604F129
:104250003403049304F118030893631C0993404644
:10426000154B0B93FFF796FBFF280CD0134A0C213C
:1042700001FB002050F8042FC4F811208288A4F814
:1042800015208279E2753846FBF7E4FA044660B9F6
:104290000646BAF1020F04AB9ED1002231464046D9
:1042A000FBF746FA0446002CABD00022AEE70746E7
:1042B0000125B9E7D8CF002093CF0020A6CB00205E
:1042C000F0B585B00446FFF741FF324F012806469E
:1042D0003D7831D12046FFF7FFFB4FF6FF73984240
:1042E0002AD0204632462946FFF710FB0023CDE9AD
:1042F0000133039301A80C238DF80430ADF8064078
:10430000FFF786FD244B1B78E3B139782046FFF791
:104310002DFBB8B9214B22491A682046FFF728FF28
:104320008628054632D011280FD070B12946204684
:10433000FFF714FE05B0F0BD002229462046FFF726
:10434000E5FADFE700221146E7E7A5F111035E4237
:104350005E410022134B20461978FFF7D7FA124B23
:10436000324619782046FFF7D1FA104B002219780F
:104370002046FFF7CBFA0E4B002219782046FFF7B4
:10438000C5FA002DD6D0112DD4D0CFE700260122BA
:10439000E0E700BFAE2C0020BFD000207CCF002083
:1043A000BAD00020AD2C0020AC2C0020AB2C00207B
:1043B000AA2C0020F0B587B0074601A8FFF704FE3D
:1043C00002AD0024019B9C4201D307B0F0BD35F83B
:1043D000026B39463046FFF7C9FA10B13046FFF795
:1043E0006FFF0134EEE700002DE9F04F054687B07E
:1043F000904699460F4639B9A14B1B78F3B905246D
:10440000204607B0BDE8F08FFFF7A0FE0138C0B22C
:10441000012800F22D8100212846FBF78BF9044684
:10442000862C00F0B080112C00F09980002C00F058
:104430009680B9F1000F00F0BF80B9E0FFF786FE6B
:10444000012800F09E80022840F012818D490B78EF
:10445000284613F001048B4614BF4FF0010A4FF0B9
:10446000020AFFF739FB4FF6FF739842064659469A
:104470003AD03B4602AA0721FEF7F4FC0446F0B905
:10448000039B93F84420D10740F1C780B8F1000F97
:1044900040F0D68003F1340202F112012846FBF706
:1044A00045F94FF0000A044600230093BAEB0303DA
:1044B00018BF0123B4FA84F25209314645E00528B9
:1044C000F2D1BDE004AB012207213046FDF7BAFB73
:1044D0000446002840F0C1803046FBF7BBF9044693
:1044E000002800F0B280B8E0002C41D06648FDF70B
:1044F00043FBB0F5807F834637D0B04236D004AB63
:1045000001220721FDF79EFB044650B95846FBF7F0
:10451000A1F9044628B95B492846FBF70BF9044684
:1045200038B107215846FDF779FC10B1052818BFAE
:1045300003244FF6FF73BBEB030318BF0123B4FA48
:1045400084F200935209012359462846FFF78EFA58
:10455000002C7FF465AF51462846FEF72DFCA4F1F0
:1045600011035E425E4100220FE0B3460324E0E700
:104570002846FBF7DFF8009704460123B0FA80F2E3
:104580009AE7404948E700260122404B284619781F
:10459000FFF7BCF93E4B324619782846FFF7B6F9CB
:1045A000B9F1000F08D0002C3FF42AAF112C17D01E
:1045B00021462846FFF7D2FC0D2C3FF421AF06D848
:1045C000002C3FF41DAF082C18BF032418E7862CDD
:1045D00014D043F202039C423FF412AF112C1AD1C3
:1045E0002C4B3A4619782846FFF790F92A4B424659
:1045F00019782846FFF78AF9002401E7254B3A4647
:1046000019782846FFF782F9234B42461978284645
:10461000FFF77CF9F4E60324F2E6B8F1000F0FD1BE
:10462000598D03F1180200297FF436AF03F12C01F4
:10463000343311F8010B00287FF42EAF8B42F8D1F0
:104640009BF80030DA073FF53DAF0E492846FBF7EF
:1046500071F8044600283FF427AF07213046FDF7E4
:10466000DDFB00283FF420AF052818BF03241BE71B
:1046700043F20204B9F1000F3FF4C2AE98E700BF65
:10468000BFD00020BAD00020D8CF0020AB2C002013
:10469000AA2C0020A92C0020A82C00202DE9F047EE
:1046A00086B00746FFF726F958B101A8FFF78CFC42
:1046B000DFF84880DFF8489002AE0025019B9D425C
:1046C00002D306B0BDE8F08736F8024B39462046E3
:1046D000FFF74CF980B198F800102046FFF746F933
:1046E00099F8001082462046FFF740F90123014661
:1046F00052462046FFF778FE0135DFE7A82C002060
:10470000A92C002010B50378062B0ED9072B1BD13E
:104710000E4B1C782046FFF7EDF810B12046FFF74E
:1047200049FE0B4B1878FFF7B9FF0A4B1C7820465F
:10473000FFF7E0F810B12046FFF73CFE064BBDE85E
:1047400010401878FFF7AABF10BD00BFAD2C0020A5
:10475000AB2C0020AC2C0020AA2C00201FB5037825
:104760000446092B09D8DFE803F0050A20202020A1
:10477000202020204088FFF7A3FD04B010BD144B7B
:10478000197819B3134B00791B7803F0010290429A
:1047900006D86179C3F34003994294BF00210121F7
:1047A000012300226088FFF71FFE23788DF8043074
:1047B000043434F8023CADF8063094E8030004AB4E
:1047C00003E9030001A8FFF723FBD6E70121E7E790
:1047D000BFD00020BAD0002037B5174B174A5B88EE
:1047E0001188174C174D994208D852889A4205D320
:1047F0006369FBB900232B7003B030BD2B783BB14C
:104800006369002BF6D000228DF8042001A80FE088
:104810000D490E480978D4E9012300290CBF11463F
:104820001946FDF741F90028E4D0A369002BE1D037
:104830009847DFE70122E7E706CC002018D00020E8
:1048400068CB0020FCCA0020E0D0002084CB0020F0
:104850007BDF70477ADF704776DF704775DF704720
:1048600037B5164B18884FF6FF73984210D0144A8C
:10487000144D1378297B0133DBB2994213702C4617
:1048800008D31149FFF7EAFF10B1AB6903B19847AC
:1048900003B030BD002313702B7C33B13B21FFF7F5
:1048A000DBFF10B1AB6903B198476369002BEFD010
:1048B00000228DF8042001A8E9E700BF64CB0020A6
:1048C000E0D0002068CB002018D0002065DF7047C2
:1048D0002DE9F74F0C9CBDF834B0278800258046A1
:1048E0008A4691462E46B8F80020B2420BDC35B11C
:1048F0002288013AD21B92B2FF2A39D8DA55002019
:1049000003B0BDE8F08FD8F8042052F826000190DB
:1049100000220DF1030101A8FFF7D8FF0028EFD115
:104920009DF803204A4521D12288002D14BF002084
:10493000022002EB09010144594519DC3DB901325D
:1049400092B2228003F802A02288013222802288BB
:104950000DF103011A4401A8FFF7B8FF0028CFD1D9
:1049600021889DF803200A44228001250136BAE7F8
:104970000C20C5E72DE9F341089CBDF824501746EB
:10498000CDE9004502220646FFF7A2FF48B91022F2
:1049900039463046CDE9084502B0BDE8F041FFF7A1
:1049A00097BF02B0BDE8F0812DE9FF4700231380D7
:1049B00090F82D3006460D4614463BB302A8FAF790
:1049C000C7FF002840F0FB8013880822CA542388C0
:1049D00001339BB21B222380CA54238801339BB22C
:1049E000CA18DDF809102380E950BDF80D30938016
:1049F00023889DF8082006339BB212F0FE0218BFF0
:104A000001222380EA54238801332380B378FBB149
:104A1000238804331F2B21D802A8FAF797FF002818
:104A200040F0CD8023880322EA54238801339BB2CF
:104A300019222380EA542388BDF8082001339BB251
:104A4000E9182380EA54120A4A702388023323802B
:104A5000F278AAB12388D91C1F2901D90C20AEE015
:104A60000221E954238801339BB201212380E954B8
:104A700023880B449BB22380EA5423880B44238071
:104A80007268AAB12388D91C1F29E7D8022192F99C
:104A90000020E954238801339BB20A212380E95482
:104AA000238801339BB22380EA5423880133238077
:104AB0003389002B76D1338A5BB11F23CDE90043C4
:104AC00007222B46032106F11000FFF753FF0028B1
:104AD00075D1338B5BB11F23CDE9004315222B46E3
:104AE000142106F11800FFF745FF002867D1326A4C
:104AF000002A67D1776A4FB3BB882188981C8A1C2B
:104B000002441F2AAAD8FE28A8D803336B5423884E
:104B100001339BB2FF222380EA54238801339BB2E6
:104B200023803A88EA54E918120A4A702088023031
:104B300080B22080BA884AB1B96800294AD0284496
:104B400038F058FB2388BA881344238096F82C3019
:104B5000002B79D1307890B33388012B3AD0238859
:104B60009F1C1F2F3FF67AAF012805D172780232C1
:104B70001A441F2A3FF672AFC3F11D039BB202A96C
:104B8000E819ADF80830FAF7DFFEC0B93278022A2A
:104B900040F09880BDF808209A4240F2AE80ADF80F
:104BA000083098E01F23CDE9004306222B4602215E
:104BB00006F10800FFF7DEFE00283FF47CAF04B0EA
:104BC000BDE8F0872788BB1D1F2B3FF647AF118834
:104BD000052901D80720F2E76FF4486C01EB0C03BC
:104BE0009BB24FF27D3C6345F4D95388052BF1D934
:104BF0006FF44860181880B26045EBD94FF6FF702B
:104C0000814203D0834201D09942E3D80523EB557A
:104C1000238801339BB212212380E9542388013376
:104C20009BB223801188E954E818090A417023884F
:104C300002339BB223805288EA54E918120A4A7060
:104C400023880233238055E7B36A002BC2D04FF08C
:104C500000084FF00C094FF0160A96F82C305FFA56
:104C600088F293427FF676AFB16A09FB02F28F18A1
:104C7000BB88981CFE283FF6F1AE208803332B54E6
:104C8000238801339BB2238005F803A023880133D6
:104C90009BB223808A5AEA54E918120A4A70208883
:104CA000023080B22080BA884AB1B968002991D018
:104CB000284438F09FFA2388BA881344238008F1E7
:104CC0000108CAE7012A7FF46AAF72789342FFF4C1
:104CD00066AFADF808200821BDF80830FE2B3FF67E
:104CE000BDAE22880133AB542288013292B22280B9
:104CF000A95422881344238061E70921ECE70000CE
:104D000007B5144B1A686AB1002018601B6800933D
:104D10004FF08042009B0123C2F808330E4A5370C3
:104D2000FAF718FE0D4B1A688AB100221A601B6848
:104D30000193019B4FF080430222C3F80823064BE6
:104D40000120987003B05DF804EBFAF703BE03B0DE
:104D50005DF804FB0001004048CB00200401004046
:104D600013B5104B104C114800221A601B680193B8
:104D70002146019BFAF704FE88B9A27E0C48FF2A5F
:104D80001FBF012393404FF0A042C2F80835002313
:104D900063762371236802B0BDE81040184702B063
:104DA00010BD00BF08310040BCCA002000300040E8
:104DB000C0CA002070B52D4C86B094F82130019304
:104DC00094F820300093E36904F1260204F12301F2
:104DD0004FF04020FAF705FE2346E0B994F823602F
:104DE000A56906BB217B8A1E012A1CD8E0692269BD
:104DF000904218D16269E37BE261C5F34015032953
:104E000084F8203084F8215007D100954FF04021DC
:104E10002046FAF7BDFE06B070BD4FF04021204697
:104E2000FAF759FEF7E7124A07CA06AC04E9070089
:104E3000C6B14FF04021D1F8C424C1F8C424900772
:104E40000CD501228DF80820002283F824206A075F
:104E5000E1D4D3E9002102A89047DCE75107F3D55C
:104E60000222EFE78DF80860EEE700BF94CA002049
:104E7000A0CA0020F7B515464FF0FF32C1F808234D
:104E800090F8242004460F4602F0FF0E2AB18368F2
:104E9000C1F80433112003B0F0BD012680F824606E
:104EA000836100F10C0C95E807008CE80700AA78F4
:104EB00084F820206A68E2616A78C7F888252A7831
:104EC000B24212D012B91E1C18BF012684F821600C
:104ED0000096AB786A6839462046FAF759FE23688F
:104EE000002BD8D184F82430D5E784F821E0AB78C2
:104EF0006A6839462046FAF7EEFDF0E70023435092
:104F000082B043580193019B02B07047064A08B52E
:104F10004FF492711046FFF7F1FF4FF48471FFF7E1
:104F2000EDFF0123136008BD0020004010B5CB7DCC
:104F30000A464FF4847123B9FFF7E0FFD0F8183523
:104F400010BDFFF7DBFF537ED168D0F81805C854B9
:104F5000537E0133DBB25376F2E70000F8B52C4CF8
:104F6000626822B12B4B4FF40171C3F80813E37D43
:104F70004BB1237E7BB322B1264B4FF40172C3F8B1
:104F80000423112026E00122E275E0606376A27E10
:104F9000237612B90BB9FFF7B9FF636873BB4FF4FF
:104FA000A2711C481B4E1A4FFFF7A8FFD6F82431F8
:104FB000D6F80821D6F8445182B90DB9002BF5D0A6
:104FC0000022E27503BB0DBBA17E124B012299B1F9
:104FD0001A600020F8BD20610123D8E7002BEFD133
:104FE000002DEDD139463046FFF7A0FF637EE27D0C
:104FF0009A42DBD82B46E3E75A60EAE7054B4FF4C9
:105000000172C3F80423E4E70320E3E70F20E1E79C
:1050100078CA0020002000400A4610B54FF48E7177
:10502000FFF76CFF938A91689BB2C95C938A013346
:105030009BB29382C0F81C1510BD000030B54A4ADF
:10504000D2F8043313F4007F85B015464AD0D2F865
:105050002431002B46D04FF492711046FFF74EFFDB
:105060004FF40173C2F80833404B997E09B901210E
:1050700051603D4902228DF80020D1F88024C1F80A
:1050800080240392DA7D8DF80820DA6801920022EC
:10509000DA751A766846D3E9001290473248D0F89C
:1050A0001C313BB1314A938A917D994247D91146CF
:1050B000FFF7B2FF2C4AD2F844318BB14FF4A27102
:1050C0001046FFF71BFF294B997E09B101211160A2
:1050D000DA7D2AB10022DA75587ED968FAF74AFAE1
:1050E00005B030BDD5F804335B07D7D5D5F8083106
:1050F000002BD3D01D4C1C482146FFF717FF637EC1
:10510000E27D9A422346C9D1227E52B12369E168E9
:10511000E3600023607EE27523766376FAF72AFA6D
:10512000BCE7A27E0AB901226A600F4A4FF40171FE
:10513000C2F808130022DA75587ED968EEE74FF4FA
:105140008E71FFF7DBFE917D0029B3D000238DF82F
:10515000081091688DF80030019193756846D2E986
:1051600000139847A6E700BF0020004078CA00203F
:10517000800000F1A040D0F8003723F44033C0F89D
:105180000037D0F8003743EA0141C0F800177047F4
:1051900000F1804000F5C040002382B00360036846
:1051A0000193019B02B070472DE9F04F85B00024B8
:1051B000594D01944FF48072012102F1804303F5AF
:1051C000C04390B21B68012B06D1D5F804330B42C3
:1051D00002D0FFF7DDFF0C430432B2F5907F4FEAB7
:1051E0004101EAD14D4B1B68012B0AD14FF4BE702F
:1051F000FFF7CEFF4FF0A04344F00044D3F8103542
:10520000019314F0FF0F1AD0454F012600253442B8
:1052100010D0AB0003F1804303F5C043D3F8100571
:10522000D3F8101557F8253023B1C1F30141C0F36D
:10523000042098470135082D4FEA4606E7D1002C97
:1052400063DA4FF0FF330022CDE90232344D354EA0
:105250000024A24601274FF0A04816F9012B531C49
:1052600046D0D2B222F0C0094FEAD90104A80844BE
:1052700002F0070310F808CC07FA03F31CEA030F47
:1052800036D005EB090C92099CF930C055F82CB0CA
:10529000BBF1000F0AD1032A2AD10DF10C0E1EF822
:1052A00001C04CEA030C0EF801C001E0032AF4D05F
:1052B00009F5E07110F80C0C58F821101842C1F3F0
:1052C000014105D0022913D1032A0BD1114604E074
:1052D00003290DD1032A05D102214846FFF748FFD3
:1052E0000134E4B2BBF1000F02D011464846D84762
:1052F0000AF1010ABAF1040FAFD134B14FF0A04363
:10530000019AD3F81035934202D105B0BDE8F08F71
:105310000193039B02939AE7006000407C61004088
:1053200020CA002070CA00200028C3B2A8BF00F124
:1053300060424FEA501010B5BABF0D4A03F00F0497
:1053400002F561424FEA41114FEA8000C9B200F113
:105350006040B4BF115582F8001300F5614003F0BE
:105360001F0201239340C0F88031036010BD00BFCD
:1053700014ED00E02DE9F8430446C279C17A0E200D
:1053800025F05CFA237B644A0BB3537843F0100397
:1053900053702568EB175906604B41EAD511680632
:1053A0004FF0FF328B4208BF82420AD35C4A00238F
:1053B00037F054FD00F5006020F47F6626F00F06FC
:1053C0004EB929465748BDE8F84331F0DBBC537865
:1053D00003F0EF03DCE7207928F0E0F840B96079CA
:1053E00028F0DCF820B95048BDE8F84331F0CABCD9
:1053F0004E4F3B781BB100233B70FBF793F82579A8
:105400004B4B002228461A7028F0C8F820B14FF400
:10541000407128461CF0C4F86579284628F0BEF88B
:1054200020B14FF4985128461CF0BAF8637A2579D8
:10543000002B284614BF4FF00E094FF0000928F04A
:10544000ADF800285AD03B4B05EB85051D4495F877
:1054500001806479204628F0A1F8002851D0354B0E
:1054600004EB84041C446378334CE27E002A4BD165
:105470005A1C0AD04FF0A04101229A40C1F80825D9
:1054800003F5E072032041F82200B8F1FF3F2B4DF5
:105490001FBF4FF0A04108F5E072002041F8220044
:1054A000C5F82465C5F86C950026C5F81485C5F8BF
:1054B0000C35234B636028464FF48E712660FFF74E
:1054C0001DFD4FF4A271FFF719FD1E4BC5F8043303
:1054D00002210846FFF728FF0423C5F80035B8F17C
:1054E000FF3F4FF48073E6822676638310D0FFF788
:1054F0000DFD0123A37616F0D1F909E04FF0FF3836
:10550000A7E74FF0FF33AFE708210F4831F01AFC4F
:1055100001233B70BDE8F883C8C9002047E80100BB
:1055200048E8010075D405008AD40500D9D10020CF
:10553000DAD1002020D5050078CA002000200040E4
:10554000D5B8030080000200A0D4050010B50D4CB2
:1055500000226260A2602261E2600B4A106810F0D3
:10556000010002D10621FFF7DFFE084B1B7823B9AB
:105570004FF080430122C3F8182501232370002037
:1055800010BD00BF48CB002000E100E0C1D00020EA
:10559000F8B50E46D11C48BF911D144641F3870152
:1055A0000546671EFAF70DFC00214AB2A24201F13E
:1055B000010100DBF8BDBB1A23F00300B25C03F06D
:1055C0000303DB0002FA03F32A581A432A50ECE7DC
:1055D000F0B500254F1E6CB28C4205F1010500DBD1
:1055E000F0BD3B1B23F0030603F003039659DB00D9
:1055F00026FA03F30355EEE72DE9F041B3F9024033
:1056000014F11F0548BF04F13E050F4603F12406BF
:1056100045F34715904601462B4632463846FAF781
:105620000FFCB8B9B4EB451F16DA6211012304F080
:105630001F0403FA04F457F822301C4214BF01245B
:1056400000242B46324639464046FAF7F9FB2046FD
:10565000BDE8F0810124F4E70446F2E710B5002329
:105660001A465CB2A14203DCB2FA82F0400910BDD6
:1056700050F8234001332243F3E700002DE9F04FB7
:105680008A46234F8BB00646114650461446FAF719
:1056900078FB3B68FBB10425C0EB441014FB05FB11
:1056A00000B205FB04654FF0FF38043D28FA00F80E
:1056B0004FF040093B6859463046984758B12B682F
:1056C00003EA08032B6021463046FFF7C7FF20B1ED
:1056D000B9F10109EED1002017E0234632465146C8
:1056E00002A8FAF77DFB2146019002A8FFF7B6FF5A
:1056F000019B003318BF01235B00002814BF5842F0
:10570000C3F10100C0B20128E2D10BB0BDE8F08FB7
:10571000802D00202DE9F04FD1B0CDE905015B9D32
:1057200095F9004048A8914622461F46FAF71DFB0E
:10573000A3000793069BA20013441946224638A8EB
:105740000293FAF712FB95F90060002F00F08C80AD
:105750003246394628A8FAF708FB0DF5807A32461A
:1057600030AF48A95046FAF700FB38A93846FAF797
:10577000FCFA2B4628AA38A948A8FAF7B5FA2B460E
:1057800028AA38A948A8D5F8A460B0472B4628AA6B
:1057900039465046FAF7A8FABDF968310497023B3A
:1057A0001BB2002B67DCD9F80030009503F001082C
:1057B0004FEA481840AADB4302EB080A03F0010352
:1057C00030AA90445B0140AA1A44039230AAD3182D
:1057D0004146039A0493504605F10409FAF727FD60
:1057E0004B4640AA48A908A80094FAF790FC08A9DB
:1057F00008462B464246FAF736FA08A908462B46D1
:10580000069AFAF730FA214608A8FFF727FF002882
:105810005DD008A8FAF7D5FA08A92B46029A0846DF
:10582000FAF721FA08A92B4652460846FAF71BFA5E
:10583000DDE90301434652460095FAF77AFC2B4610
:1058400008AA30A940A8FAF74FFA224640A90598BD
:10585000FAF78BFA059B079C234430A91846FAF700
:1058600084FA51B0BDE8F08F314628A8FAF7A9FABA
:105870000123289371E71FFA83F85B1108F01F02D8
:1058800059F823300095012101FA02F21A42049BD3
:1058900013BF20270027202600260AEB070B1F44F2
:1058A0000AEB06030393049B039A1E4433463946CE
:1058B0005846FAF7BCFC08F1FF383B4600955A46BB
:1058C00031460398FAF735FC0FFA88F369E710AF11
:1058D000224608A938460DF1600BFAF746FA20AEC9
:1058E00049465846FAF741FA30462146FAF769FA2E
:1058F000012328A82093FAF764FA2246594638462D
:10590000FAF71EFA28B9224620A908A8FAF72DFAB4
:1059100082E73B68DA0709D421463846FAF703FAEA
:10592000224649463046FAF7D6FBE6E7189BDB07E6
:1059300007D421465846FAF7F6F92246494628A8E0
:10594000F1E7002823461CDD5A4639463846FAF767
:1059500047FA21463846FAF7E6F9224628A93046A2
:10596000FAF7EEF9002805DA23464A463146304672
:10597000FAF766FA234628AA31463046FAF730FA93
:10598000CEE73A4659465846FAF72AFA214658468B
:10599000FAF7C9F92246314628A8FAF7D1F90028C2
:1059A00005DA28A923464A460846FAF749FA28A9FB
:1059B000234632460846FAF713FABEE72DE9F047C8
:1059C00093F9006092B00446894610463146154668
:1059D0009846FFF743FE002840F091804246494632
:1059E0000AA8FAF77DF943460AAA214602A8FAF75F
:1059F0003AF90AA908464246FAF772F943462A4696
:105A000049464846FAF72FF908F104074246294665
:105A10002846FAF765F93B462A4621462046009675
:105A2000FAF7ECFB3B462A46294628460096FAF749
:105A3000E5FB3B462A46214628460096FAF767FBD7
:105A400043462A4621462046FAF70DF93B462246B0
:105A5000214628460096FAF7D1FB3B4600962A4697
:105A600021462046FAF7CAFB2368DB074AD53346AE
:105A70003A4621462046FAF7E3F931468246204667
:105A8000FAF751F906F18043013B54F8230040EA4C
:105A9000CA7044F82300424621462846FAF720F906
:105AA0003B4602AA294628460096FAF730FB3B46B9
:105AB00002AA294628460096FAF729FB02A90846B9
:105AC0003B462A460096FAF722FB434602AA2146A5
:105AD0002046FAF7C8F80AAA3B4610462146009627
:105AE000FAF715FB324629462046FAF73EF94946B1
:105AF0002846FAF73AF90AA94846FAF736F912B0F1
:105B0000BDE8F08731462046FAF70DF9C3E70000FB
:105B100073B500230DF102008DF80230FBF712FB84
:105B2000264B1B7803F0FF04002B41D1244B1A684D
:105B3000002A3DD0234AD2F80813C90738D51C6083
:105B40001B68214D01930DF10300019BD2F80865FC
:105B50008DF80340FBF7F6FA6A6829681F2A98BF98
:105B6000541CA142F6B26C6004D1202C14BF611CFD
:105B70000021296015499DF803008E542A6894423B
:105B80003ABFC2F121021319A31AAA689A4238BF78
:105B9000AB60FBF773FF6B682A681F2B94BF013360
:105BA00000239A4201BF074A0123C2F80833536019
:105BB0009DF80200FBF762FF02B070BDC1D000206B
:105BC00000D1004000D00040ACD0002088D00020A0
:105BD00030DF70472DE9F74F3B4F06468846B8F156
:105BE000000F03D1012003B0BDE8F08F4546202D02
:105BF00028BF20255FFA85FB002400230DF1020059
:105C00008DF80230FBF79EFA304B1B7803F0FF094A
:105C100093BB0DF103008DF80390FBF793FAD7E9DE
:105C200000148C4204D3641AA54207D9052414E059
:105C30002134641AA542F9D8C1F12104244BA542AC
:105C4000194431D82A46304637F0D4FA3B682B4401
:105C5000212B28BF00233B6000249DF80300FBF7A5
:105C60000DFF1C4B00221A601B680193019B1A4B0D
:105C70000122C3F804231A609DF80200FBF7FEFE20
:105C8000B9F1000F08D059463046FFF7A1FF42F2A4
:105C9000070398420446ADD0022CAED0002CA9D107
:105CA000A8EB05082E449AE72246304637F0A2FAC0
:105CB000074BA5EB040A52461946301937F09AFAF9
:105CC000C7F800A0C8E700BFACD00020C1D00020BA
:105CD00088D0002000D1004000D0004017B4314AE5
:105CE000314B116889B90021304A106820BB00206F
:105CF0005A79D40740D408B9002949D01C68DA88F9
:105D0000234603B05DF8044B184700211160126868
:105D1000D9680092009A0029E5D0254AD2F84005BA
:105D2000814204BFD88801EB8001C2F840155A793E
:105D300042F004025A71D7E7002010601268986898
:105D40000192019A0028D2D0194AD2F83845A042CF
:105D500004BFDC8800EB8400C2F838055A7942F0B1
:105D6000020214075A71C3D512F0010402BF64F392
:105D7000C3025A712046BBE702F00601062907D18B
:105D800022F0060211075A7106D56FF3C3025A7149
:105D900003B05DF8044B7047054AD2F83805D2F8D5
:105DA0004015ABE71451024010CA002004510240D4
:105DB00000500240A5DF7047A4DF7047A3DF7047A3
:105DC0002DE9F0470E4690B016F010058146924638
:105DD0009846189C0CD011238DF8083023788DF844
:105DE000093001224FF0000362F342038DF80A30BC
:105DF0001C22002109A8F9F795FB8DF8246005B154
:105E000002AD42F64D23ADF80C3063789DF8641076
:105E10008DF804300022A3788DF80530134661F325
:105E2000C303DBB243F00303CDE906220E9501273D
:105E300001AD8DF80630089203AE1A9BB9F8000048
:105E40008DF80E7004AA09A9CDE90465ADF81CA06F
:105E5000FDF706FD58BB42F60813ADF80C30637829
:105E60008DF80430A3788DF80530034667F34203BC
:105E70008DF806301A9A98F800308DF8003098F8AE
:105E80000130CDF81A00ADF81E008DF8013032F85F
:105E9000080B8DF80E70022304A9CDE90465ADF856
:105EA0001830ADF81C30CDF820D0FFF787FF10B0C8
:105EB000BDE8F087A1DF7047BFF34F8F0549064B60
:105EC000CA6802F4E0621343CB60BFF34F8F00BF98
:105ED000FDE700BF00ED00E00400FA0508B5FAF7A1
:105EE0007FFA10B1664B674A1A60FAF759FA28B17F
:105EF000654B664A1B68C3F342331360FAF770FAC6
:105F000020B1634AD36823F08073D360FAF748FA6C
:105F100040B14FF080430022C3F80C21C3F8102198
:105F2000C3F83825FAF75CFA10B15A4B03221A600D
:105F3000FAF756FA40B1584B05221A6001229A67C7
:105F400000229A603F225A60544B1B78062B50D196
:105F5000534B1B681B074CD1524B1B6803F0F003DB
:105F6000502B46D14FF080524F4BD2F80414C3F857
:105F70002015D2F80814C3F82415D2F80C14C3F86D
:105F80002815D2F81014C3F82C15D2F81414C3F83D
:105F90003015D2F81814C3F83415D2F81C14C3F80D
:105FA0004015D2F82014C3F84415D2F82414C3F8CD
:105FB0004815D2F82814C3F84C15D2F82C14C3F89D
:105FC0005015D2F83014C3F85415D2F83414C3F86D
:105FD0006015D2F83814C3F86415D2F83C14C3F82D
:105FE0006815D2F84014C3F86C15D2F84424C3F8ED
:105FF0007025FAF7D5F928B12C4B2D4A1B6803F010
:106000004F0313602B4AD2F8883043F47003C2F870
:106010008830BFF34F8FBFF36F8F4FF01023D3F84B
:106020000022002A03DBD3F80432002B24DA224BAF
:106030000122C3F80425D3F80024002AFBD04FF036
:1060400010221521C2F80012D3F80024002AFBD038
:106050004FF010231522C3F80422174B1A46D3F829
:1060600000140029FBD00021C3F80415D2F8003435
:10607000002BFBD0FFF720FF104B114A1A6008BD20
:1060800074C007400DF0ADBA440200103C0500405A
:10609000F0ED00E0A005004010560040E00F00F0D9
:1060A000E40F00F0E80F00F000C0004058020010BC
:1060B000E40E004000ED00E000E00140A42C0020D0
:1060C0000090D003002382B0036003680193019B1A
:1060D00002B070472DE9F341844BD3F8042162B339
:1060E000D3F800339F0728D5814D8248FFF7EAFF98
:1060F0002B7803F0FF08F3B97F4F804E7B783C4646
:1061000003F0FF02002B00F0AF8073684046984711
:1061100001A88DF80480FBF715F87B689DF8040052
:1061200001337B60FBF7AAFC754B0122DA601A6031
:10613000744B00221A6001232B706C4BD3F818218A
:10614000D2B1D3F80023560616D5D3F824356E48BD
:10615000DB08C3F3080113F4FF7F18BF0239FFF710
:10616000B1FF624B4FF48052C3F808254A1EFE2A45
:1061700040F2A4800122DA615C4AD2F81031D3B136
:10618000D2F80033DD0616D56048FFF79BFF1023D9
:10619000C2F808335E4BC2F81035FF23C2F814353D
:1061A0000123D3615B4B1C682CB15B4800231A466A
:1061B00003210068A0474D4AD2F84C3133B3D2F8DE
:1061C00000331C0322D55548FFF77CFF4E48FFF7EC
:1061D00079FF5348FFF776FF4D4BC2F81035FF2388
:1061E000C2F814350123D3614FF48863C2F8043335
:1061F0000D23C2F80C34C2F80434464B1C682CB191
:10620000454800231A4619460068A047374AD2F885
:1062100028315BB1D2F80033580507D54048D2F891
:106220000C34FFF74FFF0D23C2F80C342F4AD2F87D
:106230001C31B3B1D2F80033190612D53948D2F85F
:106240000414FFF73FFFCB0707D5374B197821B16F
:106250000121C2F8041400221A70244B0D22C3F845
:10626000042402B0BDE8F0810DF103008DF8032095
:10627000FAF768FFBA68134683B93260A6606368AC
:1062800033B92A4B1B7803F0FF025BB1F9F776FBB9
:1062900063689DF803000133636043E7B342EED0C7
:1062A0001B68E9E7224B1A601B680193019B4FF0C2
:1062B00080430122C3F804231A60E9E7144A1078E6
:1062C000502803D1184901220A7054E71148046884
:1062D000002C3FF451AF4FF6FF70C3F808050E488D
:1062E0000B4600680221A04746E700BF005000406F
:1062F00034CC00200451004048CB00205CCB00206F
:1063000000B001407C2D0020185100401051004089
:10631000E0CD0020ECCE0020F0CE00204C5100401B
:10632000285100401C510040C0D00020C1D00020A6
:106330000001004013B5284B2849D3F83C3413F032
:10634000030345D10A680132072A0A602CD9244A7E
:10635000012414610DF107008DF80730FAF7F2FE01
:10636000204B5A68013A5A605A6822B91E4A12787C
:1063700002B3F9F701FB9DF80700FBF77FFBBFF3C2
:106380005F8F1A4A00231360BFF35F8F01211160F2
:10639000174A14681CB117481A460068A047164BE4
:1063A00000221A70FAF750FE0D4B0022C3F840216C
:1063B00002B010BD114A4FF080411460D1F80C2496
:1063C00002F00112B2F1011FF8D000225A70D2E798
:1063D00000230B60E8E700BF005000407C2D002048
:1063E00000B0014048CB0020C1D00020FC5F00403D
:1063F000ECCE0020F0CE002034CC00200400004081
:106400008DDF704777DF704701381F289DBF034B32
:1064100023FA00F000F00100002070478B8080809C
:1064200030B551EC100B85B053EC112B8DED000BFA
:1064300055EC124B8DED021B36F03AFC9DED000B36
:1064400028B19DED021BB0EE410AF0EE610A53EC5B
:10645000102B204629468DED000B36F029FC9DEDD2
:10646000000B08B145EC104B05B030BD38B555EC0C
:10647000104B0022002310EE100A294636F018FCBB
:1064800010B105F100431D4645EC104B38BD00002E
:106490002DE9F04F89B00E4600AF0023044607F106
:1064A000140130467B612DF060FF054618BB304675
:1064B0002FF0D4FD804678612CF000F908F5807348
:1064C00083420CD9A64901202FF088F93246A5490C
:1064D00001202FF083F92437BD46BDE8F08F08F185
:1064E000070323F00703ADEB030D6D464246294633
:1064F00030462FF0A3FD7E6926B99B4901202FF07D
:106500006DF9E8E74FF00308B6FBF8F303EB43033C
:106510009E4201D09549F1E7204627F03FF808B99F
:106520009349EBE7934BC7F808D004EB84041C4471
:106530006178914C2079002840F009818F4A01232D
:10654000C2F80405FF29C2F82405C2F82005C2F8E4
:106550001C35C2F82805C2F818054FF0C050C2F823
:106560001405C2F8103518BF01F5E0704FF0A043D4
:1065700008BF4FF0FF31C3F85887C3F8FC8A18BF33
:1065800043F820801623C2F86435FF23C2F868352B
:106590004FF0FF33C2F860352520C2F87015C2F8FD
:1065A0006C350221764B2360FEF7BEFE012323717A
:1065B0000323B6FBF3F39BB203EB430808F1010896
:1065C00028F001029100ADEB010D6846FA606D4ABA
:1065D0003A6041184FF0000C796082F800C0E91C65
:1065E0004FF0EE09851C4FF0880A4FF08E0B634583
:1065F0005FDC0C2202FB030300227968994200F25F
:106600009E802679012E40F0A28000F06043B3F115
:10661000005F40F0A280FB68C3F34E02574B00219D
:10662000C3F85025C3F83815C3F80815C3F840055A
:10663000C3F80C656579E28025F0090545F0080589
:106640006571C4E90210C3F80065022323710D4689
:10665000002977D04FF6FE7208EA0202F8F762FFCF
:10666000494B00221A601B68FB61FB69474B1A60AB
:106670001B68BB61BB69414B2222C3F80423012282
:106680001A603A681278042AFBD94149002222256F
:106690000120C3F808530860C3F80025C3F8085365
:1066A0000860C3F800253B4B2021C3F884102271F9
:1066B00050E011F8026C11F8032C360246EA02464B
:1066C00011F8012C05F10C0E164306F44012B2F538
:1066D000001F1ED0B2F5401F20D0B2F5801F20D180
:1066E00005F802BC06F44002B2F5000F1CD0B2F56A
:1066F000400F1ED0B2F5800F1ED105F801BC023547
:10670000AE454FEA0616E0D10CF1010C0331754697
:106710006DE76FF0170205F8022CE3E705F8029C1D
:10672000E0E705F802ACDDE76FF0170205F8012C91
:10673000E5E705F8019CE2E705F801ACDFE703F8BF
:10674000012B5AE7014623682846984788E7082026
:10675000FBF732F9D7F808D0BDE61020F8E700BF04
:10676000B1D305005FF205008BF20500ABF2050026
:10677000D6F2050020D5050010CA002000500240C6
:10678000B5820300EDD100200451024014510240B3
:106790000450024000E100E010F5A24F0FD006DCEB
:1067A00010F5A34F0ED04142084830F0EBBA10F577
:1067B000A14F09D010F1220FF5D1054900E005499C
:1067C0000548F2E70549FBE70549F9E7E3EE05006F
:1067D000BFEE0500D4EE05006E0B060099EE050035
:1067E000ABEE0500024B0349586800222FF078BA3F
:1067F000682D0020004206002DE9F04FADF51B7D0D
:1068000000AF144605461022884607F11800002103
:106810009B46F8F787FE204631F0D6FC0646002856
:1068200059D00022BE4920462FF05AFA064680B1C0
:10683000102207F118012FF001FCF389A3F5007372
:106840009BB2F381F38903F4F05313B9304631F06E
:106850008DFE20460022B3492FF042FA044600285C
:1068600043D0B1492DF0FEFC002840F05582AF49DD
:1068700020462DF0F7FC002840F05182AC4920461C
:106880002DF0F0FC002840F04D82AA4920462DF062
:10689000E9FC002840F04982A74920462DF0E2FC9F
:1068A0000646002840F044822246A44901202EF0EA
:1068B00095FFB146E389A3F500739BB2E381E389B9
:1068C00003F4F05313B9204631F050FEB9F1000F34
:1068D0000DD1002603E044B1994830F053FA304618
:1068E00007F51B77BD46BDE8F08F4FF001094FF467
:1068F0008C72002107F13800F8F714FE002307F12D
:10690000140128467B612DF030FD0446D0B928469D
:106910002FF0A4FB064678612BF0D0FE06F58073BD
:10692000834204D9874901202EF058FFD1E7F31D97
:1069300023F00703ADEB030D6C4632462146284693
:106940002FF07CFB002307F1100140463B612DF046
:106950000CFD0546A8B940462FF080FB064638617D
:106960002BF0ACFE06F580738342DBD8F31D23F0D9
:106970000703ADEB030D6D463246294640462FF026
:106980005DFB3E69F600BBF1000F3DD14FF48C7208
:10699000594607F5A870F8F7C5FD07F140033246E0
:1069A000294607F5A870FB631BF0A0FB8046F8B9E9
:1069B000D7F85011D7F85401B9630B01C218C35866
:1069C0003B6453687B649368BB64D368FB645E4E2E
:1069D0004B1E7B60103A07F150037968002921DCD7
:1069E000116819605168596091689960D268DA60DD
:1069F000002340F21912184607F5A8711944013313
:106A0000934208D00870F7E73246294607F138006C
:106A10001BF06CFB8046B8F1000F2ED04046FFF70C
:106A2000BBFE56E7A2F1040E03F1100A5EF8040F54
:106A30004649C5B216F805C0050E51F82CC0755D63
:106A4000434951F8255043498CEA050CC0F307250A
:106A5000C0F30740755D305C51F825503E4951F850
:106A600020008CEA0505454043F8045B5345DDD121
:106A7000796801397960103AAFE707F10C0178695C
:106A8000C7F80C80FAF7F0F9FD6806461DB93348DF
:106A900030F078F91DE709F1FF39B9F1040F00F280
:106AA0003381DFE819F00500AF00E30031012F0169
:106AB000D7F814A01AF00F0F40F02981BBF1000F96
:106AC0004ED0013D0F3405F10109BAF1000F4FD04E
:106AD00007F11801A4F1100328468B4613F801CFE3
:106AE00011F8012B9C4282EA0C0200F8012FF5D12B
:106AF0004A46494607F138001BF09CF94A465B4676
:106B000005F1110E106851689C46ACE8030008328C
:106B100072456346F6D1AAF1100A10351034D2E757
:106B200024EE0500A51F060027EE05002BEE05004C
:106B30002FEE050033EE050037EE05003BEE0500B5
:106B400052EE0500B1D30500E3D50500C8D7050016
:106B5000C8E30500C8DB0500C8DF05007CEE0500C2
:106B60000F35A24407F5A8795445A5F10F0222D1AB
:106B7000002340F21912184607F138011944013375
:106B8000934240F0C780B8F1000F3FF4A8AE4046F2
:106B9000FFF702FE002E3FF49CAEF389A3F50073CD
:106BA0009BB2F381F38913F4F0547FF492AE304634
:106BB00031F0DCFC8DE62346CE4604F1100B18685C
:106BC0005968F446ACE8030008335B45E646F6D165
:106BD000214607F138001AF0CFFF07F11801A5F19F
:106BE00010038C4613F8010F11F8012B9D4282EA25
:106BF00000021A70F6D199E80F0010348CE80F00EB
:106C00001035B1E77B69E3187B6007F5A87A07F1D7
:106C100018097B68A342ABD099E80F008AE80F00FF
:106C20004A46494607F138001BF004F9BBF1000F52
:106C300002D123788AF8103099F8003014F8012B2B
:106C4000534005F8013BBBF1000F01D08AF810302A
:106C500007F25113CC4607F2611E18685968624664
:106C600003C2083373459446F7D1D2E707F5A87BF2
:106C700010220021584607F1280AF8F753FC102289
:106C800000215046F8F74EFC7A694FF00009A3182E
:106C90009C423FF46DAFB9F1000F0BD01AF80920F8
:106CA00014F8011B09F101094A4005F8012B09F00C
:106CB0000F09EDE75946524607F138007B601BF09B
:106CC000B9F87B6807F5B07111F8012D0132D2B225
:106CD0000A70002AE2D18B45F6D1DFE7FA68611924
:106CE0002A4407F13800BBF1000F08D01BF0A2F8CE
:106CF00010357A6905F10F039A42EFD838E71AF098
:106D00003BFFF5E70025F4E7DFF82C8030E76FF074
:106D100021082DE708702FE74FF00109CAE54FF071
:106D20000209C7E54FF00309C4E54FF00409C1E5C6
:106D30004FF00509BEE500BF80AFFFFF0023FFF75E
:106D40005BBD0123FFF758BD70B50022164905460B
:106D50002EF0C6FF2EF022F9144B154906460322E9
:106D600058682EF0BDFF044678B10022B1B22DF074
:106D700069FDE389A3F500739BB2E381E38903F422
:106D8000F05313B9204631F0F1FB0A4B1C6824B1D3
:106D9000E38903F500739BB2E3812846002113F0D9
:106DA0002BFD204670BD00BF71E80500682D002056
:106DB0007EE80500DCD1002008B540B2FFF722FBD9
:106DC000BDE8084013F004B938B5054608460C463E
:106DD00031F039FA002808BF002422460E4928461F
:106DE0002DF0A4FD0D4B4FF6FF72198874B18A4245
:106DF00004D10020BDE8384013F0EAB8002218881A
:106E0000114614F053FA0828F4D1F2E78A42F0D080
:106E1000188814F049FAF6E74CE80500B42C002075
:106E2000014B188813F0EEB8B42C0020014B1888E1
:106E300013F0E8B8B62C002008B5074B1A884FF6B7
:106E4000FF71914207D018881321FDF705FDBDE8B9
:106E5000084013F0BDB808BDB62C002007B50023CC
:106E60000846072269460093CDF803302DF0C4FA96
:106E7000094B1A884FF6FF71914209D018886A466B
:106E8000012114F03FFA13F0A3F803B05DF804FBFE
:106E900043F20200F7E700BFB42C002038B500220F
:106EA0000E4905462EF01CFF0446A8B90C4927F0F0
:106EB0002FF80A490446024628462DF037FD2A4697
:106EC000084920462DF032FD002030F039FF0649F8
:106ED000024620462DF04DFD204638BD26E805002F
:106EE0002BE8050045E8050067E8050010B50446F5
:106EF00031F06AF9224630B92CB107490320BDE8C8
:106F000010402EF06BBC054B054958682EF04CF92B
:106F1000BDE8104013F000BBD3EC0500682D002045
:106F2000FCEC0500F8B5044628B9214A136823F49F
:106F300080431360F8BD1F492DF094F90028F4D167
:106F4000204631F090F9054690B1194A1368204661
:106F500043F4804313602FF0E5F953EC102B10EE4F
:106F6000100A194616F06CF8BDE8F84013F030B876
:106F7000204631F029F90028DCD00D4A0E4913686B
:106F800043F48043136020462A462EF0A9FE2FF0DA
:106F90002FFE2A4606460F46204608492EF0A0FE40
:106FA0002FF026FE02460B4630463946DAE700BF90
:106FB000E0D100209FEB0500A4EB0500B0EB05003D
:106FC000084B1A6818B142F400521A60704722F454
:106FD00000521A60044B1860044B01221A7012F020
:106FE00099BD00BFE0D10020F0D10020EFD10020FA
:106FF000F0B583B0044600AF28B9014612F0C6FDD3
:107000000C37BD46F0BD31F04DFA28B120462DF0C9
:1070100087FA0421C0B2F1E77860391D20462DF0CF
:10702000A4F90546F0B920462FF018F80646786016
:107030002BF044FB06F58073834208D90D490120EB
:107040002EF0CCFB0C4901202EF0C8FBD8E7F31D35
:1070500023F00703ADEB030D6D463246294620466B
:107060002EF0ECFF79680029ECD0284612F0C0FD24
:10707000C6E700BFB1D3050006F4050008B5044B10
:10708000044958682EF076F8BDE8084012F0E8BDD3
:10709000682D002046F40500F0B583B0044600AF2B
:1070A00012F0DEFD002C69D00023391D20467B60E4
:1070B0002DF05BF9054610BB20462EF0CFFF0646AB
:1070C00078602BF0FBFA06F5807383420CD93A49BD
:1070D00001202EF083FB394901202EF07FFB002494
:1070E00020460C37BD46F0BDF31D23F00703ADEB82
:1070F000030D6D463246294620462EF09FFF7868E4
:107100000028E8D030F0DEFE044608B92C49E3E759
:107110002C4B2D49024658682DF008FCE389A3F555
:1071200000739BB2E381E38903F4F05313B9204663
:1071300031F01CFA20462CF013FA7A68294636F012
:1071400059F820462CF00CFA054620462DF0E4F8BC
:107150000146284612F094FD0023391D0A207B6069
:10716000F9F782FE7B680446002BB9D0174A1168F4
:1071700019605168596012891A81B1E7204630F0D0
:10718000A1FE044620B90E4901202EF027FBA7E7F7
:107190000C4B0D49024658682DF0C8FBE389A3F556
:1071A00000739BB2E381E38903F4F053002BC8D151
:1071B000204631F0DBF9C4E7B1D3050006F4050041
:1071C0001DF40500682D002046F40500DFCE0020E8
:1071D000F0B583B0054600AF48B9424B4249586804
:1071E0002DF0C8FFFFF74AFF0C37BD46F0BD002366
:1071F000391D7B602DF0B9F80646F0B928462EF00F
:107200002DFF044678602BF059FA04F58073834211
:1072100008D9364901202EF0E1FA354901202EF037
:10722000DDFAE1E7E31D23F00703ADEB030D6E4646
:107230002246314628462EF001FF78680028ECD01F
:10724000133030F03FFE054608B92A49E6E7254BE2
:107250002549024658682DF069FB28462CF080F934
:10726000EB89A3F500739BB2EB81EB8903F4F05338
:10727000044613B9284631F079F91F4B224603F131
:10728000100153F8040B42F8040B8B42F9D11B8810
:1072900013807D6831462A4604F1120035F0AAFFBA
:1072A00065742544FE23AB740020FFF7F5FE3946D4
:1072B00005462DF05AF828B10368236043686360DF
:1072C00003892381002D8FD0EB89A3F500739BB236
:1072D000EB81EB8903F4F053002B85D1284631F084
:1072E00045F981E7682D0020FEF30500B1D30500C4
:1072F00006F405001DF40500C8D505002DE9F04190
:1073000082B0054600AF50B9594B5A4958682DF024
:1073100031FFFFF7B3FE0837BD46BDE8F08131F01D
:1073200054F828B92A46544903202EF057FAF2E7B8
:107330000023391D28467B602DF017F80446F0B96C
:1073400028462EF08BFE064678602BF0B7F906F53E
:107350008073834208D9494901202EF03FFA4849F9
:1073600001202EF03BFAD6E7F31D23F00703ADEB27
:10737000030D6C463246214628462EF05FFE7D689E
:10738000002DECD007223F49204635F025FF60B99B
:10739000073D07347D604FF0030878681B3030F0FC
:1073A00091FD064680B93849DAE708223749204678
:1073B00035F012FF28B9083D08347D604FF004080D
:1073C000EBE74FF00008E8E7294B2A4902465868E6
:1073D0002DF0ACFA30462CF0C3F8F389A3F5007316
:1073E0009BB2F381F38903F4F053054613B9304699
:1073F00031F0BCF8264B2A4603F1180153F8040B70
:1074000042F8040B8B42F9D11B8813807E6885F803
:1074100019802146324605F11A0035F0EBFEF3B231
:1074200003F108022E440133EB75FE236A74002039
:10743000B376FFF731FE394604462CF096FF28B1AB
:1074400003682B6043686B6003892B81002C3FF439
:1074500062AFE389A3F500739BB2E381E38903F490
:10746000F053002B7FF457AF204631F07FF852E7FE
:10747000682D0020FEF3050092F30500B1D305004E
:10748000ADF30500C4F30500D5F30500CCF305000A
:10749000C8D5050010B5044630F0D5FE084B0949A3
:1074A000002808BF0024224618682DF03FFA201C4F
:1074B00018BF012013F0FCFEBDE8104012F088BD9B
:1074C000682D00204CE805002DE9F74F504B51493D
:1074D0000546032258682EF003FC0646002845D0D6
:1074E00000224D49DFF8308128462EF0F9FB314665
:1074F000814668462BF0C3FB009CECB120462EF081
:1075000014FB0022414607462EF0EAFB012300222D
:1075100049468246F9F740F958BBFB8903F50073E9
:107520009BB2FB813C465046394631F039FB6846F8
:107530002BF090FB002CDFD0009850B1C389A3F54D
:1075400000739BB2C381C38903F4F0530BB931F0CC
:107550000DF82946002C57D001A82BF090FB019D77
:107560004DB932464946204631F0EEFA03B0BDE847
:10757000F08F0024D7E7EB8903F500739BB2EB8112
:1075800028462EF0D2FA01222946074620462DF041
:1075900057FB2249804628462CF064FE204982464B
:1075A00028462CF05FFEBAF1000F00D1D0B1404662
:1075B0002EF0BBFA834610B3BAF1000F1BD00122A4
:1075C000394630F0FAF8BBF80E20A2F5007292B2FC
:1075D000ABF80E20BBF80E2002F4F05212B9584658
:1075E00030F0C4FF40463A46294631F0ADFA01A8D2
:1075F0002BF030FBB3E739462EF04FFBE3E739467B
:1076000040462BF0F3FEEDE730462DF0D3F8A8E727
:10761000682D002053E90500ADEA05005AE9050090
:1076200063E90500F8B5064608460C4630F0CCFD87
:10763000074620B30022394920462EF051FB2DF099
:107640002EFE00220746364920462EF049FB04460E
:10765000E0B130F0B1FDC8B9E389A3F500739BB286
:10766000E381E38903F4F05313B9204630F07EFF41
:1076700022462C490320BDE8F8402EF0AFB82CB1CB
:107680002246294903202EF0A9F83C46304630F026
:10769000DAFD00283AD0002E38D048F248012348BD
:1076A00030F0CEFB0546D0B12246002131F004F97E
:1076B00032461F4928462DF039F91E4B1E491868DD
:1076C0002A462DF033F9EB89A3F500739BB2EB81C9
:1076D000EB8903F4F05313B9284630F047FF301C10
:1076E00018BF0120394612F04BFB12F071FCA4B117
:1076F000E389A3F500739BB2E381E38903F4F053BC
:107700005BB92046BDE8F84030F030BF094B0A496C
:1077100018682DF02FFD0026E1E7F8BDC6EB050047
:107720006FEA0500CDEB050001EC0500F5780200DD
:107730001AEC0500682D00201FEC05002DE9F84328
:1077400080460C4630F07FFD30B938494246012072
:10775000BDE8F8432EF042B8204630F084FD0546DF
:107760002046C5B12EF0DEFD57EC106B00243246EA
:107770003B463046394635F0C3FA30B900222C4B2F
:107780003046394635F094FAC8B12A490120BDE89F
:10779000F8432EF023B830F017FD50B12A462649A1
:1077A00020462EF09DFA40B12FF022FA06460F46F1
:1077B000DDE714B122462149C9E7214F0026214DBA
:1077C000D5F8049030F046FB1F49024648462DF09C
:1077D000D0F842461D4968682DF0A8F808211C48D9
:1077E00030F02EFB054670B12146FFF71BFFEB89F9
:1077F000A3F500739BB2EB81EB8903F4F05313B94B
:10780000284630F0B3FE0021124830F019FB044640
:1078100048B1002147EC106B0DF0B6FA2146BDE8E7
:10782000F84331F0BDB9BDE8F88300BFE9E80500D1
:10783000000024403AE9050042E9050017E9050087
:1078400000409F40682D002053E905004AE90500EB
:10785000C97402005978020037B5144C002108465B
:10786000FFF7E0FE0322124960682EF039FA002289
:107870000190104960682EF033FA0D4905466068A2
:107880002DF078FC0B4960682DF074FC019B33B13E
:107890002DB1012301AA2946002023F091FD29469C
:1078A000019831F07DF903B030BD00BF682D002094
:1078B00053E905004AE905001FB54FF08052D2F8A0
:1078C000A430D2F8A820D8B20290C3F307200190C8
:1078D000C2F30721C3F3074000901B0ED2B241F060
:1078E000C00103482FF090FB05B05DF804FB00BF1A
:1078F0006FE905002DE9F04F8BB000AFC7E9020139
:107900001446002A76D09E49002026F001FB002272
:10791000054638619B4920462EF0E2F99949024616
:1079200028462DF026F8002297493D6920462EF082
:10793000D7F99549024628462DF01BF830F08AFA0F
:10794000804604F0A4FE00228346904920462EF093
:10795000C7F98146E8B102468C4938692CF0E6FF48
:10796000002307F1240148467B622CF0FEFC04460C
:1079700000284ED148462EF071FB054678622AF069
:107980009DFE05F58073834238D9814901202DF091
:1079900025FFB8F1000F07D0D8F8003023B14246D8
:1079A0007C4938692CF0C2FF58462CF0B5FC20B158
:1079B0005A46794938692CF0B9FF5A46414648463B
:1079C00031F0C2F8FB68002B40F0C08007F11003D3
:1079D00001220021B86827F09BF8386950B1C389AB
:1079E000A3F500739BB2C381C38903F4F0530BB9B1
:1079F00030F0BCFD2C37BD46BDE8F08FEB1D23F009
:107A00000703ADEB030D6C462A46214648462EF08F
:107A100015FB7B6A002BBCD0B8F1000FC4D0BBF1C2
:107A2000000FB6D0002514E0092A09D1A91C214471
:107A3000701ED7F810A030F063FF5849024619E0D5
:107A4000911E012927D89A4602239E4216DA013652
:107A500035447B6AAB429CD96319665D5A78082A23
:107A6000E2D1A91C2144701ED7F810A030F048FFC5
:107A70004B49024650462CF07CFFE8E73AF8021FDB
:107A800048487B602FF0C0FA014640462CF0C6FE05
:107A90007B680233D9E7911F012908D8A81C20442C
:107AA0001BF016F8014640462CF0B8FECFE7162A28
:107AB00033D159883B482FF0A7FA30F094F882462A
:107AC0000028C4D00122014658462DF0B9F8291DDE
:107AD00078602144F01E2BF061FB7B6802463BB1CD
:107AE00030B10146386018462BF080FCD7E90023FE
:107AF0001846114631F054F8BAF80E30A3F5007369
:107B00009BB2AAF80E30BAF80E3003F4F053002BF3
:107B10009DD1504630F02AFD99E7FF2A97D1D878B9
:107B20009B78D7F810A043EA002030F011F91E49E5
:107B3000024650462CF01DFF291D2144F01ED7F8A7
:107B400010A02BF02BFB1949024693E7D7E9031647
:107B500007F114002BF093F8786948BB0446786964
:107B600050B1C389A3F500739BB2C381C38903F4E9
:107B7000F0530BB930F0FAFC002C7FF427AF2CE760
:107B800090EC0500ADEA050052E8050018F4050088
:107B9000B1D305005AE9050063E905006EF405005C
:107BA000A0EC050067400600AAEC0500B7EC050054
:107BB0002DF0BBFF0022BA4905462EF091F8804611
:107BC000002800F00F810022B54930462EF088F8D9
:107BD0004146814607F118002BF051F80124B8699D
:107BE000002840F0CC804946404630F0D9FF0022C2
:107BF000AC4928462EF074F88046E0B10022A9492D
:107C000030462EF06DF88146404630F017FC0028D3
:107C100000F0EA80484630F011FC002800F0E480D3
:107C2000494640462BF0E8FF00284946404608BF39
:107C3000002430F0B5FF00229B4928462EF050F872
:107C4000804610B30022974930462EF049F881460D
:107C5000404630F0BAFB98B1484630F0B6FB78B1F8
:107C600040462CF025FB824648462CF021FB8245FD
:107C700006D80123002249464046F8F78DFD00B1A1
:107C800000244946404630F08BFF002287492846B1
:107C90002EF026F8804680B10022844930462EF02E
:107CA0001FF80146814640462BF0A6FF49460028B2
:107CB000404608BF002430F073FF00227C4928466C
:107CC0002EF00EF88046F0B130F07EFA60B14146F9
:107CD00007F124002AF0D3FFDFF8D4A1D7F824B0AD
:107CE000BBF1000F40F09480B8F80E30A3F500739C
:107CF0009BB2A8F80E30B8F80E3003F4F05313B965
:107D0000404630F033FC00226A4928462DF0E8FF57
:107D10008046F0B130F058FA60B1414607F12400D6
:107D20002AF0ADFFDFF894A1D7F82490B9F1000F45
:107D300040F09980B8F80E30A3F500739BB2A8F814
:107D40000E30B8F80E3003F4F05313B9404630F05B
:107D50000DFC5DB1EB89A3F500739BB2EB81EB8960
:107D600003F4F05313B9284630F000FC07F1140077
:107D70002AF070FF002C3FF4EFAE0124EFE6B9F1DA
:107D8000000F12D02DF0D1FE014607F11C001AF0B1
:107D90001BFE494607F120002AF071FF4FF0000A50
:107DA000386A40B9BAF1000F00D1002407F1180079
:107DB0002AF050FF13E72DF0B8FE014607F124002A
:107DC0001AF002FEBA7F97F826309A4205D1BA8B94
:107DD000BB8C9A4208BF4FF0010A07F120002AF03D
:107DE00039FFDDE7012402E7334BA8EB0300001164
:107DF000013082B2B9F1000F08D0A9EB03000011E5
:107E0000013080B2131A584258410DE74846F9E74D
:107E1000BBF80E3003F500739BB2ABF80E300022B6
:107E2000514630462DF05CFF814648B90024584643
:107E3000494630F0B5FE07F124002AF00BFF4DE76C
:107E4000002259462CF0FCFE0028EFD0C389A3F590
:107E500000739BB2C381C38903F4F053002BE6D1B6
:107E600030F084FBE3E7B9F80E3003F500739BB202
:107E7000A9F80E300022514630462DF031FF8346DE
:107E8000014648462BF0B8FE59460028484608BF30
:107E9000002430F085FE07F124002AF0DBFE43E7E2
:107EA0005AE905006EF40500C8EC0500ADEA0500CE
:107EB00063E90500B7EC0500882D0020AAEC050059
:107EC0002DE9F04186B000AF00238846391D0646F3
:107ED0007B602CF04AFA0546E0B930462EF0BEF839
:107EE000044678602AF0EAFB04F58073834206D9E1
:107EF0003F4901202DF072FC32463E4938E0E31D37
:107F000023F00703ADEB030D6D46224629463046AC
:107F10002EF094F87B68002BEED0404630F093F9B9
:107F200028B1354B3549186842462CF0FFFC344BDC
:107F30001A6812F0400F1E4607D1324901202DF079
:107F40004DFC1837BD46BDE8F0812F4A12884FF628
:107F5000FF71914201D12D49F0E71A6812F08002B9
:107F600001D02B49EAE77C68102C05DD2949102255
:107F700001202DF033FCE4E7274B93F800C0274B9A
:107F8000A4B2BCF1000F23D19A7C62B3B3F876019E
:107F900088422AD09B8A7C80C7F80AC0A7F80EC006
:107FA0003B810123BB7207F10801BB1CC7E9043503
:107FB000FBF754FC18B97B88A34218BF0C2012F0C1
:107FC00007F80028BDD1336843F080033360B8E779
:107FD000B3F87601884208D07C80C7F80A20FA817D
:107FE000B3F84E31DCE70720E9E70820E7E700BFF8
:107FF000B1D3050016EB0500682D0020A6EA0500A8
:10800000E0D10020B0EA0500B62C0020C4EA05004B
:10801000D3EA0500EBEA0500EED1002048CC0020B1
:108020002DE9F04FB04B91B01B681B0700AF044621
:1080300007D5AE4901202DF0D1FB4437BD46BDE840
:10804000F08F15F077F8204630F0BEF88046002813
:1080500000F05E81214607F114002AF010FEDFF8DF
:10806000ACA2796981B10023BB61CB8903F50073B0
:108070009BB2CB8107F118001AF0A6FC024698B11A
:108080009B4901202DF0AAFB78690028D5D0C3892F
:10809000A3F500739BB2C381C38903F4F053002B93
:1080A000CBD130F063FAC8E77D691DB128462DF0C9
:1080B0003CFD0546294607F11C002AF0E0FDF96960
:1080C000B8F1000F0FD071B1CB8903F500739BB2EB
:1080D000CB8107F120001AF077FC024610B38549E6
:1080E00001202DF07BFBF86950B1C389A3F5007323
:1080F0009BB2C381C38903F4F0530BB930F036FA55
:108100005DB1EB89A3F500739BB2EB81EB8903F4BE
:10811000F05313B9284630F029FA07F114002AF079
:1081200099FD9EE707F128003C8C97F822601AF031
:108130000FFD08B1F9F740FC4FF00009002207F1EC
:108140003001388DC7F830901AF000FD052810D0A6
:1081500043F2030290420CD0A8B93B8EA34214D143
:1081600097F83230B34210D1B7F82890B9F1000F28
:108170000FD1386A1AF0C2FC5F490446024601205A
:108180002DF02CFB48E0F9F717FC3B8D01333B85C4
:10819000D4E7FC691CB120462DF0C7FC0446002240
:1081A000564920462DF09CFD0022554906462046A2
:1081B0002DF096FD2DF073F80022B860514920464D
:1081C0002DF08EFD2DF06BF8F8602EB3002307F133
:1081D000240130467B622CF0C8F88346002837D152
:1081E00030462DF03BFF786278602AF067FA7A68B3
:1081F00002F58073834221D9434901202DF0EEFA24
:10820000F389A3F500739BB2F381F38903F4F05370
:1082100013B9304630F0AAF95CB1E389A3F50073D5
:108220009BB2E381E38903F4F05313B9204630F0A5
:108230009DF907F11C002AF00DFD40E7D31D23F046
:108240000703ADEB030DEB46594630462DF0F6FE25
:108250007A6A002AD4D0002179853A85494607F107
:108260002802BAF80000C7F82CB0FDF7A5FD11F000
:10827000AFFEBB6880F001005FFA80F813B9FB68BD
:10828000002BBDD0BAF800204FF6FF719142B7D055
:10829000FB68BAF80000A7F830900022002BC7F85E
:1082A0003220FA867A6A7A8214BF0222012287F883
:1082B000322007F1300107F11202C7E90E2BFBF75C
:1082C000CDFA30F008029BD043F20402904297D0DE
:1082D00043F20142904293D011F07AFE002818BF79
:1082E0004FF000088CE700BFE0D1002069ED0500E9
:1082F00091ED0500AAED0500DAED05005114060028
:10830000CAED0500D1ED0500B1D30500B62C002063
:10831000002C3FF492AE2246024903202DF05EFA73
:108320008BE600BFFEED05002DE9F04F9BB000AFDE
:108330000D4604463C22002107F12C00F7F7F2F825
:10834000022387F82C302846062387F82F302FF099
:108350003BFF002800F08D8000228E4928462DF03A
:10836000BFFC38B12CF09BFF002814BF0223002370
:1083700087F82C300022884928462DF0B1FC38B10E
:108380002CF08DFF002814BF0623052387F82F301B
:108390000022824928462DF0A3FC064618B300238C
:1083A00007F10C01FB602BF0E0FF804600284ED166
:1083B00030462DF053FE8146F8602AF07FF909F52A
:1083C0008073834237D9764901202DF007FAF3896B
:1083D000A3F500739BB2F381F38903F4F05313B94F
:1083E000304630F0C3F8284600226E492DF078FC64
:1083F000054690B13B6D002B36D02CF091F83B6DCB
:108400001880EB89A3F500739BB2EB81EB8903F431
:10841000F05313B9284630F0A9F820462FF0CCFECF
:1084200080B3E38903F500739BB2E38120466C3788
:10843000BD46BDE8F08F09F1070323F00703ADEB5C
:10844000030DE8464A46414630462DF0F7FDFA68EE
:10845000002ABCD084B06B464FF6FF713B65198093
:108460009A80C3F80880B2E74F4903202DF0B6F98F
:10847000C7E7002DD1D04D492A4603202DF0AEF993
:108480000024D3E720462FF07BFE06460028C8D103
:1084900020462FF099FE002876D020462AF086FF4D
:1084A0000C235843073020F00700ADEB000D2146A8
:1084B00007F108002AF0E3FBE946DFF8E4B04D4697
:1084C000B246B868C0B987F85860C7F854901F23FF
:1084D00007F1080207F10C0107F12C003B81FCF7C2
:1084E00063FA11F075FD0028CAD107F10C01388933
:1084F0002AF054FE044699E72DF017FB07F10C0112
:108500000446C7F80CA02BF030FF804678B920460F
:108510002DF0A4FDF86078602AF0D0F87A6802F5B2
:108520008073834225D9594601202DF057F95CB15B
:10853000E389A3F500739BB2E381E38903F4F0536D
:1085400013B9204630F012F8B86820B1C38903F59A
:1085500000739BB2C3812CF021FDFB682880AB80A7
:10856000C5F8088007F108002AF074FB01360C35C5
:10857000A7E7D31D23F00703ADEB030DE846414603
:1085800020462DF05BFDD2E7002CA0D02246084902
:1085900073E700BF8DE9050096E90500B7EC05001B
:1085A000B1D30500AAEC0500A3E90500D7E9050051
:1085B0000DEA050008B5054A136823F4007313603B
:1085C00011F098FDBDE8084011F002BDE0D1002097
:1085D00008B5054A136843F40073136011F0FAFB01
:1085E000BDE80840FEF728BCE0D1002008B512F035
:1085F000ABFF41EC100B08BD08B50C4B1B884FF6C8
:10860000FF729BB2934203D1094A1288934208D069
:10861000084824F0F5FC084A136843F00803136087
:1086200008BDBDE8084014F0E9BA00BFB42C002032
:10863000B62C002077EA0500E0D1002038B50F4CB9
:108640000F490022054660682DF04AFB2CF0A6FC7D
:10865000C3B27DB143F0010098420ED064682FF0A0
:1086600077FB0749024620462CF083F9BDE83840E5
:10867000FFF7C2BF03F0FE00EEE738BD682D002013
:10868000BCEB05002DE9F0418CB006460F462FF0FB
:108690009BFD40B93EB13246524903202DF09EF871
:1086A0000CB0BDE8F0810023029301934E4B03937D
:1086B00002AB05934D4B06934FF003080B23ADF827
:1086C0001C300DEB080301220893494B8DF8032061
:1086D0000993424601AB03A93846ADF81080ADF8C6
:1086E00028800B932EF022F80028D9D00298414D13
:1086F000414C2FF087FE48B1029A404968682CF03F
:1087000015F9236843F00803236009E0029B002B5E
:108710004AD13A4968682CF02DFD23685906F0D4F7
:10872000029850B1C389A3F500739BB2C381C3897A
:1087300003F4F0530BB92FF019FF9DF80330002B11
:1087400037D023682E4968689A065EBF236843F0D5
:10875000080323602CF00EFD32462A4968682CF08D
:1087600023FD3A46284968682CF01EFD019A1AB18B
:10877000236843F008032360244968682CF014FD43
:10878000019850B1C389A3F500739BB2C381C3891B
:1087900003F4F0530BB92FF0E9FE236813F0180F20
:1087A0001BD0FFF729FF7BE7194940462DF016F84B
:1087B000B6E72368D5F804809B0648BF23684FF0CE
:1087C000000044BF43F0080323602FF0B9FA0C49BE
:1087D000024640462CF0CDF8BEE7304614F030FAA1
:1087E0005EE700BFFEED0500ACEA050004ED050004
:1087F00009ED0500682D0020E0D1002013ED0500F3
:1088000042ED05004BED050055ED05005FED05005F
:108810001DED050013B5694604461AF0E9F828B9BC
:10882000074901202CF0DAFF02B010BD054B0649C4
:10883000586822462CF07AF8FFF7DEFEF4E700BF16
:108840002EEB0500682D002064EB050070B50D4D82
:108850002A7806460C462AB101200B492CF0BEFFAF
:10886000002070BD09F04CF9084B2E70186024B13F
:10887000E38903F500739BB2E381054B01201C6083
:10888000EFE700BFE4D1002003E80500DCD10020C1
:10889000E8D1002037B50546002105208DF80610E7
:1088A000FFF7D4FF70B1084B1C6824B1E38903F5CE
:1088B00000739BB2E3810199284611F001FB204629
:1088C00003B030BD0446FAE7DCD1002037B50546D9
:1088D0000C4605200021FFF7B9FFD0B1214601A8C1
:1088E00019F0B2FF024638B10B4901202CF076FF97
:1088F0000024204603B030BD084B1C6824B1E38936
:1089000003F500739BB2E3810199284611F0D8FA70
:10891000EFE70446EDE700BF6E0B0600DCD1002058
:1089200013B5002104208DF80610FFF78FFF68B102
:10893000074B1C6824B1E38903F500739BB2E38104
:10894000019811F00DFB204602B010BD0446FAE775
:10895000DCD1002013B50C4604200021FFF776FF80
:10896000C8B1214601A819F06FFF024638B10B4982
:1089700001202CF033FF0024204602B010BD084B2C
:108980001C6824B1E38903F500739BB2E38101986D
:1089900011F0E6FAF0E70446EEE700BF6E0B0600C2
:1089A000DCD1002038B5124D2A8801464FF6FF7001
:1089B000904215D00320FFF749FF78B10D4B1C689A
:1089C00024B1E38903F500739BB2E3811321288866
:1089D000FBF742FF11F0FCFA204638BD0446F5E7EC
:1089E000FDF70EFDBDE83840084609F0FDB800BFB0
:1089F000B42C0020DCD100202DE9FF4100220F46DD
:108A0000314980462DF06CF90022304906462DF0A0
:108A100067F96946054619F0EBFF044658B929463F
:108A2000304630F0BDF82A4903202CF0D7FE20460E
:108A300004B0BDE8F0815EB1F389A3F500739BB289
:108A4000F381F38903F4F05313B930462FF08EFD10
:108A500041460220FFF7FAFE80B90024002DE6D03F
:108A6000EB89A3F500739BB2EB81EB8903F4F05320
:108A7000002BDCD128462FF079FDD8E74821154896
:108A80002FF0DEF904460028E7D00223014602AAAF
:108A90000020CDE9025722F093FCE389A3F500738F
:108AA0009BB2E381E38903F4F05313B920462FF01E
:108AB0005DFD094B1C68002CD0D0E38903F50073E1
:108AC0009BB2E381CAE700BF45E80500ADEA0500B7
:108AD000A5E80500A1B60200DCD1002070B504466F
:108AE0000E460020184925F013FA054610B9002556
:108AF000284670BD224615492BF018FF2846FEF780
:108B0000CDF9EB89A3F500739BB2EB81EB8903F4FC
:108B1000F053044613B928462FF028FD002CE6D068
:108B200031462046FFF768FFE389A3F500739BB247
:108B3000E381E38903F4F0530546002BD8D12046A6
:108B40002FF014FDD4E700BF90EC0500ADEA05005E
:108B50002DE97043064658B12FF036FB044638B96C
:108B600032464E4903202CF039FE2046BDE8708382
:108B700000224B4930462DF0B3F804462FF01CFB81
:108B800098B95CB1E389A3F500739BB2E381E389F3
:108B900003F4F05313B920462FF0E8FC2246414974
:108BA00003202CF01BFE0024DFE75CB1E389A3F572
:108BB00000739BB2E381E38903F4F05313B92046B9
:108BC0002FF0D4FC0022384930462DF089F82EF0E1
:108BD0000FF802460B468046894634F091F830B9CA
:108BE000002200234046494634F06CF818B1DFF803
:108BF000C8904FF0000800212C482FF021F90446BE
:108C0000002846D0002149EC108B0CF0BDF8E38918
:108C1000A3F500739BB2E381E38903F4F0530546A7
:108C200013B920462FF0A2FC29460120FFF70EFEC3
:108C3000002830D008211E482FF002F9044670B1F8
:108C40003146FEF7EFFCE389A3F500739BB2E381A5
:108C5000E38903F4F05313B920462FF087FC154B3A
:108C60001C6824B1E38903F500739BB2E381002DF6
:108C70003FF47BAFEB89A3F500739BB2EB81EB89EB
:108C800003F4F053002B7FF470AF28462FF06EFCF6
:108C90006BE70546C8E70446E9E700BF3AEA050086
:108CA0006FEA0500CDEB050042E90500B5B2020010
:108CB0000DB80200DCD1002000409F4030B50021FB
:108CC0008FB0044609202FF01BFE154D019002467F
:108CD00080B114496868FF23CDE9021300231249CB
:108CE0008DF810302BF045FE01A81AF059FF01A8AD
:108CF0001AF05CFF01A81AF053FF01A81AF042FF16
:108D000022460A4968682BF011FE094B02221A70AC
:108D1000E38903F500739BB22046E3810FB030BDB9
:108D2000682D00200300FFFF084506008EF30500B4
:108D3000F4D1002019F0FABF19F00CBF38B5054680
:108D400009B119F095FF0022124928462CF0C8FFFE
:108D50002CF0A5FA10B110482FF038FE0446014659
:108D6000284619F085FF5CB1E389A3F500739BB237
:108D7000E381E38903F4F05313B920462FF0F6FBA7
:108D800001202EF0DDFF054902462846BDE83840A7
:108D90002BF0EFBDEDD405005251060021F2050085
:108DA00008B519F065FF002008BD000070B58EB051
:108DB000044601A80E4615461CF030FBD8B12046EB
:108DC00000220E492CF08CFF0446A0B132460C491B
:108DD0002BF0ACFD2A460B4920462BF0A7FDE3897A
:108DE000A3F500739BB2E381E38903F4F05313B955
:108DF00020462FF0BBFB0EB070BD00BF00EF05009A
:108E000004EF050013EF050010B58EB0044601A86D
:108E10001CF004FB30B101A821461AF09DF901A80D
:108E20001AF0B0FE0EB010BD38B505462CF07DFE30
:108E300004462FF008FAA0B9214618482DF0A2FFE9
:108E400014B90024204638BDE389A3F500739BB212
:108E5000E381E38913F4F055F3D120462FF086FB2C
:108E6000EFE75CB1E389A3F500739BB2E381E3898B
:108E700003F4F05313B920462FF078FB0849002083
:108E800025F046F804460028DCD001211AF0F4F958
:108E90002A46044920462BF049FDD3E725F2050078
:108EA0004CF2050054F2050038B505462CF03DFEA5
:108EB00004462FF0C8F9A0B9214618482DF062FFEA
:108EC00014B90024204638BDE389A3F500739BB292
:108ED000E381E38913F4F055F3D120462FF046FBEC
:108EE000EFE75CB1E389A3F500739BB2E381E3890B
:108EF00003F4F05313B920462FF038FB0849002043
:108F000025F006F804460028DCD000211AF0B4F958
:108F10002A46044920462BF009FDD3E725F2050037
:108F20003EE8050054F2050030B591B0044603A8B0
:108F30000D461CF073FA48B1002303A800932A469B
:108F4000214619F0A3FF03A81AF01CFE002011B05F
:108F500030BD30B58FB0044601A80D461CF05EFA56
:108F600058B11DB129462046FFF7DEFF01A8214672
:108F70001AF0F2F801A81AF005FE0FB030BD00009B
:108F800030B58FB0054601A81CF048FA78B300212F
:108F90001A481AF07FF9044630B3294601A81AF09E
:108FA00033F92946012220462EF0E4FB054600B3A2
:108FB000014620462CF006F8EB89A3F500739BB21E
:108FC000EB81EB8903F4F05313B928462FF0CEFA66
:108FD000E389A3F500739BB2E381E38903F4F053C3
:108FE00013B920462FF0C2FA01A81AF0CBFD0FB03A
:108FF00030BD03482DF0A6FEEAE700BF4AF30500A6
:1090000050F305002DE9F04391B0814603A888464E
:1090100016461F461CF002FAB8B1002118982DF030
:109020004FF904462FF01FF980B330462BF078FA41
:10903000064638462BF074FA07461B202EF020FE19
:10904000054628B903A81AF09DFD11B0BDE8F083CC
:109050003B46324641462AF00EFC012118982DF07D
:109060002FF92646074630462BF05AFA80B2009078
:109070003B462A46494603A819F008FF4545E1D07A
:109080003A46314628462FF05FFDDBE70CB94546EE
:10909000E9E7E389A3F500739BB2E381E38903F475
:1090A000F053002BF3D120462FF060FAEFE70000D9
:1090B0002DE9F04F8BB0824601912FF086F920B94F
:1090C000002630460BB0BDE8F08F03F0E0FA06460C
:1090D0000028F5D04FF000094FF0FF35002251462F
:1090E00005A82AF045FACB462C46A8462F464A4604
:1090F0004946DDE905308342C0F0D780089850B179
:10910000C289A2F5007292B2C281C28902F4F05201
:109110000AB92FF02BFAB4F1FF3F08BF5C46B8F153
:10912000FF3F08BFA046002F09DD7A1E00215046F0
:109130002AF0E4FBBB49024630462BF01AFCBA4841
:109140002FF044FCB949024630462BF012FC791C42
:10915000A8EB010250462AF0D1FBB5490246304641
:109160002BF007FC6FF00042214650462AF0C6FB68
:1091700007462BF09DF818B9AE4938462AF0F1FBA6
:109180003A46AD4930462BF0F4FB691C14BF2A1B4C
:109190006FF00042214650462AF0B0FB04462BF007
:1091A00087F818B9A34920462AF0DBFB2246A349D9
:1091B00030462BF0DEFB6A1C00F0B9806FF00042F5
:1091C000294650462AF09AFB02469D4930462BF02C
:1091D000D0FB09F1FF324FF6FE739A4240F2AB80AA
:1091E00002202EF04DFD0246964930462BF0C1FB81
:1091F0006B1C00F0A4806FF00042691C50462AF0FE
:109200007DFB019B0446002B49D02EF09AFF0546BA
:10921000002844D10246214605A82AF0A9F903F006
:1092200036FA81461B202EF02BFD07461B202EF020
:1092300027FD8046DDE905239A42C0F08480089826
:1092400050B1C389A3F500739BB2C381C38903F4F2
:10925000F0530BB92FF08AF95CB1E389A3F50073E1
:109260009BB2E381E38903F4F05313B920462FF056
:109270007DF938462BF01CF8002800F0978038461E
:109280002EF0B1FC414607462FF00AFA394648460F
:109290002BF0E2F9414638462FF082FC4C4622463C
:1092A000694930462BF065FB0BE7099888B1C05C33
:1092B0002F2812D1B4F1FF3F08BF5C46012A01F10B
:1092C000010106D1022904D17B1C02D13D463C4656
:1092D0005F46B8F1FF3F0DD119E03A2807D17B1C5A
:1092E00002F10102F5D0631CF3D1D8460FE0B8F1CA
:1092F000FF3F16D0D84514DA631C40F090802F2829
:1093000005D9392803D830380A2303FB090905A8F1
:10931000CDE902210BF1010B29F040FDDDE902212D
:10932000E7E63F28F3D1601CF1D05D46EFE702206D
:109330002EF0A6FC48E748462EF00AFD53E702202F
:109340002EF09EFC5DE7099B002B53D09B5C262BE7
:1093500025D138462AF0ACFFC0B138462EF043FC88
:10936000414605462FF09CF9294648462BF074F9F2
:10937000414628462FF014FC1B202EF081FC0746A6
:109380001B202EF07DFC8046002504E040462AF09C
:109390008FFF0028E1D105A829F000FD4AE765B953
:1093A0003D2B31D1019DF6E7824611E040462AF07F
:1093B0007FFF00287FF463AF6CE7252B1BD105A846
:1093C00029F0ECFC09980028EED0059B10F803A0CA
:1093D00005A829F0E3FC504629F0C5FA00014FFA30
:1093E00080FA099808B1059BC05C29F0BCFA4AEAEA
:1093F0000000C3B255B101220DF1130140468DF8B2
:1094000013302AF08BFACDE7252BD8D001220DF1AD
:10941000130138468DF813302AF080FAB4E73F285C
:1094200083D074E751F405005AF405005EF405009A
:1094300011450600CAF3050065F405006AF405004D
:1094400073F405007AF405007FF405002DE9F04F70
:1094500091B0014602A81CF0FDFA28B94FF00009AE
:10946000484611B0BDE8F08F9DF81370012F06D06B
:10947000182F04D0464901202CF0B0F9EEE7BDF8D2
:109480000F50BDF811607D431F35012F4FEA651560
:109490000CBF4FF0200A4FF01A0AAD0005FB06A6DC
:1094A00030462EF00FFD81460028D7D02AF058F81C
:1094B000422303704D23437086700C233612C6700E
:1094C00080F80AA08373BDF80F3083741B0AC3743D
:1094D000BDF8113003751B0A43750123012F8375F5
:1094E0009DF81330037608BFFF23044602BF83763E
:1094F000C37603770022BDF811609642B0DD9DF877
:10950000133002F1010BA6EB0B06012B05FB06A69F
:1095100038D04FF0000817B2BDF80F3043452FDDAB
:109520003A460FFA88F102A81CF026FA9DF813308B
:10953000DB0808FB0363020AE0542344000C5A7062
:10954000987008F10108E7E700235B0039B2009A40
:10955000019302A81CF010FA0137019B00F00100F2
:10956000B84543EA0003F0D106EBE80208F1080829
:1095700002F8013CBDF80F30A8F10807BB42E3DC5C
:109580005A46B8E713B24FF0080800932644F1E7B3
:1095900051EF050038B5FFF759FF054610B9002512
:1095A000284638BD0BF0AAFEEB89A3F500739BB2E9
:1095B000EB81EB8903F4F053044613B928462EF0EF
:1095C000D5FF002CEBD0214608482DF01DFDE38986
:1095D000A3F500739BB2E381E38903F4F0530546DE
:1095E000002BDDD120462EF0C1FFD9E77FEF05002B
:1095F00010B5FFF7CFFF044668B123F04BFDE389B8
:10960000A3F500739BB2E381E38903F4F05313B92C
:1096100020462EF0ABFF0248BDE8104023F03EBDCF
:109620005151060030B58FB00C46014668461546CC
:109630001CF010FA20B12AB221B268461CF09CF945
:109640000FB030BD30B58FB00D46014668461CF0F6
:1096500001FA00284CD0BDF91B20BDF91F309A42F9
:1096600044DC03F014F8044618B3BDF91B002EF0D7
:109670006FFB2049024620462BF07BF9BDF91D0007
:109680002EF066FB1C49024620462BF072F9BDF90C
:109690001F002EF05DFB1949024620462BF069F9A8
:1096A000BDF921002EF054FB1549024620462BF04F
:1096B00060F9C5B100226FF07F038DF81F208DF88F
:1096C00020308DF821208DF822304FF0FF327F239B
:1096D00068468DF81B208DF81C308DF81D208DF804
:1096E0001E301CF07DF920460FB030BD0024E0E7AD
:1096F0000446F8E78EF1050091F1050094F10500AC
:1097000097F1050070B58EB004460D4601466846D7
:1097100016461CF09FF950B3BDF80530022D23F01A
:1097200070039BB21DD0032D1ED0012D08BF43F046
:109730003003ADF805304EB1BDF80530DA064CBF48
:1097400083F0400383F02003ADF8053068461CF039
:1097500047F9E38903F500739BB2E38120460EB01D
:1097600070BD43F06003E4E743F05003E1E70446D3
:10977000F4E770B58EB004460E46014668461546BD
:109780001CF068F970B16846ADF81660ADF8185075
:109790001CF026F9E38903F500739BB2E3812046B0
:1097A0000EB070BD0446FAE7F0B58FB004460E4621
:1097B0000146684615461F461CF04CF900B3012EC1
:1097C0009DF81A10A8BF0126012DA8BF012546EA61
:1097D000E67666F3010145EAE57565F3830187F3F3
:1097E000020767F3051168468DF81A101CF0F8F8A7
:1097F000E38903F500739BB2E38120460FB0F0BD0F
:109800000446FAE72DE9F0438FB004468846014646
:10981000684616461D46169F1CF01CF9002846D0C7
:1098200040462EF0D2FD40B9224901202BF0D6FF50
:10983000002420460FB0BDE8F083FF2E01D91E4959
:10984000F3E728462EF0C1FD28B928462EF02AFE5F
:1098500008B91A49E9E77B1EFE2B01D91849E4E74C
:109860004246184920462BF061F82A461649204600
:109870002BF05CF838462EF06BFA1449024620466D
:109880002BF077F830462EF063FA11490246204655
:109890002BF06FF84FF6FE736846ADF814301CF0ED
:1098A0009FF8E38903F500739BB2E381C1E70446A7
:1098B000BFE700BF9AF10500B7F10500D4F105003C
:1098C000FEF105000DF2050012F2050017F2050089
:1098D0001CF205002DE9F04317461D46421E47F6CF
:1098E000FE739A428FB08146884602D84A1E9A4239
:1098F00008D93D4901202BF071FF002420460FB00C
:10990000BDE8F0833846FCF77FFD044620B93749AF
:1099100001202BF063FFF1E728462EF055FCD8B16B
:109920000022334928462CF0DBF900220446314955
:1099300028462CF0D5F92546064628462EF083FC0D
:10994000044680B92A462C4901202BF047FF3146B6
:1099500028462FF025F9D1E7EB8903F500739BB278
:10996000EB810646E9E736B130462EF06CFC044642
:1099700008B93246E7E72149002024F0C9FA044635
:109980000028BBD000234FF0FF32CDE903238DF830
:1099900005308DF806304FF6FF730593069B184986
:1099A000009003F4400343F07F4343F47023069395
:1099B000144B07938023ADF820308DF822302A46CF
:1099C00001238DF80430ADF80790ADF809808DF8CB
:1099D0000B702AF0ABFF32460B4900982AF0A6FF25
:1099E00068461BF0FDFFB2E76BF0050078F005005C
:1099F00084F005008DF0050096F0050076EF050077
:109A0000CAF005007FFF7F00D4F005002DE9F0418A
:109A100092B006460D46014604A814461CF01AF8FA
:109A20004FF00008002869D00DF10A0202A904A82D
:109A3000ADF80C50ADF80E40ADF80880ADF80A80D6
:109A40001BF0F8FD0DF10E0203A904A81BF0F2FDB6
:109A5000BDF90830BDF90A20BDF90C50BDF90E4022
:109A6000ED1AA41A119B2246294604A89847DDE95D
:109A700007734545079326DDBDF81920013A12B258
:109A80006B1E00921BB24246414604A80F9DA84798
:109A9000002C26DDBDF81730013C013B24B20094B8
:109AA0001BB20022002104A80F9CA04704A807971E
:109AB0001BF096FFF38903F500739BB2F3813046E8
:109AC00012B0BDE8F081E3D0BDF81920BDF8171041
:109AD000013A4B1E12B2294400921BB2424609B20F
:109AE000D3E7E3D0BDF81910BDF817300A190139D2
:109AF000013B09B200911BB212B2D3E70646DEE782
:109B0000F0B58FB004460E460146684615461F461E
:109B10001BF0A0FFE0B1B7B9039B36B22DB22A46C5
:109B2000314668461BF048FF6846ADF81660ADF850
:109B300018501BF055FFE38903F500739BB2E381D6
:109B400020460FB0F0BD38462AF0EAFC0346E4E7B1
:109B50000446F5E72DE9F04F9DB004460D46014659
:109B60000EA8CDE905231BF075FF20B9002420467F
:109B70001DB0BDE8F08F28462EF026FB20B97649AF
:109B800001202BF02BFEF1E70022744928462CF02F
:109B9000A7F82BF003FA00227149029028462CF016
:109BA0009FF82BF0FBF900226E49009028462CF01C
:109BB00097F82BF0F3F9002201906B4928462CF01E
:109BC0008FF880462AF0ACFC0390B8F1000F0ED05D
:109BD000B8F80E30A3F500739BB2A8F80E30B8F8B1
:109BE0000E3003F4F05313B940462EF0BFFC284664
:109BF00000225E492CF074F805462EF0C1FAA8B197
:109C0000029B002B18DC5A4901202BF0E7FD002DA8
:109C1000ACD0EB89A3F500739BB2EB81EC8914F413
:109C2000F054A3D128462EF0A1FCA0E728462EF040
:109C3000CCFB0028E4D1E6E7009B002BE3DD019B91
:109C4000202BE0DC284629F063FC07465DB1EB8958
:109C5000A3F500739BB2EB81EB8903F4F05313B9C6
:109C600028462EF083FC019B012BB8BF01239B46A5
:109C700009AB00221846394629F07AFC012202FA83
:109C80000BF2531E0025049309AB2E46A946AA46A3
:109C900007935E455BDADDE909239A4202D2009B15
:109CA000994522DB0C9850B1C389A3F500739BB290
:109CB000C381C38903F4F0530BB92EF057FC5FB195
:109CC000FB89A3F500739BB2FB81FB8903F4F0537E
:109CD00013B938462EF04AFC0EA81BF081FEE3892A
:109CE00003F500739BB2E38141E72B020D9D0DB19B
:109CF000099AAD5C079808361D4329F04FF8B34523
:109D0000F3DCA6EB0B06049A25FA06F31340B8F130
:109D1000000F02D0039A9A420DD0019A012A01DC69
:109D20009BB1119B069A05994A44514412B209B25B
:109D30000EA81BF041FE029B0AF1010A5345DCBF4D
:109D400009F101094FF0000AA3E7129BEAE7009B23
:109D50009945D6DBA6E700BFF1F005001AF1050032
:109D600006F2050020F1050024F105009417060015
:109D700030F10500F0B5DBB004460D4601460CA8F5
:109D80001BF068FE18B9002420465BB0F0BD2846E1
:109D90002EF038FB0028F6D02946012201A829F030
:109DA000CCFF1AAE0025374601A828F032FF08B1D3
:109DB000802D16D101A828F0EDFE802D03D1402181
:109DC0000D482CF0BFFF3A4669100CA81BF052FC5E
:109DD0000CA81BF005FEE38903F500739BB2E38139
:109DE000D2E701A82BF0D0FE26F8020B01A801351E
:109DF0002AF00CFCD8E700BF5AF105002DE9F04F1E
:109E00009FB004460E46014610A803921BF022FEA6
:109E100020B9002420461FB0BDE8F08F30462EF058
:109E2000F1FA0028F5D03146012205A829F085FF76
:109E3000002605A828F0EDFEC0B905A828F0AAFE66
:109E4000039B53B12DB200950FFA8AF3BDF9582048
:109E5000BDF9561010A81BF013FD10A81BF0C0FD93
:109E6000E38903F500739BB2E381D3E705A82BF0E8
:109E70008BFEF307834616D5012E0FFA87F90FFAEA
:109E800080F816D0CDF800804B46BDF95820BDF9BA
:109E9000561010A81BF0F4FCAB465D46ADF856908A
:109EA000ADF85880BB4605A801362AF0AFFB5F46E7
:109EB000BFE7BA46F1E770B590B004460E460146DA
:109EC00002A815461BF0C6FDC8B136B22DB2334606
:109ED000BDF92020BDF91E10009502A81BF0D0FC92
:109EE00002A8ADF81E60ADF820501BF079FDE389A3
:109EF00003F500739BB2E381204610B070BD0446A9
:109F0000FAE7F0B591B004460D46014602A81646A0
:109F10001F461BF09FFD98B1BDF95830009332B237
:109F20003BB229B202A81BF0ABFC02A81BF058FD03
:109F3000E38903F500739BB2E381204611B0F0BDC5
:109F40000446FAE72DE9F04F95B004460D46014668
:109F500006A81BF07FFD002839D0BDF92C30023354
:109F600038D10022374920462BF0BAFE002236496C
:109F7000064620462BF0B4FE2BF010F8804628460B
:109F80002BF0C2F900220146814601A829F0F0FA1F
:109F90000027DFF8B8A03C464FF0C00BDDE90132E6
:109FA00093421BD3049850B1C389A3F500739BB2AD
:109FB000C381C38903F4F0530BB92EF0D7FA484696
:109FC00031462EF0EDFDBC422046B8BF384615B0F4
:109FD000BDE8F08F4FF000084646D0E7059D35B14B
:109FE000ED5C0A2D03D1A742B8BF27460024BDF976
:109FF0002C20002A0FDD203DEBB25E2B97BF1AF814
:10A000001530002313FB02F3B3FBFBF31C4401A840
:10A0100028F0C4FEC2E7531C01D10434F7E7023232
:10A02000F5D130462EF0D1F940B14545EFDBA5EB37
:10A030000801304629F0FDFB0444E8E730462AF0E9
:10A040006FFAF9E712F205001CF20500E1080600BC
:10A050002DE9F04FA5B000AF0D46F862014607F1BB
:10A060005800BA621C461BF0F5FC002800F0608224
:10A07000B7F96C30002B05DD7B624FF0000BC7E9B0
:10A0800007BB21E05E1C00F08380023340F0858036
:10A090000022A049F86A2BF023FE0022F8619E49B5
:10A0A000F86A2BF01DFE00229C493862F86A2BF0FA
:10A0B00017FE2AF073FF002278629949F86A2BF0A4
:10A0C0000FFE2AF06BFF834697F87220B7F85D30D9
:10A0D0003B8102F0300110299BB263D183F0300341
:10A0E000A7F85D30BB6AB7F85F10BC620133CC1AC9
:10A0F00002F00302012A0FD82946F86AFFF722FF6F
:10A1000097F8723003F0030303FB0000BB6A00EB17
:10A11000D070A3EB6003BB6297F87230C3F3810287
:10A12000012A08D87A6A03F0030303FB022303EB36
:10A13000D373A4EB6304B7F85F307B61B7F8613089
:10A14000BB61B7F85D30D80648BFD7E9052328467C
:10A1500048BFC7E905322BF0D7F80022F860014666
:10A1600007F1300029F004FABE6AD7E90C239A42BD
:10A1700080F0A3803B6C9BB313F80290B9F10A0FF7
:10A180002FD17B6A07F130001C4428F007FEEBE773
:10A1900006234FF0000B7B6271E74FF0000BC7F80E
:10A1A00024B06CE720290ED183F06003A7F85D305E
:10A1B000BB6AB7F85F100133CB1ABB62B7F86130E6
:10A1C00001341C1B94E7302992D183F05003B7F877
:10A1D0006110A7F85D30631CCB1ABC6ABB6287E7CD
:10A1E0009946B7F96C80B8F1000F40F38C80A9F163
:10A1F00020095FFA89F25E2A9BBF4A4B13F8193097
:10A20000002313FB08F39CBFC021B3FBF1F33B61B8
:10A210003B695B42B34249DA7B699E4246DAC8F148
:10A220000003A34242DABB699C423FDA5E2A3DD872
:10A2300000233C4A1D4699455BDC02EB4902C7F806
:10A2400000D053787B60384B88B000201D44EA462C
:10A25000814660237A68914526DA2A7895F801C00C
:10A260004FF0300E02F07F0218FB02E2B2FBF3F275
:10A2700032442AF810200AEB40010CF07F0218FB50
:10A2800002E21CF0800FB2FBF3F222444A8000F19C
:10A29000020034D04110524607F158001BF0EAF991
:10A2A00028F004FA602350B3D7F800D03B691E446D
:10A2B00028F0FCF9002800F02881F86B002840F015
:10A2C0002981D7E90712F8682EF03EFC3B89A7F8F0
:10A2D0005D3007F158001BF083FBFB6AFA6ADB89EB
:10A2E00003F500739BB2D381F86A9437BD46BDE88D
:10A2F000F08F02EB4301013349780D449BE709F1EC
:10A3000002090235A6E7B8F1FF3F5FD1F11C0DDA73
:10A310000436CDE70DF2050012F2050017F2050034
:10A320001CF20500E1080600C5F405007B699E42A9
:10A33000EEDA621DECDBBB699C42E9DAA9F1210986
:10A34000B9F15E0FE4D8052399FBF3F303EB830225
:10A35000A9EB020909EB49023A614FF00609754A77
:10A3600009FB03F302EB430906F1010A33B20025AE
:10A370007B600FFA8AFA39F8028B3B6948FA03F8D6
:10A3800018F0040F07D062197B6E796812B207F1DA
:10A3900058001BF011FB18F0020F07D02A197B6E32
:10A3A00012B2514607F158001BF006FB18F0010FDE
:10A3B00008D02A19B11C7B6E12B209B207F15800FD
:10A3C0001BF0FAFA0135062DD5D1A1E718F1020FDD
:10A3D0007FF46EAF386A2DF0F8FF00285DD0CB45D2
:10A3E00000F3918007F144050022396A284629F0DC
:10A3F000BFF84FF00008A9EB0B09796CBB6C7A6DC4
:10A40000994203D2FB6C0B444B453DDB002A42D002
:10A41000555C386D50B1C389A3F500739BB2C381FD
:10A42000C38903F4F0530BB92EF0A0F86B42B3428A
:10A430003DDA7B699E423ADA7B6A5B42A34236DAB6
:10A44000BB699C4233DA7B6AF96908FB03F807F1C0
:10A45000440A4FEAD802504629F08AF808F0070863
:10A460004FF00009C7F804A0A94545DB386DF0B1ED
:10A47000C389A3F500739BB2C381C38903F4F0536E
:10A48000ABB92EF073F812E002B1525C284690444A
:10A4900028F084FCB1E71546BBE7386A2AF040F89B
:10A4A000A9EB0B08CB45054600FB08F8BEDD2E44A2
:10A4B000FEE67B6D73B17A6C9B5C03FA08F31B06B6
:10A4C00008D504EB0A027B6E396912B207F1580015
:10A4D0001BF072FA08F10108B8F1080F04D178688E
:10A4E00028F05CFC4FF000080AF1010A7B6A534532
:10A4F000DFDC09F10109B7E706EB09031BB24FF0F6
:10A50000000A3B61F2E70025D1E707F1300028F0AF
:10A5100045FC2AE6C389A3F500739BB2C381C389B6
:10A5200003F4F053002B7FF4CCAE2EF01FF8C8E6F6
:10A53000F862D9E6E4D605002DE9F04F99B00AACEF
:10A5400081460F460146204616461D461BF082FAFC
:10A55000002800F08980229BADF826300DF1220200
:10A5600008A92046ADF82070ADF82260ADF824505F
:10A570001BF060F80DF1260209A920461BF05AF8DD
:10A58000BDF92000BDF92420BDF92210BDF9263007
:10A590008518121ACE1802EBD27A5B1A4FEA6A0AB1
:10A5A000013203EBD378B8BFCAF1000A4FEA68085A
:10A5B0000133B8BFC8F1000808FB08F30393039AFE
:10A5C0000AFB0AF305EBD57506EBD6766D1076100F
:10A5D000049353430793009605EB0A033246A5EB19
:10A5E0000A0120461AF034FF0023CDE90534012783
:10A5F000B8450DDA0AA81BF0F3F9B9F80E3003F5E7
:10A6000000739BB2A9F80E30484619B0BDE8F08F30
:10A61000059B049A5C1E07FB07F3AAEB0404534353
:10A62000002C17DCF21BAAEB040305EB040BA5EBD3
:10A63000040A5146059300925B4606981AF008FFFB
:10A64000F219514600925B4606981AF001FF013755
:10A65000A246CDE7039904FB04F201FB02320799FD
:10A660009142DFDA013CDBE78146CDE737B50546AD
:10A670001C4613440093121B0B19091BFFF75CFFC8
:10A68000EB8903F500739BB22846EB8103B030BD24
:10A69000F0B593B004460F46014604A816461D4681
:10A6A0001BF0D8F9002849D0189BADF80E300DF1F9
:10A6B0000A0202A904A8ADF80870ADF80A60ADF866
:10A6C0000C501AF0B7FF0DF10E0203A904A81AF0FE
:10A6D000B1FFBDF90A200092BDF90C30BDF9081098
:10A6E00004A81AF0B5FEBDF90C30BDF90E20009299
:10A6F0001946BDF90A2004A81AF0AAFEBDF90E20D9
:10A700000092BDF90C30BDF9081004A81AF0A0FEA3
:10A71000BDF90830BDF90A2000921946BDF90E2096
:10A7200004A81AF095FE04A81BF05AF9E38903F572
:10A7300000739BB2E381204613B0F0BD0446FAE7F4
:10A74000F0B593B004460F46014604A816461D46D0
:10A750001BF080F958B3189BADF80E300DF10A02CA
:10A7600002A904A8ADF80870ADF80A60ADF80C5065
:10A770001AF060FF0DF10E0203A904A81AF05AFFA7
:10A78000BDF90E300093BDF90A20BDF90C30BDF9BA
:10A79000081004A81AF05CFE04A81BF021F9E38954
:10A7A00003F500739BB2E381204613B0F0BD04466D
:10A7B000FAE730B591B004460D46014602A81BF0F9
:10A7C00049F978B38DB100234FF0FF32CDE905236D
:10A7D000ADF820309DF8223023F03F034FF6FF7292
:10A7E00043F00F0307928DF82230DDE90553BDF8E1
:10A7F00011200593013ABDF80F3012B20092013BCF
:10A8000000221BB2114602A81AF022FE02A80595EA
:10A810001BF0E6F8E38903F500739BB2E381204661
:10A8200011B030BD0446FAE72DE9F04F9DB00EADF2
:10A8300003900F460146284616461C461BF00AF9AF
:10A84000002800F0C680269BADF836300DF13202AC
:10A850000CA92846ADF83070ADF83440ADF8326040
:10A860001AF0E8FE0DF136020DA928461AF0E2FEB4
:10A87000BDF93040BDF93420BDF93200A31803EB17
:10A88000D3734FEA630ABDF93630C118121B01EBCE
:10A89000D1711B1A491002EBD27464100491013279
:10A8A00003EBD371B8BF64424FEA610B0133B8BF09
:10A8B000CBF1000B0BFB0BF30793079A04FB04F39C
:10A8C000089353430B93049A119BAAEB0401284667
:10A8D0001AF00BFE119B049A0AEB040128461AF0A9
:10A8E00004FE002301270993BB450DDA0EA81BF0D7
:10A8F00077F8039B039ADB8903F500739BB2D3813E
:10A9000003981DB0BDE8F08F099B089A5E1E07FBF7
:10A9100007F3A61B5343002E2BDCA31B0993AAEBC2
:10A9200006030593049BA3EB07090AEB06030693B2
:10A93000049B03EB0708A31B012B24DC119B059947
:10A940004A4628461AF0D1FD119B06994A462846E8
:10A950001AF0CBFD119B0599424628461AF0C5FD19
:10A96000119B0699424628461AF0BFFD013734462E
:10A97000BAE7079906FB06F201FB02320B999142F6
:10A98000CBDA013EC7E7AAEB0403544401334A463D
:10A990000599CDF800902846013C0A931AF058FD1D
:10A9A00023464A460699CDF8009028461AF050FDF5
:10A9B0000A9B0599CDF80080424628461AF048FDCA
:10A9C000CDF8008023464246069928461AF040FDFD
:10A9D000CCE7039094E737B505461C461344009333
:10A9E000121B0B19091BFFF71FFFEB8903F50073FF
:10A9F0009BB22846EB8103B030BD00002DE9F04743
:10AA00008AB080462DF0E1FC044638B96149032044
:10AA10002AF0E4FE20460AB0BDE8F0870022414655
:10AA2000684628F0A5FD00273C463E46B9463D460F
:10AA3000DDE90032934212D3039850B1C389A3F5E4
:10AA400000739BB2C381C38903F4F0530BB92DF09B
:10AA50008DFD01F01CFE0546D8B90024DAE7049A02
:10AA60006AB1D35C0A2B0AD155EA090308BF012752
:10AA700009F101090025684628F090F9D8E7A145B9
:10AA800005F10105A8BF09F10104AE42B8BF2E4689
:10AA9000F1E730462DF05CF93F490246284629F09F
:10AAA00068FF20462DF054F93C490246284629F01B
:10AAB00060FF04FB06F007300021C0102DF020FFDE
:10AAC000044668B9EB89A3F500739BB2EB81EB896F
:10AAD00003F4F053002BC0D128462DF047FD99E731
:10AAE0003A464146684628F043FD4FF00008474685
:10AAF0004FF08009DDE90032934213D3039850B13F
:10AB0000C389A3F500739BB2C381C38903F4F053D7
:10AB10000BB92DF02BFD22462149284629F029FFAB
:10AB20002C4677E7049A5AB1D35C0A2B06D108F178
:10AB300001080027684628F031F9DBE7202B26D0F2
:10AB400020462DF042FC10B306FB087A21464FEA5E
:10AB5000DA0205A828F00CFD099909B1059BC95C2A
:10AB60000AF0070A49FA0AFA41EA0A0105A8C9B235
:10AB700028F064FA089850B1C389A3F500739BB21A
:10AB8000C381C38903F4F0530BB92DF0EFFC0137F7
:10AB9000D0E700BFDEF005001AF1050006F205005F
:10ABA000941706002DE9F04316461D46421E47F64F
:10ABB000FE739A428FB080460F4602D84A1E9A42D0
:10ABC00005D9774901202AF009FE002408E0304623
:10ABD000FBF71AFC044638B9724901202AF0FEFD41
:10ABE00020460FB0BDE8F0836F49002023F090F9B4
:10ABF00004460028F4D04FF000094FF0FF33CDE9B0
:10AC000003394FF6FF730593069B009003F440034E
:10AC100043F07F4343F470230693644B0793284625
:10AC200080238DF805908DF80690ADF820308DF8D2
:10AC300022308DF80490ADF80780ADF809708DF8DA
:10AC40000B602DF0C1FA002865D04A4658492846C5
:10AC50002BF046F82AF023FB28B1BDF8053043F06D
:10AC60000103ADF805300022524928462BF038F890
:10AC70002AF015FB28B1BDF8053043F00403ADF808
:10AC8000053000224C4928462BF02AF82AF007FB11
:10AC900028B1BDF8053043F00803ADF805300022B7
:10ACA000464928462BF01CF82AF0F9FA88B19DF89D
:10ACB0000B0001280BD1BDF8053043F00203ADF8BD
:10ACC0000530BDF809305B0703D03D497BE73D49BE
:10ACD00078E7284600223C492BF002F80546D0B11F
:10ACE0003A4929F0BFFA50B93949284629F0BAFA49
:10ACF00050BBBDF8053043F08003ADF80530EB895B
:10AD0000A3F500739BB2EB81EB8903F4F05313B905
:10AD100028462DF02BFCBDF80900BDF80730434351
:10AD20009DF80B0058430730C0100DF027FC294A4E
:10AD300005460146009829F03BFE29462DF030FFDC
:10AD400068461AF04DFE4BE72349284629F08AFA57
:10AD500020B9BDF8053043F48073CEE71F4928467B
:10AD600029F080FA20B9BDF8053043F4C073C4E778
:10AD70001B49284629F076FA20B9BDF8053043F47E
:10AD80000073BAE71749284629F06CFA20B9BDF8D4
:10AD9000053043F42073B0E713482BF0D3FFAEE740
:10ADA0006BF0050078F0050076EF05007FFF7F006F
:10ADB00098EF05009FEF0500A3EF0500AFEF05003A
:10ADC000EDEF0500BDEF050026F0050032F00500AF
:10ADD00036F00500941706003AF005003EF0050035
:10ADE00042F0050046F005004AF0050000000000B2
:10ADF00008B500222DED028BB0EE408AF0EE608A9D
:10AE0000002351EC100B31F067FF98B1B0EE480A07
:10AE1000F0EE680A2FF028FD0B4B51EC100B0022CE
:10AE200031F0D4FCBDEC028B41EC100BBDE80840C6
:10AE30002FF096BCBDEC028B9FED010B08BD00BF4F
:10AE4000000000000000F87F0000E03F000000006C
:10AE5000F8B555EC104B25F000474FF0FF32284B6A
:10AE60002046394631F04CFF60B94FF0FF32244B99
:10AE70002046394631F03AFF20B9B5F1004F08BFFE
:10AE8000002C05D145EC104BBDE8F8402CF04EBF2E
:10AE9000002200232046294631F00AFFC8B912A13A
:10AEA000D1E900012B46224631F0DAFA06460F4678
:10AEB00031F0ECFF04460D4654EA05030DD10022A3
:10AEC00000233046394631F0F3FE30B19FED080BD8
:10AED000DAE709A1D1E90001E4E720462946BDE807
:10AEE000F8402CF0D9BF00BF2083E4FFFFFFDF3F15
:10AEF00000000000000000802083E4FFFFFFDFBFB0
:10AF0000FFFFEF7F2FF028BC2FF00AB92FF0C4BB52
:10AF10002DE9F04790B004460E4605F093F808B9C5
:10AF200000242AE0214601A804F0F8FF0028F7D009
:10AF3000029B93F8252202F0FD02012AF0D10022A3
:10AF40000092DD689B68ED1AEAD026EAE676B54203
:10AF500028BF354628462CF0B5FF0446C8B1029EEE
:10AF600028F0FEFA6B4601462A4630461BF034F9BB
:10AF7000014610B1284804F0FBFF204610B0BDE8A0
:10AF8000F0871AF8081003A827F080FE08F10108DE
:10AF900023E005468146AE4226D9771B202F28BFE5
:10AFA00020270DF1200A6B463A4651460298CDF80B
:10AFB00000901BF011F9804640BB009B83B154B94F
:10AFC0001B202CF05DFE04460028A9D00146424615
:10AFD00003A828F0CDFA4FF00008009B4345D0D8D5
:10AFE000009BBB421D44D6D0002C99D00698002867
:10AFF000C3D0C389A3F500739BB2C381C38903F493
:10B00000F053002BB9D12DF0B1FAB6E70146024852
:10B0100004F0AEFFE8E700BF1FEF05002DE9F043A5
:10B020009DB000AF00230E4607F108018046BB60CB
:10B0300029F09BF90546F8B940462BF00FF8044675
:10B04000B86027F03BFB04F58073834209D961495E
:10B0500001202AF0C3FBA84640467437BD46BDE830
:10B06000F083E31D23F00703ADEB030D6D4622468D
:10B07000294640462AF0E2FF012E01D1142000E0CB
:10B08000F0104FF00009391DC7F80490F5F7ECFEF9
:10B090007C68804624B950482BF074FEA046DBE75C
:10B0A000012E78D15C22494607F11400BE68F4F7FE
:10B0B00039FA4A4BFB6103F188333B6203F12943C0
:10B0C000A3F59613A3F68B637B62A3F18833BB626F
:10B0D000434BFB622EB13246294607F1140017F0AC
:10B0E00037FB7A69B969530F43EAC1031BBAFB60A6
:10B0F000D30002F03F02372A1BBA94BFC2F13802D4
:10B10000C2F1780237493B6107F1140017F020FBC8
:10B11000082207F10C0107F1140017F019FBFB7F5F
:10B120002370FB8B6370FB691B0AA370FB69E370E0
:10B1300097F8233023717B8C63713B6A1B0AA371E0
:10B140003B6AE37197F827302372FB8C63727B6A4A
:10B150001B0AA3727B6AE37297F82B3023737B8DF3
:10B160006373BB6A1B0AA373BB6AE37397F82F3040
:10B170002374FB8D6374FB6A1B0AA374FB6AE3747C
:10B1800000231A4607F11401194401335D2B3FF4E3
:10B1900063AF0A70F6E7E02E06D101232246B968B4
:10B1A000284617F00BFA57E7B6F5807F01D14B46DA
:10B1B000F4E7B6F5C07F06D101232246B9682846D8
:10B1C00017F06AF848E7B6F5007F7FF445AF4B46C5
:10B1D000F3E700BFB1D305007CEE0500012345670E
:10B1E000F0E1D2C385F40500024B03495868002200
:10B1F0002AF076BD682D0020F9E7050010B51D4C3A
:10B200002378834206D002461B490420BDE8104043
:10B210002AF0E4BA00232370184C206890B129B3B7
:10B22000114603F08BFC206850B1C389A3F500736D
:10B230009BB2C381C38903F4F0530BB92DF096F987
:10B24000002323600E4C206850B1C389A3F500731E
:10B250009BB2C381C38903F4F0530BB92DF086F977
:10B2600000232360074B01221A7010BD114603F022
:10B27000C5FCD8E7E4D10020C8E70500DCD10020F8
:10B28000E8D10020ECD1002010B50A460C46002180
:10B29000FFF7B4FF6CB1E389A3F500739BB2E381C0
:10B2A000E38903F4F05323B92046BDE810402DF0A4
:10B2B0005DB910BD10B5094B1C78012C0CD10021D3
:10B2C0000846FCF7AFF906482DF080FB0146204602
:10B2D000BDE81040FFF7D8BF10BD00BFE4D100208B
:10B2E00056EA05000A460021FFF788BF73B5002221
:10B2F000414905462AF0F4FC29F050FE3F4B4049F5
:10B300000646032258682AF0EBFC044678B12A4628
:10B31000B1B229F097FAE389A3F500739BB2E381F8
:10B32000E38903F4F05313B920462DF01FF90022EE
:10B33000344928462AF0D4FC29F030FE80B2002897
:10B3400046D129460820FDF781FA18B90024204685
:10B3500002B070BD2C4B1C6824B1E38903F5007367
:10B360009BB2E381294E33884FF6FF729A4207D190
:10B3700027482DF02BFB01460820FFF785FFE6E765
:10B3800000221D4928462AF0ABFC29F007FE0130B7
:10B3900080B2ADF80400ADF8060001A930880FF0C6
:10B3A0007FFF0EF02FFD05460028D0D00146082073
:10B3B000FFF798FFEB89A3F500739BB2EB81EB8954
:10B3C00003F4F053002BC2D128462DF0CFF8BEE78E
:10B3D00000210920FDF73AFA0028B7D00A4B1C6873
:10B3E00024B1E38903F500739BB2E3810121284670
:10B3F0000FF002FAABE700BF71E80500682D0020EE
:10B400007EE8050057E80500DCD10020B42C0020C0
:10B4100063E8050070B5014606460720FDF716FAF9
:10B4200000283AD01E4B1C6824B1E38903F5007351
:10B430009BB2E3811B4D2B884FF6FF729A4208D1D5
:10B4400019482DF0C3FA01460720FFF71DFF2046DB
:10B4500070BD0022154930462AF042FC29F09EFDBD
:10B460002B8881B2002218460FF018FF0EF0CAFC9C
:10B4700005460028EBD001460720FFF733FFEB8994
:10B48000A3F500739BB2EB81EB8903F4F053002B1F
:10B49000DDD128462DF06AF8D9E70446D7E700BF8A
:10B4A000DCD10020B42C002063E8050071E8050021
:10B4B0002DE9F04F85B0884600AF00230646394697
:10B4C00040463B6028F051FF0546F8B940462AF057
:10B4D000C5FD0446386027F0F1F804F58073834217
:10B4E00009D9424901202AF079F92C46204614371F
:10B4F000BD46BDE8F08FE31D23F00703ADEB030D60
:10B500006D462246294640462AF098FD0021062035
:10B51000FDF79CF908B90446E8E7354B1C6824B1EF
:10B52000E38903F500739BB2E381324B1A884FF62F
:10B53000FF719142984607D12F482DF047FA0146F6
:10B540000620FFF7A1FED1E700222C49D7F8009092
:10B5500030462AF0C5FB29F021FD00221FFA80FAAF
:10B56000274930462AF0BCFB064600283CD0002282
:10B5700024492AF0B5FB29F092FEF389A3F5007364
:10B580009BB2F381F38903F4F053834613B9304639
:10B590002CF0ECFF00239B453B8114BF02230123C9
:10B5A0003B71391D0123B8F800007B71FD60A7F8DD
:10B5B00006A0A7F80A900FF01DF90EF023FC05462F
:10B5C000002893D001460620FFF78CFEEB89A3F5F7
:10B5D00000739BB2EB81EB8903F4F053002B85D110
:10B5E00028462CF0C3FF81E78346D3E7B1D305009B
:10B5F000DCD10020B42C002063E8050071E80500D0
:10B6000085E8050090E8050038B50D4601460A209A
:10B61000FDF71CF9002839D01D4B1C6824B1E389C3
:10B6200003F500739BB2E3811A4B1A884FF6FF7142
:10B63000914208D118482DF0C9F901460A20FFF7B8
:10B6400023FE204638BD1888144B1B7880B2DBB12E
:10B6500000232A461946F8F7C7FE0EF0D3FB05462D
:10B660000028EED001460A20FFF73CFEEB89A3F547
:10B6700000739BB2EB81EB8903F4F053002BE0D114
:10B6800028462CF073FFDCE70820E6E70446D8E7FD
:10B69000DCD10020B42C002063E80500C8CD0020D8
:10B6A000F0B58BB06D460C46294617F0A1F900287D
:10B6B00000F08D800022012395E80300ADF81820EA
:10B6C0008DF81830A023ADF81A30454BADF80C10AA
:10B6D000CDE90732434B0290090C58688DF80E10E3
:10B6E000414909922AF0FCFA29F058FCC3074CBFE3
:10B6F0003E4B3F4B089320464FF0C87309932CF004
:10B7000063FD002841D000223A4920462AF0E8FA99
:10B710002BF06EFA02460B4606460F4631F0F0FA61
:10B7200090B90022344B3046394631F04FF82AA305
:10B73000D3E9002331F074F90022304B30F090FE51
:10B7400031F01CFBADF8200000222D4920462AF0E4
:10B75000C7FA2BF04DFA02460B4604460D4631F06F
:10B76000CFFA90B90022244B2046294631F02EF81A
:10B7700019A3D3E9002331F053F900221F4B30F015
:10B780006FFE31F0FBFAADF8220002AB93E8030044
:10B79000ADF81410090C04908DF8161008AA06A92B
:10B7A00004A80FF07FFD0EF02DFB044678B1014692
:10B7B0000220FFF797FDE389A3F500739BB2E381B5
:10B7C000E38903F4F05313B920462CF0CFFE0BB0FD
:10B7D000F0BD00BFAFF30080000000000088934080
:10B7E00090000400682D0020BCEB050090012003B0
:10B7F0001000A000A4EB050000408F400000E03FD7
:10B80000B0EB05000A460121FFF7F8BC38B5124B32
:10B810001C78012C05461DD100210846FBF702FFCC
:10B8200021460E482CF019FB044609F0F9F95CB1E9
:10B83000E389A3F500739BB2E381E38903F4F0533A
:10B8400013B920462CF092FE29460120BDE838406D
:10B85000FFF7D8BF38BD00BFE4D10020E8D10020F9
:10B860007CDF70472DE9F04FAC4D85B02B6800AF01
:10B87000044603F0040308460E463B602CF0A4FC8B
:10B88000002800F0BC800022A54930462AF028FAA2
:10B89000B0B129F083FB4FF47A73584340F271231F
:10B8A00090FBF3F080B2B0F5804F9E4B28BF4FF471
:10B8B000804020281A8838BF2020824218BF188074
:10B8C0000022994930462AF00BFA38B129F0E7FCFA
:10B8D0002B68002875D023F400632B600022934965
:10B8E00030462AF0FDF938B129F0D9FC2B68002840
:10B8F0006AD023F480532B6000228D4930462AF011
:10B90000EFF98146002800F08480002307F10C0144
:10B91000FB6028F02AFD8046002864D148462AF0C2
:10B920009DFB8246F86026F0C9FE0AF580738342CB
:10B930004DD98049012029F051FFB9F80E30A3F507
:10B9400000739BB2A9F80E30B9F80E3003F4F0532F
:10B9500013B948462CF00AFE20462CF035FC8246EE
:10B9600008B9002C58D131462046FCF7DDFC002CEC
:10B9700040F0D2800024704D70496868224629F05A
:10B9800013FC32466E49686829F00EFC5CB1E3890D
:10B99000A3F500739BB2E381E38903F4F05313B979
:10B9A00020462CF0E3FD3B680BB10EF013FA404645
:10B9B0000EF00EFB3B6843B30EF09CFB0EF008FB51
:10B9C00023E043F4006388E743F4805393E70AF1EC
:10B9D000070323F00703ADEB030DE846524641464B
:10B9E00048462AF02BFB11234146BA893B7207F1E6
:10B9F0000800FFF735FF80460EF0EAFA9DE746B1F2
:10BA000032465049032029F0E9FE1437BD46BDE80F
:10BA1000F08F4FF000089FE720462CF0CDFB7860B8
:10BA2000002868D0E38903F500739BB2E3812B689B
:10BA300023F47F0323F40043214607F10C002B601D
:10BA400027F01DF9D346F86850B9BAF1000F92D02B
:10BA5000BBF1010F8FDD2B6843F400432B608AE7B5
:10BA60002AF063F881462CF0AFFB10B9B9F1000F52
:10BA70001ED131464846FCF757FC8246F86810B1A3
:10BA8000514627F0B3FCBAF1000F0ED0BAF80E30D1
:10BA9000A3F500739BB2AAF80E30BAF80E3003F487
:10BAA000F05313B950462CF061FDD7F804A009E01B
:10BAB00048462CF081FB0028F7D148462CF060FB6B
:10BAC0000028F2D10BF1010BB9F1000F0ED0B9F83B
:10BAD0000E30A3F500739BB2A9F80E30B9F80E3002
:10BAE00003F4F05313B948462CF040FD07F10C0065
:10BAF00027F0B0F8A7E720462CF042FB00283FF4DF
:10BB000039AFE38903F500739BB2E3812B6823F41B
:10BB10007F0323F40043A1E704462CE7E0D1002093
:10BB20006CEB0500B22C002075EB050081EB0500E5
:10BB30006EF40500B1D30500682D00208BEB0500E5
:10BB400095EB0500D7E9050072DF7047F0B5264B8D
:10BB5000264983B0044600AF0246586829F024FB0A
:10BB600020462CF029FBE8B10023391D20467B60DC
:10BB700028F0FBFB054668BB20462AF06FFA064614
:10BB8000786026F09BFD06F58073834217D918492B
:10BB9000012029F023FE1749032029F01FFE0C374E
:10BBA000BD46F0BD20462CF0EBFA0028DCD1002C7D
:10BBB000F5D022461049032029F010FEEFE7F31DCF
:10BBC00023F00703ADEB030D6D46324629462046B0
:10BBD0002AF034FA00213B792A460846FFF7B4FFE1
:10BBE0000EF0F6F9DBE700BF682D00202AEC050017
:10BBF000B1D3050033EC05005FEC050070B5384C9F
:10BC00003849206800222AF06BF8054678B10021F7
:10BC100001200EF0B5F8EB89A3F500739BB2EB8120
:10BC2000EB8903F4F05313B928462CF09FFC002253
:10BC30002D4920682AF054F8054670B101200FF014
:10BC400037FBEB89A3F500739BB2EB81EB8903F41F
:10BC5000F05313B928462CF089FC00222349606870
:10BC60002AF03EF800220546214960682AF038F89B
:10BC7000064605B918B131462846FFF7F3FD2846B8
:10BC800031462CF08DFF00221A4960682AF028F80E
:10BC9000054668B110F0D4FFEB89A3F500739BB2A1
:10BCA000EB81EB8903F4F05313B928462CF05EFCCA
:10BCB0006068114900222AF013F8044678B1FFF7B2
:10BCC00045FFE389A3F500739BB2E381E38903F4A5
:10BCD000F05323B92046BDE870402CF047BC70BD3E
:10BCE000682D00201FEC05004CE805008BEB0500DB
:10BCF00095EB05004BED05002AEC05002DE9F0431E
:10BD0000C38903F5007391B09BB20446C38103A8B5
:10BD10008846154619F082FB90B301212E4817F092
:10BD2000B9FA064648B31FFA88F02CF011F82B49EF
:10BD30000246204628F01DFE00222949204629F00F
:10BD4000CFFFDDF82690009007461FFA88F3002207
:10BD5000294603A8C847002816DA2249042029F0FA
:10BD60003DFD01202BF0ECFF1F490246204628F044
:10BD700000FE314638462CF013FF03A817F002FFEF
:10BD8000204611B0BDE8F08301302BF0E1FF1749E8
:10BD90000246204628F0EDFD022D17D1012114485E
:10BDA00017F078FA05460028E3D0214628F002FD76
:10BDB000EB89A3F500739BB2EB81EB8903F4F0539D
:10BDC000002BD6D128462CF0D1FBD2E721463046B5
:10BDD00028F0F0FCCDE700BF4AF305007AF4050037
:10BDE00000EF050062F305007BF3050082F3050018
:10BDF00087F3050013B5C389019003F500739BB267
:10BE00000C46C3810E4928F091FD0222214601987B
:10BE1000FFF774FF50B1C389A3F500739BB2C381D0
:10BE2000C38903F4F0530BB92CF0A0FB019804492B
:10BE3000012301AA1FF012FB019802B010BD00BF40
:10BE4000F8EE05002DE9F0478EB005468A46174604
:10BE50002CF0BBFA814620B128460021FDF728F9D5
:10BE6000054628462CF0B0F9044638B9574829460B
:10BE70002AF088FF20460EB0BDE8F087BAF1000F27
:10BE800007D050462CF0DFF9044610B9514650480F
:10BE9000EEE7022F16D101A817F088FE90B100221C
:10BEA0004C49284629F01CFF29F078F8DDF80D30C0
:10BEB000834204DACDF80D0001A817F071FE01A845
:10BEC00017F060FE0121444817F0E4F90646002807
:10BED0007AD0012F6DD14149002022F019F8044693
:10BEE00090B9F389A3F500739BB2F381F38903F44E
:10BEF000F05313B930462CF039FBB9F1000FB9D02B
:10BF0000002D39D12C46B5E73549002022F000F844
:10BF1000A046044644B33946204617F0ADF9BAF1BD
:10BF2000000F10D02F4A5146204628F041FD50B155
:10BF3000C389A3F500739BB2C381C38903F4F05393
:10BF40000BB92CF013FB2146304628F033FCB8F136
:10BF5000000F04D042462449204628F0E7FC2A4638
:10BF60002249204628F0E2FC314640462CF018FEDB
:10BF7000B9F1000F0CD05DB1EB89A3F500739BB252
:10BF8000EB81EB8903F4F05313B928462CF0EEFA59
:10BF9000002F7FF46FAF01A819F040FA00283FF49A
:10BFA00069AF01A8214616F0E3FE01A817F0EAFDEB
:10BFB00060E7022F0CBF0E490E49002021F0A8FFB8
:10BFC0004FF000080446A5E70446D1E7E8F2050073
:10BFD00025F2050018F3050027F305002EF30500F0
:10BFE00036F3050054F205005012060000EF05007C
:10BFF0003EF3050043F3050070B58EB0044601A87A
:10C000000E4619F00BFA18B9002420460EB070BD88
:10C0100020462CF0D9F858B11F482CF0D7FC1F4A05
:10C0200001460546204628F0B6FC29462CF0B8FD0E
:10C03000304629F07AFD0546F8B12CF004F980B9B4
:10C04000294617482AF09EFEEB89A3F500739BB2A0
:10C05000EB81EC8914F4F054D6D128462CF086FA02
:10C06000D3E7EB89A3F500739BB2EB81EB8903F473
:10C07000F05313B928462CF079FA204601223146B4
:10C08000FFF7E0FE044618B1014601A817F064F876
:10C0900001A817F077FDB8E75AF405005EF4050033
:10C0A00025F2050070B58EB004460D46014668467F
:10C0B000164619F0CFFC48B33EB140F2FF339D4223
:10C0C000A8BF1D46012DB8BF0125BDF914300233AC
:10C0D0000FD10F49204629F04DF80E49204629F08E
:10C0E00049F80D49204629F045F80C49204629F029
:10C0F00041F86846ADF8145019F072FCE38903F575
:10C1000000739BB2E38120460EB070BD0446FAE78F
:10C110000DF2050012F2050017F205001CF20500F1
:10C120002DE9F04D2DED028B90B004460E460146F0
:10C1300002A890461F469DF8685019F08BFC002815
:10C1400000F0998030462AF0EDF84046B0EE408A83
:10C15000F0EE608A2AF0E6F838465BEC10AB2AF085
:10C16000E1F88DED000BB8F1000F7ED0002F7CD0F0
:10C170000022424B51EC180B30F028FB30F0D6FD7A
:10C1800000223E4B07465946504630F01FFB30F028
:10C19000CDFD9DED000B0022384B064651EC100BF7
:10C1A00030F014FB30F0C2FDBDF80D2012F46072C7
:10C1B00087F3080386F3080680F3080008D0B2F579
:10C1C000C07F29D020D8802A2AD0B2F5807F2CD0F9
:10C1D0009DF81320102A2FD1D910B210C90241EABC
:10C1E000421141EAE000002D43D0059002A819F069
:10C1F000F7FBE38903F500739BB2E381204610B09F
:10C20000BDEC028BBDE8F08DB2F5007F11D0B2F528
:10C21000207FDDD1324601E01A463346064606E06D
:10C220001A46034630461646D2E71A4603461046DB
:10C23000CEE71A463346F6E7202A06D11A0442EA28
:10C240000622104340F07F40CDE7182A04D119049C
:10C2500041EA06210843C6E733441844B0F5C07FDD
:10C260004FF0FF30B8BF0020BDE7304628F058F946
:10C27000B9E70690BAE70446C0E700BF0000704087
:10C2800010B58EB00C460146684619F0E3FB40B18C
:10C29000BDF80530DB0648BF84F001041CB1BDF8D1
:10C2A00009000EB010BDBDF80700FAE72DE9F04F08
:10C2B00097B00546014608A819F0CCFB28B94FF005
:10C2C0000009484617B0BDE8F08F00F0E0F90446D9
:10C2D0000028F4D000212846FFF7D2FF01210746AD
:10C2E0002846FFF7CDFF054638469DF82B602BF01A
:10C2F0002FFD3D490246204628F03BFB28462BF007
:10C3000027FD3A490246204628F033FB012E07D08C
:10C3100030462BF01DFD36490246204628F029FB09
:10C3200005FB07F0704307300021C0102CF0E8FA3D
:10C33000814668B9E389A3F500739BB2E381E38981
:10C3400003F4F053002BBAD120462CF00FF9B8E7D4
:10C350000146002203A827F00BF90025A846AB46AA
:10C36000AA46DDE90312914213D3069850B1C3895E
:10C37000A3F500739BB2C381C38903F4F0530BB9D7
:10C380002CF0F4F84A461B49204628F0F2FAA14660
:10C3900097E70FFA8BF20FFA8AF108A819F0ECFA76
:10C3A0000AF1010A08FA06F8574548EA000806EBC0
:10C3B000050203DC0BF1010B4FF0000A15460AE001
:10C3C000083D28FA05F1C9B203A8019226F0EAFD5A
:10C3D000019A4FEA1828072DF2D8D5086FF0070305
:10C3E00003FB0525BDE700BF1AF1050006F20500B5
:10C3F00020F10500941706002DE9F74F21F00045C4
:10C40000894616461F464FF0FF32414B294680466B
:10C41000044630F075FC002876D14FF0FF323C4BDB
:10C420004046294630F062FC00286DD132463B463A
:10C430003046394630F064FC002865D100220023E4
:10C440004046494630F034FC28B309F1004500224B
:10C4500000233046394630F02BFC10B107F1004381
:10C460001F46002200233046394630F017FC78B9C9
:10C470004FF0FF32264B3046394630F023FC38B1BE
:10C480004FF0FF32224B2046294630F01BFCE8B922
:10C490000024002522E04D46D9E700221D4B20460E
:10C4A000294630F093F9CDE90001B246BB46524629
:10C4B0005B46DDE9000130F00FFC52465B46E0B917
:10C4C000204629462FF0CAFF04460D4622462B4639
:10C4D0003046394630F0F6FB0028DED1002200233A
:10C4E0004046494630F0E4FB10B105F100431D46DB
:10C4F0002046294603B0BDE8F08F104619462FF0BC
:10C50000AFFF82468B46D2E70024034DF0E700BF21
:10C51000FFFFEF7F0000E03F0000F87F2DE9F843C8
:10C5200055EC114B11EE100A294657EC106B30F008
:10C53000FDFB0928804619D830F0DEF822462B464C
:10C5400030F0ACFB90B1B8F1000F63D03046394603
:10C55000B8F1010F03D141EC100BBDE8F88332466E
:10C560003B4630F033F908F1FF38F1E700220023B1
:10C570003046394630F09CFB0022D8B3284B204689
:10C580002946FFF739FF0022002330F087FBF0B384
:10C5900000224FF0804320462946FFF72DFF00225E
:10C5A000002330F07BFBB04607F1004949EC108BCB
:10C5B00068B12EF059F922462B4651EC100B30F0A1
:10C5C00005F9BDE8F84341EC100B2EF0C9B82EF088
:10C5D0004BF922462B4651EC100B30F0F7F841ECAA
:10C5E000100B2EF0BDF853EC102B10EE100A03F1D7
:10C5F0000041B0E700233046394630F04FFB30B100
:10C60000002200232046294630F05CFB28B147EC8D
:10C61000106BCEE7002002499DE7002000219AE739
:10C620000000F03F37B50D4601466846144603F05A
:10C6300075FC98B1019890F82532013B022B0DD87A
:10C6400074B18168294419F0DFFC014630B1054816
:10C65000054B002C08BF184603F08AFC03B030BD20
:10C660002146EFE733EF050042EF0500436833B1A1
:10C67000013B436003685A1C0260187870474FF012
:10C68000FF3070470B685A1C0A601870704705200D
:10C690002BF0F6BAFFF7FBBFFFF7F9BF28F0B0BDEC
:10C6A00008B50B4640220146184627F0A5FE402853
:10C6B00005D10120034929F091F8002008BD01208F
:10C6C000FCE700BF620A0600F0B585B000AF0023AA
:10C6D000391D06467B6027F048FE0446F0B9304617
:10C6E00029F0BCFC0546786025F0E8FF05F580736D
:10C6F000834208D91949012029F070F825462846B7
:10C700001437BD46F0BDEB1D23F00703ADEB030D61
:10C710006C462A462146304629F090FC7B6810483A
:10C72000FB60002207F10801BC601CF0FCF800234C
:10C7300039463B60F4F798FB3E68054626B9094840
:10C740002AF020FB3546DAE77B680548BC603246B4
:10C7500007F10801FB601CF0E6F8D0E7B1D3050053
:10C760006DC602007CEE0500F0B583B000AF00237B
:10C77000391D06467B6027F0F8FD0446F0B93046C7
:10C7800029F06CFC0546786025F098FF05F580736C
:10C79000834208D91649012029F020F82546284669
:10C7A0000C37BD46F0BDEB1D23F00703ADEB030DC9
:10C7B0006C462A462146304629F040FC00231A46A2
:10C7C000796820461CF0A2F9002339463B60F4F753
:10C7D0004BFB3E68054626B906482AF0D3FA354693
:10C7E000DDE73B46044A796820461CF08FF9D6E71E
:10C7F000B1D305007CEE050085C60200F8B5051E24
:10C800000C4606DC2949012028F0E8FF00242046D8
:10C81000F8BD08462BF0D8FC0646A8B100222449F2
:10C82000204629F05DFA28F03AFD0022214906460B
:10C83000204629F055FA28F0B1FB30F0080309D062
:10C84000102809D01C49DEE724B122461B490120EB
:10C8500028F0C4FF012400E002242946204626F0E7
:10C86000BEFC07469EB12946204626F0B8FC054688
:10C870001349002021F04CFB044610B10FB146B122
:10C880003DB92A46394620462CF05EF9BEE73546CA
:10C89000EEE73A460B49204628F06BF8002DB6D05B
:10C8A0002A460949204628F064F8B0E757140600E4
:10C8B0007614060095140600831406009A140600E8
:10C8C000D114060094170600DA14060070B50D1E88
:10C8D000064606DA0B49012028F080FF0024204696
:10C8E00070BD1B202BF0CCF9044615F1FF35F6D3B3
:10C8F00025F0DCFE0028F2D13146204626F0F9FF73
:10C90000F3E700BF4314060038B504462BF05CFC87
:10C91000D8B100220E49204629F0E2F905462BF055
:10C9200054FD10B1284627F0C3FC04465DB1EB89E5
:10C93000A3F500739BB2EB81EB8903F4F05313B9B9
:10C9400028462BF013FE204638BD0446FBE700BF07
:10C950000A140600F8B506460F4614462BF035FDBE
:10C960000546E8B120462BF07EFCD8B1204627F0E2
:10C97000D7FD0546384628F0C7FC044627F098FC4A
:10C980002D1A13D500255CB1E389A3F500739BB282
:10C99000E381E38903F4F05313B920462BF0E6FD5D
:10C9A0002846F8BD304627F083FCE2E7204627F012
:10C9B0007FFC2F18304627F07BFC8742E2D82A46BE
:10C9C000012321463046F3F7E7FEB0FA80F56D0902
:10C9D000D9E7F8B507460D4616462BF0F6FC044697
:10C9E00098B1284628F090FC002E05460FDA002466
:10C9F0005DB1EB89A3F500739BB2EB81EB8903F486
:10CA0000F05313B928462BF0B1FD2046F8BD27F0AE
:10CA10004FFC8419384627F04BFC8442E7D80123A9
:10CA2000324629463846F3F7B7FEB0FA80F4640977
:10CA3000DEE7F0B587B028F067FC0546002842D055
:10CA40000146002201A826F093FD4FF0FF34002795
:10CA5000DDE901639E4225D3049850B1C389A3F553
:10CA600000739BB2C381C38903F4F0530BB92BF05D
:10CA70007DFDA742DABFE21B01320022394628467B
:10CA800026F03CFFEB89A3F500739BB2EB81EB89A9
:10CA900003F4F053044613B928462BF067FD2046F3
:10CAA00007B0F0BD059800B1805D25F0C9FF30B931
:10CAB000039B1E4437EA240728BF3746344601A8A3
:10CAC00026F06CF9C4E70446E9E7000070B50022DF
:10CAD00086B00E461D4929F003F904462BF075FC7B
:10CAE0000546B0B10022214601A826F041FD0025EF
:10CAF000DDE9013293421CD3049850B1C389A3F5F8
:10CB000000739BB2C381C38903F4F0530BB92BF0BC
:10CB10002DFD5CB1E389A3F500739BB2E381E3894A
:10CB200003F4F05313B920462BF020FD284606B03D
:10CB300070BD059800B1C05C864214BF284645F020
:10CB40000100C5B201A826F029F9D1E79D1206001F
:10CB5000F8B506460D460AB3104627F0E1FC002D55
:10CB6000044603DA304627F0A3FB0544002C03DA21
:10CB7000304627F09DFB04441B202BF081F825EA6A
:10CB8000E57524EAE474074630B1A54204DA631B74
:10CB90002A46314626F06FFE3846F8BD00296FF070
:10CBA0000044E9DADEE7F8B505460C46C2B11046A6
:10CBB00027F0B6FC20EAE076002C05DA284627F0BC
:10CBC00077FB044424EAE4741B202BF059F8074651
:10CBD00020B133462246294626F04DFE3846F8BDA0
:10CBE0006FF00046E8E7F8B507460C46CAB11046B4
:10CBF00027F096FC20EAE07524EAE474A542B8BF69
:10CC000023464FF01B00BCBF2C461D462BF038F8C6
:10CC1000064620B12B1B2246394626F02CFE304614
:10CC2000F8BD6FF00040E5E708B508B1036823B927
:10CC30001B20BDE808402BF023B8002129F040FB61
:10CC4000BDE808402AF05ABE70B504462BF0BCFA85
:10CC500010B90024204670BD00222949204629F041
:10CC60003FF806462BF0B0FA002837D000222549BD
:10CC7000304629F035F805462BF0E5FA08B35EB1E9
:10CC8000F389A3F500739BB2F381F38903F4F053A6
:10CC900013B930462BF06AFC002D2ED02C681A4BAD
:10CCA000E31A5C425C41002DD4D0EB89A3F50073FC
:10CCB0009BB2EB81EB8903F4F053002BCAD12846D9
:10CCC00018E05DB1EB89A3F500739BB2EB81EB89B2
:10CCD00003F4F05313B928462BF048FC002EB8D0CB
:10CCE000F389A3F500739BB2F381F48914F4F05433
:10CCF000AFD130462BF03AFCACE72C46D3E700BF6F
:10CD0000DCD405005D180600251B030008B526F0DD
:10CD100090FD08BD70B5054686B01B200E462AF072
:10CD2000AFFF044630B328462BF04FFB10B3002E64
:10CD300020DB3246294601A826F01AFCDDE9012352
:10CD40009A420AD2059B03B19B5C8DF80330012205
:10CD50000DF10301204626F0E1FD049850B1C3898E
:10CD6000A3F500739BB2C381C38903F4F0530BB9DD
:10CD70002BF0FCFB204606B070BD37B505461B20E6
:10CD80002AF07EFF044628B1294601A825F077FF46
:10CD9000019810B9204603B030BD28F0C6FE28F037
:10CDA000FDF801228DF803000DF10301204626F065
:10CDB000B5FD01A825F04EFFEAE7000070B5064674
:10CDC0000D462BF002FB044630B9324613490320CE
:10CDD00028F004FD204670BD1149002021F098F88C
:10CDE00032461049044627F0A1FD45B128462BF0F4
:10CDF000ECFA68B932460949032028F0EFFC00201C
:10CE00002AF0A6FF08490246204627F0B2FDE1E7D6
:10CE10002A460649204627F089FDF0E76112060000
:10CE2000E6D405008C120600931206009D1206003F
:10CE300038B500220849054628F052FF044640B99B
:10CE4000064921F065F8044904460246284627F0C1
:10CE50006DFD204638BD00BF834F0600541206000A
:10CE6000F8B507460E462BF0AFF900283CD000225B
:10CE70001E49384628F034FF04462BF0A6FA70B35A
:10CE8000204627F015FA002E01DD864206D3174909
:10CE9000384628F06FF925462846F8BD324600216D
:10CEA000204626F02BFD6FF0004231460546204615
:10CEB00026F024FD0D490246384627F05AFD002C85
:10CEC000EAD0E389A3F500739BB2E381E38903F41D
:10CED000F053002BE0D120462BF048FBDCE71B2071
:10CEE0002AF0CEFE0546EAE70546D5E70A14060015
:10CEF00038B50C46054651F8043B9847002DA2BFB3
:10CF0000A3690133A36100280BDB04F11C05C1B246
:10CF1000284626F09AF8284625F086FF63690133F3
:10CF2000636138BD2DE9F04F89B000AF0D469246E0
:10CF3000804620F0AFFA4FF0010BF91D0446284659
:10CF400087F807B0F4F78CFB0023064607F10801C9
:10CF50005046BB6027F009FA0546F0B9504629F063
:10CF60007DF88146B86025F0A9FB09F580738342FE
:10CF700007D94549584628F031FC2437BD46BDE85D
:10CF8000F08F09F1070323F00703ADEB030D6D46A6
:10CF90004A462946504629F051F8BB68002BECD090
:10CFA000132C1DD1394A1278002AE6D0F979384875
:10CFB000BD61002291427A61FA61BB754FF0402158
:10CFC00014BF1346202307F114027E75F7F752FFB2
:10CFD00002460028D1D02F49042028F0FFFBCCE7DF
:10CFE000002CCAD12C492246404628F079FE8146C1
:10CFF000014607F10C001DF09DF890B32246274929
:10D00000404628F06DFE28F04AF93B7CB874FF2BAF
:10D0100027D07A7CFF2A24D07A753B75B875FA68D8
:10D020001F4B93FBF2F307F11400012BD8BF2346EB
:10D03000D7F808B097F807A0BB611DF041F8710060
:10D0400001F4FF7107F114001CF0F2FFA34514DC9A
:10D05000BAF1000F03D007F114001CF0FDFFBB7DF7
:10D06000BB74B87C2AF06CFE0C490246404627F09F
:10D070005DFC49462BF094FD7FE7295D07F1140024
:10D080001CF0D6FF0134E1E7B1D30500D8D1002070
:10D0900094CA0020F30D0600070E0600100E0600CD
:10D0A00090D003002DE9F04F93B000AF0E46154627
:10D0B000814620F0EFF94FF0010A044607F117010D
:10D0C000304687F817A0F4F7CBFA002D804606DC2F
:10D0D0004FF0000840464C37BD46BDE8F08F25F0C4
:10D0E000EDFA05F58073834204D95F49504628F074
:10D0F00075FBEDE7EB1D23F00703ADEB030D132CE0
:10D100006E463BD1594B1B78CBB1002307F120026F
:10D110004FF040215648C7F82230C7F826307B85AB
:10D1200087F820A087F8218087F822507E62F7F7E1
:10D13000A1FE024618B14F49042028F04FFB2946B2
:10D14000012026F04CF880460028C1D0014600227C
:10D1500007F1200026F070FA354416F8011B07F19C
:10D16000200025F072FF07F1200025F05DFEB5429A
:10D17000F3D107F1200025F0FDFCABE7002CA7D18F
:10D180003D492246484628F0ABFD8246014607F15C
:10D1900018001CF0CFFF002859D0224637494846D6
:10D1A00028F09EFD28F07BF83B7FB877FF2B4ED010
:10D1B0007A7FFF2A4BD0F97D87F8212087F820302D
:10D1C000BA6987F822002E4B93FBF2F307F1200097
:10D1D000012BD8BF2346F9607B621CF071FF4FEA38
:10D1E000480101F4FF7141F0010107F120001CF03A
:10D1F0001FFF05F1FF38A8EB0403594259410822EB
:10D200004FF0000B07F12000C7E901121CF0B8FE37
:10D21000BA6879684FEA4B0B013A40EA0B0BF1D13F
:10D2200007F120001CF0DAFE012197F8210014F02C
:10D230003BF806F804B00134A542DCD1FB681BB111
:10D2400007F120001CF008FF97F82230BB77B87F69
:10D250002AF076FD09490246484627F067FB514609
:10D260002BF09EFC6BE700BF5F0D0600D8D10020BD
:10D2700094CA0020940D0600070E0600100E06004A
:10D2800090D003002DE9F04F89B08946009020F03E
:10D2900001F94946044602A81CF04CFF40B3132C88
:10D2A00040F002819DF80C40204620F077F99DF86F
:10D2B0000D5018B1284620F071F9E0B922462946F0
:10D2C0008A4829F05FFDB9F1000F00F00A81884A11
:10D2D0000098494627F05FFB50B1C389A3F500735E
:10D2E0009BB2C381C38903F4F0530BB92BF03EF911
:10D2F00009B0BDE8F08F7F49029E7F4B04EB8404A8
:10D3000005EB85050C440D449E4294F801806F782E
:10D3100058DD7A4B9E42D4BF4FF080664FF0CD6609
:10D32000774A784C13785BB323681BB1764B102196
:10D33000C3F880104FF040234FF0FF31C3F80813BB
:10D34000D3F800120021C3F80012C3F80015012120
:10D3500084F8221094F8271079B9D3F808154FF003
:10D36000A04001F5E07140F2023540F82150D3F8B9
:10D370000C3503F5E07340F82350002384F8223085
:10D3800094F8223001251570FBB108225F49042072
:10D3900028F024FA9DF80C40204620F0FFF820B138
:10D3A0004FF42071204614F0FBF89DF80D40204604
:10D3B00020F0F4F8002886D04FF49451204614F061
:10D3C000EFF880E74FF0CC76AAE79DF81E2084F8AE
:10D3D00027209DF81D20A360C4E9003384F8253080
:10D3E00084F8243072B34FEA8800B90000F1A040FD
:10D3F00001F1A04140F20C624FF0A04BC0F80027B1
:10D4000005FA08FAC1F80027BD4040F20D62019309
:10D41000CBF808A5CBF80855C0F80027C1F80027BD
:10D420000420F5F7DDF9019BDBF810150D422BD038
:10D4300043B14FF0A04A0420CAF80C55F5F7D0F9D3
:10D44000CAF808554FF0A04308F5E07140F20C62AD
:10D4500043F8212007F5E07143F821204FF04023E5
:10D460001D46C3F80885C3F80C75C3F82465226807
:10D470001AB106210420F7F757FF0523C5F8003538
:10D48000022384F8223085E701930420CBF80CA511
:10D49000F5F7A6F9CBF808A50420F5F7A1F9019B4B
:10D4A0000133092BC0D1C4E7002C7FF40CAF9DF8E9
:10D4B0000C00FF2807D0012113F0F6FE03219DF890
:10D4C0000C0014F08BF89DF80D00FF283FF4FBAE24
:10D4D000012113F0E9FE03219DF80D0014F07EF800
:10D4E000F1E60349009827F045FE01E7A70D060085
:10D4F000070E060020D5050097AB020087F5040053
:10D50000D8D1002094CA002000E100E0D60D06002A
:10D51000F0B58DB00D4616461C461FF0BBFF122815
:10D520009DF8487005D02E49012028F057F90DB01C
:10D53000F0BD16B90CB90F2403262A4B1B78F6B29E
:10D54000E4B25BB92849ADF810306FF0FF02CDE9C5
:10D55000011201A8254A03920DF0F2FEFF2F03D01D
:10D560000021384620F024FC28462AF07CFE70B1C9
:10D57000284626F0D5FF22463146C0B2F3F7EAFE30
:10D58000FF2FD4D00121384620F012FCCFE72846E7
:10D590002AF038FFE8B1802383F31188012229465D
:10D5A00001A826F0CAFB01A825F033FB054601A817
:10D5B00025B925F0EFFA85F31188E1E728F0E4FAC0
:10D5C00022463146C0B2F3F7C5FE01A827F01EF887
:10D5D000E9E72A460649012028F000F9D0E700BF14
:10D5E000B0130600CAD10020A08601000001080087
:10D5F000D8130600F0B58DB00D4616461C461FF038
:10D6000049FF12289DF8487005D02F49012028F0C5
:10D61000E5F80DB0F0BD16B90CB9032401262B4B6B
:10D620001B7806F00F0604F00F045BB92849ADF82B
:10D6300010306FF0FF02CDE9011201A8254A0392D4
:10D640000DF07EFEFF2F03D00021384620F0B0FB06
:10D6500028462AF008FE70B1284626F061FF2246CF
:10D660003146C0B2F3F736FEFF2FD2D00121384643
:10D6700020F09EFBCDE728462AF0C4FEE8B18023C7
:10D6800083F311880122294601A826F056FB01A840
:10D6900025F0BFFA054601A825B925F07BFA85F3E8
:10D6A0001188E1E728F070FA22463146C0B2F3F75C
:10D6B00011FE01A826F0AAFFE9E72A460649012043
:10D6C00028F08CF8D0E700BF88130600CAD10020EC
:10D6D000A086010000010800D813060013B50C460F
:10D6E0001FF0D8FE8DF807000938052805D80DF180
:10D6F00007020349204628F041FB02B010BD00BFDD
:10D70000F5DA020070B586B00E4602AA01A91CF037
:10D71000FDF960B16EB9FF2502AA0199304628F0E3
:10D720002DFBFF2D03D00121284620F041FB06B040
:10D7300070BD31680029EEDD0139304628F0C0FDAA
:10D7400004462AF0CEFE30B320461FF0FCFE05460C
:10D75000304627F0BDFC50B1C389A3F500739BB2DE
:10D76000C381C38903F4F0530BB92AF0FFFE5CB107
:10D77000E389A3F500739BB2E381E38903F4F053DB
:10D7800013B920462AF0F2FEFF2DC5D0002128460D
:10D7900020F00EFBC0E7002CBDD0FF25E8E700001D
:10D7A0002DE9F04198B00E46174607A908AA1CF0CB
:10D7B000ADF9002800F0A780FF2F03D000213846E4
:10D7C00020F0F6FA30462AF04EFD80463046B8F199
:10D7D000000F1AD026F0A4FE08A920EAE070079BEB
:10D7E0009847002804DA08A94FF0FF30079B9847B4
:10D7F0002AF0AEFA0446FF2F03D00121384620F06C
:10D80000D7FA204618B0BDE8F0812AF0DEFD0546C3
:10D81000002850D01B202AF033FA314604464246F5
:10D8200002A825F0A5FE4646DDE902239A4218D358
:10D830000598002832D14645DDDD24F037FF002869
:10D84000D9D108A9079B4FF0FF30984701228DF8E6
:10D8500007000DF10701204608F1010826F05EF8E7
:10D86000E9E724F023FF0028E2D1069808B1029BE3
:10D87000C05C079B08A99847002806F1010609DB50
:10D880008DF8070001220DF10701204608F101087B
:10D8900026F044F802A825F081FAC5E7C389A3F56C
:10D8A00000739BB2C381C38903F4F053002BC2D130
:10D8B0002AF05CFEBFE7304628F0D0FB014601208D
:10D8C00025F08DFC0446002895D001462A460EA876
:10D8D000CDE90C5525F0B0FE07AA0C49304628F0DA
:10D8E0004DFADDE90C239A4203DB0EA825F042F93C
:10D8F00081E724F0DBFE0028F7D107A94FF0FF30C5
:10D90000FFF7F6FAEDE704467BE700BFF1CE020031
:10D910007FB50C4605461FF0BDFD2146064668460C
:10D920001CF050F8B0B1122E16D168460DF008FD6B
:10D9300054B3184A2146284627F02DF850B1C38920
:10D94000A3F500739BB2C381C38903F4F0530BB9F1
:10D950002AF00CFE04B070BD002EFBD19DF805002E
:10D96000FF2802D0012113F039FE9DF80600FF28A0
:10D9700002D0042113F032FE9DF80700FF28D7D013
:10D98000012113F02BFED3E70249284627F0F2FBD2
:10D99000E0E700BF070E0600F2F7CBBF2BF0B8BAE6
:10D9A000F0B589B02AF056FA044638B310224FF485
:10D9B000D82500210DEB02000095F1F7B3FD04A975
:10D9C00028462BF02DF9C8B101AD06AE0027059B06
:10D9D00001330CD196E8030085E8030028468DF852
:10D9E0000C702AF0F3FF0146204626F017FF0022B4
:10D9F00004A968462BF066F90028E8D1204609B052
:10DA0000F0BDF7B5074608460C4616461D462AF0F7
:10DA1000DBFB00B300222046114609F047FD00253C
:10DA200004462E4638462BF0AFFA00953346224680
:10DA3000F3F736F805465CB1E389A3F500739BB2B2
:10DA4000E381E38903F4F05313B920462AF08EFDF5
:10DA5000284603B0F0BD002CE4D0E28902F5007244
:10DA600092B2E281DEE738B52BF08EFA2BF090F916
:10DA7000044688B100212AF0BDF9E389A3F50073BB
:10DA80009BB2E381E38903F4F053054613B92046C2
:10DA90002AF06CFD284638BD0546FBE708B52BF09B
:10DAA00073FABDE808402BF073B938B52BF06CFA67
:10DAB0002BF06EF9044680B106F048F8E389A3F52F
:10DAC00000739BB2E381E38903F4F053054613B975
:10DAD00020462AF04BFD284638BD0546FBE708B531
:10DAE0002BF052FABDE808402BF05FB94FF4D82074
:10DAF0002BF082B90B78C1B218461CF0B5BF0000FC
:10DB00002DE9F04389B01F4680460C4691461FF030
:10DB1000C1FCA0F10903DBB2052B06463AD80E285A
:10DB20000FD1374B1B7863B94FF0FF324FF41651CA
:10DB3000CDE9041204A8334A06928DF81C30F7F799
:10DB400019FC314D8DF80060B9F1000F03D020466B
:10DB500027F0DAFB04466A462946204628F00EF9EB
:10DB6000B9F1000F0CD05CB1E389A3F500739BB24F
:10DB7000E381E38903F4F05313B920462AF0F6FC5D
:10DB80002FB169460D20A84769460A20A84709B069
:10DB9000BDE8F0830028FAD102461C49404628F02F
:10DBA0009FF8324605461A49404628F099F80DF18B
:10DBB000100806460246294640461CF0D9F85EB1D8
:10DBC000F389A3F500739BB2F381F38903F4F05357
:10DBD00013B930462AF0CAFC5DB1EB89A3F5007396
:10DBE0009BB2EB81EB8903F4F05313B928462AF07A
:10DBF000BDFC98E80F006D4607C52B70054DA3E7E7
:10DC0000D9D10020080001009DAC04002C0A0600B8
:10DC1000070E060035A2040000231A46FFF770BF66
:10DC200001231A46FFF76CBF00230122FFF768BFEC
:10DC3000F0B585B004461FF02DFC002205463C4996
:10DC4000204628F04DF8064628B93A49012027F029
:10DC5000C5FD05B0F0BD00223749204628F040F848
:10DC600032460146074668461CF082F8394630467F
:10DC70002AF096FF3049204627F07CFA2C492046AE
:10DC800027F078FAA5F10903DBB2052B44D900226D
:10DC90002A49204628F024F808B327F07FF9C4B2B7
:10DCA000002120460DF070FE00201BF0F5FF054618
:10DCB000A8B1214625F0FEFA044618B101462846CF
:10DCC00027F080F9284625F071FB20B91C4B1D492F
:10DCD000586827F04FFA294620462AF061FF9DF840
:10DCE0000600FF2802D0002113F078FC9DF8070001
:10DCF000FF2802D0002113F071FC9DF80400FF28DA
:10DD000002D0002113F06AFC9DF80500FF28A0D086
:10DD1000002113F063FC9CE7A5F10D03DBB2012B9E
:10DD2000DDD8FF22002128461CF088FDD7E700BF80
:10DD3000070E0600531306002C0A06007A1306008D
:10DD4000682D00207F130600F0B585B005460F460C
:10DD500014461FF09FFB0646D4B922465B4928466D
:10DD600027F0BEFF04462246394668461CF000F8FC
:10DD7000A0B95CB1E389A3F500739BB2E381E389A9
:10DD800003F4F05313B920462AF0F0FB05B0F0BDC0
:10DD9000E38903F500739BB2E381E4E7009829F07F
:10DDA000D7FF4B490246284626F0E3FD7CB12246C8
:10DDB0004649284626F0DDFDA6F10903DBB2052B16
:10DDC0000AD80E2EE2D16846F7F7D4FADEE73F49CB
:10DDD000284627F0CFF9EFE7002ED7D19DF80500B0
:10DDE000FF2807D0012113F0F9FB01219DF8050060
:10DDF0001FF0DEFF9DF80400FF280BD0052113F073
:10DE0000EDFB60202AF05EF8044660B9314901203C
:10DE100027F0E4FC9DF80630FF2BB7D02E490120F7
:10DE200027F0DCFCB2E702462C49284626F0A1FD8B
:10DE3000204625F095FB002680F84060044613F04C
:10DE40004DFA009B9DF80A2084F85860C4E9143606
:10DE50009DF8083013449DF80920B24218BF0133E1
:10DE6000C4E9120184F8593001219DF804000DF035
:10DE70008BFD044610B329F06BFF19490246284672
:10DE800026F077FD01201BF007FF06460028C1D0D1
:10DE90002A46214626F0D6FCF389A3F500739BB2EF
:10DEA000F381F38903F4F05313B930462AF05EFB93
:10DEB000013C0C4B0C4A43F82420ABE79DF80420AE
:10DEC0000A49012027F08AFCA4E700BF070E0600DC
:10DED0002C0A0600CE1206002B130600F4120600D0
:10DEE0007A1306002CD40020B59C0400FC12060016
:10DEF00010B50C461FF0CEFAA0F10903DBB2052BDA
:10DF000004D82146BDE810401FF004BA02490120A0
:10DF1000BDE8104027F062BCA31206002DE9F347CC
:10DF20001F46012313600C690646894615460CB14D
:10DF30000B68E45C30782E2800F0E3805B282CD15D
:10DF400001237B7296F801A0BAF15E0F02D12B6813
:10DF500001332B604FF000080CE03B4601AA494614
:10DF6000FFF7DCFF2B68019A48EA000813445FFAC8
:10DF700088F82B602B68F45CF018002C00F0C3804C
:10DF80005D2CEAD101332B6000237B72BAF15E0F66
:10DF900014BF444688F001040BE05C2866D10223DC
:10DFA0002B607078642808D1303C092C8CBF002489
:10DFB0000124204602B0BDE8F087442805D1303C5A
:10DFC000092C94BF00240124F3E7662864D06E284E
:10DFD00064D0722864D0732805D1204602B0BDE811
:10DFE000F04724F02DBD532806D1204624F028FD0B
:10DFF00080F00100C4B2DCE7742853D0762853D0F7
:10E0000077280DD1A4F13003092B7AD9204624F0CA
:10E010000BFD002875D15F2C14BF00240124C8E734
:10E0200057280CD1A4F13003092B66D9204624F0DF
:10E03000FBFC002861D15F3C18BF0124B9E7A0F1C7
:10E040003003DBB2092B31D978280FD1B3786BB10B
:10E05000F3785BB104232B60B07824F084FC804615
:10E06000F07824F080FC40EA0810C0B27B7AFBB163
:10E070002B68F35C2D2B1BD1788128680130286038
:10E080003B4601AA49463044FFF748FF2B68019AF6
:10E09000134404462B608CE70C20E7E70A20E5E7F1
:10E0A0000D20E3E70920E1E70B20DFE71846DDE775
:10E0B0003A7A62B1A4F14103192B98BF2034A0F140
:10E0C000410398BFE4B2192B9CBF2030C0B2B7F90E
:10E0D0000A30B3F5807F12D0DBB22AB1A3F141023E
:10E0E000192A9CBF2033DBB24FF480729C427A81A4
:10E0F00003D3844201D8984263E7002459E784425D
:10E100008AE7012455E70249012027F067FB50E721
:10E11000AD15060082B02DE9F047B2B00C463AA921
:10E12000064681E80C0024F0C1FA30B100252846EB
:10E1300032B0BDE8F04702B0704733780BB17C2BAA
:10E140005AD158223AA91CA82FF054F8DDE93A67B1
:10E15000DDF8F48029F07EFEA26823681A440546A3
:10E16000D21B3946304625F0C9FB00210446024641
:10E17000284626F067FB5CB1E389A3F500739BB2E8
:10E18000E381E38903F4F05313B920462AF0EEF952
:10E190000DF1800A4FF00009C1450DDB384629F02A
:10E1A000D7FD91490246284626F0E3FB32468F49C7
:10E1B000284626F0BBFBBAE75AF8041BDAF8202001
:10E1C0003046521A25F09AFB09F10109044602462D
:10E1D0004946284626F036FB002CDDD0E389A3F51E
:10E1E00000739BB2E381E38903F4F053002BD3D196
:10E1F00020462AF0BBF9CFE75E2B09D12368A2683D
:10E20000D34293D11FF080FF00288FD0013607E062
:10E21000242B1DD1D4E900329A4206F101060CD814
:10E2200050223CA968462EF0E5FF3AAB0CCB2146C4
:10E230003046FFF76FFF054679E74C223DA9684657
:10E240002EF0D8FF3AAB0ECB304600F0FAFAF2E7E8
:10E25000282B0FD13D9B2168A2683AA80A44191DBA
:10E26000082B40F8212000EB83014A63CADC01330C
:10E270003D93C7E7292B0AD13D9B002BC2DD3AAA6B
:10E2800002EB83032168A2680A441A63BAE73AAB37
:10E290001BAA21463046FFF741FE1B9FF35DA3F109
:10E2A0002A02012A804606EB070500F28480013726
:10E2B000374450B92B2B08D14C223DA968462EF08B
:10E2C00099FF3AAB0ECB3846BFE7214614A814ADF0
:10E2D00024F005FF0FCD0DF1700CACE80F005022BB
:10E2E0002B68CCF800303CA968462EF083FF3AAB8F
:10E2F0000CCB1CA93846FFF70DFF05461F9850B1FF
:10E30000C389A3F500739BB2C381C38903F4F0539F
:10E310000BB92AF02BF9D4E900239A42BFF407AFD6
:10E32000B8F1000F3FF403AF204624F037FD3AABBD
:10E330001BAA21463046FFF7F1FD2146804614A86E
:10E3400024F0CDFE0DF1500EBEE80F000DF1700C63
:10E35000ACE80F005022DEF80030CCF800303CA9C9
:10E3600068462EF047FF3AAB0CCB1CA93846FFF7A6
:10E37000D1FE81461F9850B1C389A3F500739BB2AB
:10E38000C381C38903F4F0530BB92AF0EFF8B9F154
:10E39000000F0ED05DB1EB89A3F500739BB2EB814A
:10E3A000EB8903F4F05313B928462AF0DFF84D4601
:10E3B000B1E7A946FBE7D4E900239A420BD250B15A
:10E3C000204624F0EBFC1FF09FFE00283FF4AEAE89
:10E3D0001B9B1E4424E74C223DA968462EF00AFFF1
:10E3E0003AAB0ECB284630E7CF150600D515060010
:10E3F0002DE9F047BAB08046084614AF26F084FFF6
:10E40000002283490546404627F06AFC26F0C6FDF7
:10E41000002280498246404627F062FC064629F0E9
:10E42000D4FF044640B9314628462AF0B9FB2046BD
:10E430009837BD46BDE8F087304625F039FF00F13A
:10E44000080323F00703ADEB030D0DF15009421C47
:10E450004946304625F0D0FF5EB1F389A3F500733D
:10E460009BB2F381F38903F4F05313B930462AF0D9
:10E470007DF869214046FEF729FB4FF480720023A6
:10E4800087F84800A7F84A202946524607F11800A5
:10E4900087F84930FB643D6425F06AF807F11801FC
:10E4A000384624F01CFEBC46BCE80F0007F12C04E3
:10E4B0000FC45022DCF80030236007F148016846A1
:10E4C000C7F844A02EF096FE07F140030CCB07F1ED
:10E4D0002C014846FFF71EFE0446B86B564650B165
:10E4E000C389A3F500739BB2C381C38903F4F053BE
:10E4F0000BB92AF03BF807F1180024F04FFC07F1A4
:10E50000400A1CB9D7E906239A4229D3786A50B148
:10E51000C389A3F500739BB2C381C38903F4F0538D
:10E520000BB92AF023F85DB1EB89A3F500739BB218
:10E53000EB81EB8903F4F05313B928462AF016F85F
:10E54000002C3DD1022029F09BFB002504462846E3
:10E5500029F0FEFB2E490246404626F00AFA66E7FD
:10E5600007F11801384624F0BAFDBC46BCE80F009C
:10E5700007F12C040FC40136DCF800302360502270
:10E5800007F1480168467E642EF034FE9AE80C00DC
:10E5900007F12C014846FFF7BDFD0446B86B50B1AA
:10E5A000C389A3F500739BB2C381C38903F4F053FD
:10E5B0000BB929F0DBFF07F1180024F0EFFBA0E70F
:10E5C00067214046FEF782FA00B30021204627F07B
:10E5D00077FE002210490646204627F081FB26F0F0
:10E5E000DDFC0546304625F063FE0544002EAED026
:10E5F000F389A3F500739BB2F381F38903F4F0531D
:10E60000002BA4D1304629F0B1FFA0E705469EE7D4
:10E61000931206008C120600CF1506002DE9F84F64
:10E6200005460E4629F0D1FE20B94FF000084046BD
:10E63000BDE8F88F29F00EFC80460028F5D01EB901
:10E64000294626F0B7F8F2E73046F2F7CDFB00286E
:10E6500000F08180002029F07BFB6A4902463046A9
:10E6600026F087F929463046FFF7C2FE0027044608
:10E6700084B1204629F065FD814618B3E389A3F5EE
:10E6800000739BB2E381E38903F4F05313B920468E
:10E6900029F06CFF002029F05BFB5A490246304606
:10E6A00026F067F9284625F003FEB842BFD3394665
:10E6B0006FF00042284625F021F90146404626F039
:10E6C000ADF8B4E74946204627F0FAFD4A464E49E0
:10E6D0008246204627F004FB26F060FC8146504627
:10E6E00025F0E6FD8346BAF1000F0ED0BAF80E20F1
:10E6F000A2F5007292B2AAF80E20BAF80E2002F427
:10E70000F05212B9504629F031FFA9EB0702394601
:10E71000284625F0F3F80146404626F07FF8E389C5
:10E72000A3F500739BB2E381E38903F4F05309EB93
:10E730000B0713B9204629F019FF384629F008FBCA
:10E7400030490246304626F014F929463046FFF794
:10E750004FFE04468CE7304626F0D6FD064698B1BB
:10E7600025F0A6FD8146284625F0A2FD002700F1F0
:10E77000010BABEB090A3C46544531DCB9F1000F03
:10E780001CD1C4B90134F7E78146ECE75C461FE0D1
:10E790000146404626F00EF8FB89A3F500739BB2B4
:10E7A000FB81FB8903F4F05313B9384629F0DEFEF0
:10E7B00004EB0907E6E754450AD111E05445E5D0DA
:10E7C0000123224631462846F1F7E6FF0028D9D139
:10E7D000E21B3946284625F091F807460028D7D194
:10E7E000002E3FF424AFF389A3F500739BB2F381AD
:10E7F000F38903F4F053002B7FF419AF304629F06E
:10E80000B5FE14E793120600CF15060038B5FFF7E2
:10E81000EFFD054620B129F094FC80F00100C0B264
:10E8200000F001045DB1EB89A3F500739BB2EB81AD
:10E83000EB8903F4F05313B9284629F097FE2046DC
:10E8400038BD84B0F0B59BB021AE054686E80E0019
:10E850001FF05AFC68B9044620461BB0BDE8F040E2
:10E8600004B070475C2C03D16C78002CF4D03D468A
:10E8700001352C78002CEFD07C2C05F10107F1D16B
:10E88000DDE9211215A824F073FE502223A9684661
:10E890002EF0B0FC96E80C0015A93846FFF73AFCBC
:10E8A000044618980028D7D0C389A3F500739BB2FB
:10E8B000C381C38903F4F053002BCDD129F056FE58
:10E8C000CAE70000F7B5064608460D46144629F08B
:10E8D000BAFC30B92A463349032026F07FFF03B043
:10E8E000F0BD6CB300223049304625F0D3FF0090D4
:10E8F000C0B127F0C1FB012300906A4600202946E1
:10E900001CF05EFD00980028E9D0C389A3F50073D0
:10E910009BB2C381C38903F4F053002BDFD129F0EC
:10E9200025FEDCE7214F00223946304627F0D8F992
:10E93000044638B92A463946304625F0F7FFCEE777
:10E940001B4FF0E729F038FC78B12946204625F026
:10E9500031FFE389A3F500739BB2E381E38903F4FC
:10E96000F053002BBBD12046D9E702216846CDE900
:10E97000004529F072FA394605460246304625F030
:10E98000D5FF002DE5D0EB89A3F500739BB2EB8199
:10E99000EB8903F4F053002BDBD1284629F0E6FD88
:10E9A000D7E700BFDA090600FE090600D009060015
:10E9B000D509060010B500220446FFF783FF204664
:10E9C000BDE81040FEF734BA38B5154601220446BA
:10E9D000FFF778FF25B1002229462046FFF772FF96
:10E9E0002046BDE83840FEF723BA00002DE9F04F7D
:10E9F00085B0054629F006FD044640B92A46484937
:10EA0000032026F0EBFE204605B0BDE8F08F454917
:10EA100000201FF07DFA04460028F4D048F20801D7
:10EA2000414829F00DFA06460028ECD022463F491D
:10EA3000DFF8F8B025F07AFF29F00CFA2946824673
:10EA400003A824F01CF94FF0000847460398D8B9F2
:10EA5000A7EB080029F07CF935490246204625F04D
:10EA600088FF52463349204625F083FFF389A3F5FA
:10EA700000739BB2F381F38903F4F053002BC2D1EE
:10EA8000304629F073FDBEE727F04FF80546FEF744
:10EA9000DBF800283BD048F26001274829F0D0F984
:10EAA0008146384629F054F9002102460190484633
:10EAB00029F002FF019B5BB1DA89A2F5007292B2E4
:10EAC000DA81DA8902F4F05212B9184629F04EFDC3
:10EAD00022465946484625F029FF494632462846EF
:10EAE000FFF772FF49462AF05BF85DB1EB89A3F5A9
:10EAF00000739BB2EB81EB8903F4F05313B9284602
:10EB000029F034FD03A8013724F0A4F89EE72A4633
:10EB10003946504625F096FE08F10108E5E700BFAA
:10EB2000241206005412060049EC02001AEC0500FB
:10EB3000491206004F12060089EB020037B5054660
:10EB400001910F4848F2080129F07AF90446A8B16A
:10EB50002A460C4925F0EAFE012301AA214628464F
:10EB60001CF02EFCE389A3F500739BB2E381E389DB
:10EB700003F4F05313B9204629F0F8FC03B030BD7C
:10EB800003EF02001AEC05002DE9F0410F46904614
:10EB900018490022064627F0A3F826F0FFF90022C4
:10EBA00005461549304627F09BF80446F8B1424621
:10EBB0003946013D25F046FE284629F0C9F80D49A1
:10EBC0000246304625F0D5FE1DB921463046FFF7F6
:10EBD000B5FFE389A3F500739BB2E381E38903F4F6
:10EBE000F05323B92046BDE8F04129F0BFBCBDE891
:10EBF000F08100BF491206004F12060037B50546E6
:10EC000001910F4848F2080129F01AF90446A8B109
:10EC10002A460C4925F08AFE012301AA21462846EE
:10EC20001CF0CEFBE389A3F500739BB2E381E3897B
:10EC300003F4F05313B9204629F098FC03B030BD1B
:10EC4000FDEE02001AEC050038B500220D460D4914
:10EC5000044627F045F8A0B1C389A3F500739BB221
:10EC6000C381C38903F4F0530BB929F07FFC20461C
:10EC7000044926F07FFA29462046BDE83840FFF7D0
:10EC8000BDBF38BD4F1206002DE9FF4106461046B4
:10EC90000191144629F090FA0746002852D02146E7
:10ECA00003A823F0ECFF0024039810BB454930462D
:10ECB00026F060FA4449304626F05CFA00224349C7
:10ECC000304627F00DF841490546304626F052FA05
:10ECD0001FF092F9804600283ED001462846FFF7F3
:10ECE0008DFF2A462146404629F02EFF04B0BDE89C
:10ECF000F08126F01AFF01AB0122314605461FF0D4
:10ED000007FFEFB950B1C289A2F5007292B2C28179
:10ED1000C38903F4F0530BB929F028FC5DB1EB89EA
:10ED2000A3F500739BB2EB81EB8903F4F05313B9A5
:10ED3000284629F01BFC03A823F08CFF0027B3E72B
:10ED40000446EBE7002CB1D0204601AB012231464E
:10ED50001FF0DEFE0446A9E74DB32046FDF774FF21
:10ED600050B348F208011A4829F06AF848F208013D
:10ED70000646184829F064F80746A6B198B12A4615
:10ED80001549304625F0D2FD2A461349384625F06C
:10ED9000CDFD012231462046FFF794FD424639461B
:10EDA0002046FFF78FFD3946304629F0F9FE294607
:10EDB000204629F0F5FE99E721462846FFF7BEFEDA
:10EDC000F5E700BFD0090600D5090600834F06000D
:10EDD0003DEB0200FDEB02001AEC0500414B2DE972
:10EDE000F047B2F100080E464FF000023E493F4F97
:10EDF000054608BF1F4626F073FF044668B1C38965
:10EE0000A3F500739BB2C381C38903F4F053002BB5
:10EE100066D1BDE8F04729F0A9BB012028F090FF9A
:10EE200031490246284625F0A4FD224639462846A7
:10EE300026F056FF044600284ED102462C49DFF842
:10EE4000B090284626F04CFF0446CCB9B8F1000F2C
:10EE50003BD032462749284625F068FD002C3FD09C
:10EE6000224631462846FFF70FFFE389A3F50073DA
:10EE70009BB2E381E38903F4F0538BBB2046C8E7E0
:10EE800000223946204626F02BFF8246024648B132
:10EE900031462046FFF7F8FE21465046BDE8F047D0
:10EEA00029F07EBE4946204626F01AFFE389A3F5E5
:10EEB00000739BB2E381E38903F4F053824613B9F4
:10EEC000204629F053FB5446BFE732460A49012049
:10EED000BDE8F04726F082BCB8F1000FC0D0B8E71B
:10EEE000BDE8F087D5090600070A0600D00906002C
:10EEF000834F0600FE0906000C0A06000022FFF7F9
:10EF00006DBF0122FFF76ABF2DE9F74F12F0E6F956
:10EF10008946074624F09CFF834612F0DFF98046BD
:10EF20008A46FDF7B4FB0446002800F0A580554B47
:10EF300055495868002226F0D3FE0546002800F007
:10EF40009F8025F0F5F8EB89A3F500739BB2EB8168
:10EF5000EB8903F4F053064613B9284629F006FB63
:10EF60004A49002501235A1E12018818B0F80EC024
:10EF70001CF03F0F0DD0CDE9003229F08DF901359D
:10EF8000009B424928B1019A8A580F321209134452
:10EF90001544013340F6C4129342E4D9B018AB1BB8
:10EFA000401B009328F0D4FE39490246204625F044
:10EFB000E0FC009B184628F0CBFE3649024620466E
:10EFC00025F0D7FC40F6C41028F0C2FE32490246B4
:10EFD000204625F0CEFC304628F0BAFE2A490246EB
:10EFE000204625F0C6FC584628F0B2FE2B490246C2
:10EFF000204625F0BEFCB8EB07006AEB09012DF0B6
:10F00000B7FB0022264B2DF0E1FB264B00222DF012
:10F01000DDFB41EC100B28F089FE23490246204617
:10F0200025F0A7FC214828F093FE214902462046FE
:10F0300025F09FFC002028F08BFE1E49024620464A
:10F0400025F097FC1C4828F083FE1C490246204608
:10F0500025F08FFC4FF4D82028F07AFE184902469C
:10F06000204625F086FC4FF4002028F071FE15495B
:10F070000246204625F07DFC204603B0BDE8F08F17
:10F0800006466DE7682D0020B6110600882D002089
:10F09000BE110600C3110600C9110600CF110600FB
:10F0A00000408F400000B03ED211060050E1002029
:10F0B000D9110600E9110600EC880600F5110600DA
:10F0C000061206001712060010B5FDF7E0FA044616
:10F0D000294829F07BFC29490246204625F049FCB5
:10F0E000274829F073FC27490246204625F041FCB9
:10F0F000254829F06BFC25490246204625F039FCBD
:10F100004FF4002028F024FE21490246204625F035
:10F1100030FC4FF4803028F01BFE1E49024620468A
:10F1200025F027FC05F046FE1B490246204625F047
:10F1300020FC1A4B1B78093BDBB20A2B96BF184AFE
:10F14000184852F8230029F041FC1749024620468E
:10F1500025F00FFC154829F039FC154902462046D8
:10F1600025F007FC134828F0F3FD1349024620461A
:10F1700025F0FFFB204610BD1D11060025110600DD
:10F180002D11060035110600401106004811060039
:10F190004E1106009526060054110600B82C0020DA
:10F1A000A4090600525106005B1106006311060017
:10F1B000A8110600BC2C0020B011060038B5084983
:10F1C000054600201EF0A4FE044638B1284628F06B
:10F1D00057FE04490246204625F0CBFB204638BDA9
:10F1E000DA0F0600BB0B06002DE9F74F0D46032191
:10F1F0000446CDE9002312F0F1F94FF0000B4FF077
:10F20000010A4FF08008D94615F1FF3502D203B04C
:10F21000BDE8F08F009B0AEA0306019B0BEA030797
:10F2200056EA070316D088F311880021204612F011
:10F230003BF80A200BF074FA0121204612F034F852
:10F2400089F3118837200BF06BFA1AEB0A0A4BEBA3
:10F250000B0BD9E788F311880021204612F024F81F
:10F2600041200BF05DFA0121204612F01DF889F3D0
:10F2700011880520E7E710B40C78024600232046E9
:10F2800008215DF8044BFFF7AFBF2DE9F8430D46A9
:10F290000321074612F0A2F9002401264FF080084E
:10F2A000A14615F1FF3502D22046BDE8F88388F368
:10F2B00011880021384611F0F7FF03200BF030FAD7
:10F2C0000121384611F0F0FF0A200BF029FA3846E8
:10F2D00011F0D6FF00B1344389F3118835200BF0CB
:10F2E0001FFA7600DDE710B50321044612F076F927
:10F2F0000021204611F0D8FF4FF4FA700BF010FAFD
:10F300000121204611F0D0FF50200BF009FA2046D1
:10F3100011F0B6FF04464FF4D2700BF001FA84F0FE
:10F320000100C0B210BD000008B50022034926F05C
:10F33000D7FCBDE808401EF01DB900BFBB0B06009E
:10F340002DE9F04F8BB00C46FFF7EEFF06461EF09E
:10F3500025F928B94FF0000840460BB0BDE8F08F02
:10F3600028F078FD80460028F4D0631EFF2B28BFCC
:10F37000F0242246E317CDE900234FF00009304680
:10F38000FFF7B1FF0028E7D0DDE900230821304670
:10F39000FFF72AFF01240025AA462746012130460F
:10F3A000FFF773FF01215FFA80FB3046FFF76DFF27
:10F3B000BBF1010FC0B22BD101283AD1402FCBDDD8
:10F3C0009DF80C30002BC7D005AC0DF10C090025C1
:10F3D000A34619F8017B380923F07AF9207007F069
:10F3E0000F0023F075F90135082D607004F1020457
:10F3F000EFD1002358468DF8243029F0E7FA014672
:10F40000404625F00BFAD146BAF1000FA4D0B6E77A
:10F410000AAB2B44834513F81C3C2DD14F4524DA0D
:10F420001C4214BF4FF0010B4FF0000BBBF1000F5B
:10F4300021D00AAB2B444FF0010B13F81C3C2343A3
:10F440000AAA2A44012102F81C3C30465A460023ED
:10F450006400FFF7C9FE14F0FF0404BF0135012466
:10F46000072D07F1010799DDA8E70CBF4FF0010B4D
:10F470004FF0000BDAE7BA4623EA0403E0E770B581
:10F480008AB00C46FFF750FF06461EF087F868B3B7
:10F49000204628F0E8FE18B3204625F041F8014642
:10F4A0000546012023F09BFE044650B10146002290
:10F4B000684624F0C1F815F1FF3505D2684623F0FF
:10F4C00059FB20460AB070BD08213046FFF7DDFE2B
:10F4D000C1B2684623F0B9FD684623F0A5FCEAE70F
:10F4E00008213046FFF7D1FE28F032FC0446E8E759
:10F4F00037B50D461446FFF717FF8DF807001EF0CD
:10F500004DF880B10DF107020C49284626F036FC73
:10F510009DF807004CB1012111F0C6FE01219DF8B4
:10F52000070012F05BF803B030BD042112F056F86A
:10F5300001219DF8070011F0B7FEF4E777F2020011
:10F5400010B5FFF7F1FE04461EF028F838B120464A
:10F55000CC2200230821BDE81040FFF745BE10BDB6
:10F560002DE9F04786B00C46FFF7DEFE07461EF099
:10F5700015F840B1204628F028FF38B92246304916
:10F58000032026F02BF906B0BDE8F087204624F0D2
:10F590008FFE1028F2D13846FFF7A5FE2146002243
:10F5A00001A823F0E5FF0024A146A046A246059B42
:10F5B0000BB1019A9B5C8DF8003001A823F0EEFBA3
:10F5C000059B0BB1019A9B5C8DF8013001A823F0DB
:10F5D000E5FB00231A46102168468DF802A023F0AF
:10F5E0003AFAA4F12002C4F12003A14000FA02F289
:10F5F00020FA03F31143A0401943083440EA0906F6
:10F6000041EA0805402CB146A846D0D1049850B133
:10F61000C389A3F500739BB2C381C38903F4F0537C
:10F620000BB928F0A3FF3846552200230821FFF725
:10F63000DBFD32462B4640213846FFF7D5FDA2E7D9
:10F64000E20F060010B5FFF76FFE04461DF0A6FF9F
:10F6500020B12046BDE81040FFF745BE10BD0000B8
:10F660002DE9F74305460F46904628F0ECFD044689
:10F6700040B92A466E49032026F0B0F8204603B070
:10F68000BDE8F083284628F064FD002835D0A9881D
:10F69000286828F0D5FB04460028EFD029466846A4
:10F6A00023F0EDFA009E002E37D0F38903F50073A6
:10F6B0009BB2F381304626F038FA8146304628F076
:10F6C000CAFE20B3B9F1000F33D00121304625F036
:10F6D00081F9054678B10146204624F0BDFFEB894B
:10F6E000A3F500739BB2EB81EB8903F4F05313B9DC
:10F6F000284628F03BFF01250AE0284628F09AFD1D
:10F70000002814BF0820072028F0BAFAC3E70546EE
:10F710004946304629F044FA6DB9B8F1000F0ED1D0
:10F72000009D002D57D13A464249204625F0FEF86B
:10F73000A4E74D46ECE7684623F08CFAB2E7414671
:10F7400001A823F09CFA01980028E9D026F0EDF9F1
:10F75000009D0646A5B1EB8903F500739BB2EB81D2
:10F76000284628F078FE88B9EB89A3F500739BB290
:10F77000EB81EB8903F4F05313B9284628F0F6FE29
:10F7800032460021204629F097F813E0012200219B
:10F79000284625F0CFFA3146804623F027FE414621
:10F7A000204624F059FF2846414629F0F9F96846D9
:10F7B00023F050FA5EB1F389A3F500739BB2F38195
:10F7C000F38903F4F05313B9304628F0CFFE01A8B3
:10F7D00023F040FAB7E7EB8903F500739BB20122EF
:10F7E000EB811146284625F0A5FA064678B1014678
:10F7F000204624F031FFF389A3F500739BB2F38117
:10F80000F38903F4F05313B9304628F0AFFEEB89C7
:10F81000A3F500739BB2EB81EB8903F4F05313B9AA
:10F82000284628F0A3FE684623F014FA78E700BFC4
:10F83000E50C06001AEC05002DE9F04F8FB081466B
:10F8400002AF10468A46164628F0DCFD0446002822
:10F850005ED0304624F060FD4028834680460AD9B9
:10F8600002463049012025F0B9FF002420463437F4
:10F87000BD46BDE8F08F8300DA1D22F00702ADEB34
:10F88000020D02AD2A462B440021934219D10122D8
:10F890003146381D24F051FA381D23F0BAF998B9D1
:10F8A000381D23F077F900231946CDE9008552462B
:10F8B00048461EF041FC29460446404629F0F2F82D
:10F8C000D4E742F8041BE0E7381D23F030F9044682
:10F8D00028F010FE58B1204624F022FE061E06DB5A
:10F8E000B34504DD381D26F08BF945F826005CB1E0
:10F8F000E389A3F500739BB2E381E38903F4F0533A
:10F9000013B9204628F032FE381D24F07FFEC3E7ED
:10F910002EB132460449012025F060FFA6E7B0462B
:10F920003546C0E7620C0600AA0C06002DE9F34735
:10F93000044608460D4628F086FC30B95649032097
:10F9400025F04CFF02B0BDE8F087204628F001FC0E
:10F950000646284628F0FDFB864208D0284628F0B7
:10F96000F8FBE389002855D043F04003E3812046AB
:10F9700028F060FC0646284628F05CFC86420BD046
:10F98000284628F057FCE3899BB223F03F03002868
:10F9900045D043F00803E38100224049DFF8FC90A2
:10F9A000DFF8FCA0204624F075FF00223C49074602
:10F9B000204624F06FFF0646204625F0FFFB29462F
:10F9C00001A823F05CF9019D65BB7FB13946204653
:10F9D00024F042FEFB89A3F500739BB2FB81FB89F7
:10F9E00003F4F05313B9384628F0C0FD002EA9D017
:10F9F0003146204624F030FEF389A3F500739BB214
:10FA0000F381F38903F4F053002B9BD1304628F0A7
:10FA1000ADFD97E723F040031B041B0CA6E743F062
:10FA20000703B8E7EB8903F500739BB201A8EB81EC
:10FA300023F010F94946284624F014FCE8B9514651
:10FA4000284624F00FFCC0B90121284624F0C2FF4B
:10FA5000804690B10146204624F0FEFDB8F80E30F5
:10FA6000A3F500739BB2A8F80E30B8F80E3003F47B
:10FA7000F05313B9404628F079FDEB89A3F50073E4
:10FA80009BB2EB81EB8903F4F053002B9BD128460A
:10FA900028F06CFD97E700BF1C0D06005A0D06000C
:10FAA000A77A0600F8B507460C46164628F041FD31
:10FAB00028B935490320BDE8F84025F08FBE20461F
:10FAC00028F083FC00285CD02146304827F09CFABF
:10FAD0000546002857D001460122384625F0B0F8E7
:10FAE000EB89A3F500739BB2EB81EB8903F4F05330
:10FAF000044613B9284628F039FD204626F015F8AB
:10FB0000054688B186421ED12146384625F05AFA6C
:10FB1000EB89A3F500739BB2EB81EB8903F4F053FF
:10FB200013B9284628F022FD6CB3E389A3F50073CE
:10FB30009BB2E381E38903F4F05323BB2046BDE885
:10FB4000F84028F013BD28F037FB0028E0D03146FC
:10FB50000122284627F00EFE06460028D8D001468E
:10FB6000284625F02FFAF389A3F500739BB2F381A1
:10FB7000F38903F4F053002BCAD1304628F0F6FC89
:10FB8000C6E7034996E7F8BD5A0F0600910F060035
:10FB9000970F06002DE9F74305460F46914628F0DA
:10FBA000C8FC30B94649032025F018FE03B0BDE873
:10FBB000F083384628F009FC08B94249F3E7484683
:10FBC00028F041FB28B9484628F0FFFB08B93E4918
:10FBD000E9E739463D4827F017FA04460028E5D002
:10FBE00001460122284625F02BF8E389A3F500738E
:10FBF0009BB2E381E38903F4F053064613B9204630
:10FC000028F0B4FC304625F090FF8046002830D123
:10FC10004946304623F0EAFB3146404628F0C0FF13
:10FC20002B49384624F01EFB0028BFD0002229496A
:10FC3000284626F055F8019028F0C7FB48B1264920
:10FC40002846012301AA1BF009FC2249284625F079
:10FC500091FA01980028A9D0C389A3F500739BB23B
:10FC6000C381C38903F4F053002B9FD128F07EFC9D
:10FC70009CE728F0A1FA20B14946404624F09AFDBD
:10FC8000CAE728F0E7F84146044624F093FD4946C8
:10FC9000204624F08FFD2146304623F0A7FB002CA0
:10FCA000BAD0E389A3F500739BB2E381E38903F43F
:10FCB000F053002BB0D1204628F058FCACE700BF31
:10FCC0005A0F06006A0E0600A10E0600910F0600EC
:10FCD00018F405000A140600F90E0600F8B50646E9
:10FCE000084614461F4628F071FE39460546204650
:10FCF00028F0A6F82946044602463046FFF74AFF98
:10FD000029462046BDE8F84028F04ABFF0B585B046
:10FD100006460D4628F00DFC20B93049032025F099
:10FD20005DFD2CE0284628F050FB50B329462C48B6
:10FD300027F06AF9054610B301460122304624F047
:10FD40007FFFEB89A3F500739BB2EB81EB8903F492
:10FD5000F053044613B9284628F008FC7CB121462C
:10FD6000304625F02FF9E389A3F500739BB2E381B8
:10FD7000E38903F4F05313B9204628F0F7FB05B0EC
:10FD8000F0BD4DBB314603A822F079FF154F039C0F
:10FD9000002CF4D0E38903F500739BB2E38103A840
:10FDA00022F058FF0095002301223946204624F016
:10FDB000CBF918B12146304625F004F9E389A3F5C3
:10FDC00000739BB2E381E38903F4F053002BDED18F
:10FDD000204628F0CBFBDAE703499FE75A0F0600DD
:10FDE000910F0600010F0600050F060038B5054605
:10FDF000084628F0EBFD044688B101462846FFF787
:10FE000085FFE389A3F500739BB2E381E38903F4E3
:10FE1000F05323B92046BDE8384028F0A7BB38BDD1
:10FE20002DE9F04387B000AF81460C461546E84601
:10FE300028F07FFB40B93549032025F0CFFC1C3763
:10FE4000C546BD46BDE8F083204628F0BEFA08B995
:10FE50002F49F1E721462F4827F0D6F8064600281B
:10FE6000EDD02946381D22F00AFF0024786830B111
:10FE7000042C3FD122462849032025F0AFFC7868A6
:10FE800050B1C389A3F500739BB2C381C38903F446
:10FE9000F0530BB928F06AFB00223146484624F0A3
:10FEA000CFFE26F0E9F8F389A3F500739BB2F38146
:10FEB000F38903F4F053054613B9304628F056FB96
:10FEC00095B1234607F10802294648461BF078FA07
:10FED000EB89A3F500739BB2EB81EB8903F4F0533C
:10FEE00013B9284628F042FB07F10801204628F004
:10FEF000D9FDA4E725F019FE07F1080343F8240013
:10FF0000381D22F0A7FE0134B0E700BF5A0F0600EB
:10FF1000180E0600910F0600510E0600F8B50F46A8
:10FF2000064600221149384625F0DAFE0546D8B1CA
:10FF300028F0B2F9044648B1284623F011FB376097
:10FF4000706090F82642631E5C425C41EB89A3F529
:10FF500000739BB2EB81EB8903F4F05313B928468D
:10FF600028F004FB2046F8BD0446FBE7360A0600ED
:10FF7000024621B3012924D0022924D0032924D008
:10FF8000042924D0052924D0062924D0072924D0E7
:10FF9000082924D0092924D00A2924D00B2924D0C7
:10FFA0000C2924D00D2924D00E2924D0134B144819
:10FFB0000F2908BF03461349012025F00FBC124B3F
:10FFC000F9E7124BF7E7124BF5E7124BF3E7124B49
:10FFD000F1E7124BEFE7124BEDE7124BEBE7124B59
:10FFE000E9E7124BE7E7124BE5E7124BE3E7124B69
:10FFF000E1E7124BDFE7124BDDE700BFCA0A06005C
:020000023000CC
:10000000610B0600690B0600D20A0600D50A06003D
:10001000DE0A0600E60A0600F00A0600F80A0600F4
:10002000000B06000D0B0600140B06001A0B060051
:10003000290B0600390B0600470B0600530B060080
:10004000BD0A060070B50E4E34783CB915F0C6FEF8
:10005000054628B90B49012025F0C0FB204670BD9C
:1000600009490A48012216F06BFB014618B10848FD
:10007000FFF77EFFF2E7012333702C46EEE700BF67
:10008000F5D10020760A060052510600F8D1002072
:10009000A70A06002DE9F04F9BB005460C46FFF776
:1000A000D1FF002800F00B81294605A8FFF736FF95
:1000B00028B94FF0000B58461BB0BDE8F08F069BE7
:1000C00093F82532023B012BF3D8012221460FA8D9
:1000D00023F033FE4FF0000B0FA822F09AFD08B971
:1000E000054659E007AC0027A2460FA825F04CFDB5
:1000F00004F8010B0FA824F089FA0FA8013722F0A9
:1001000088FD08B1202FF0D1069C204615F062FF33
:100110000546002840F0CB80E379002B40F0C680F4
:10012000A3799E0740F1C680A368FB42814604D2B2
:1001300004F124030393A3684FB9D4E90232934234
:1001400088BFE360A37943F02003A3711DE0C3F3EC
:100150000802002A40F09780206890F8028008F199
:10016000FF3808EA532818F0FF02029230D123BB6F
:10017000216921B918F078F901460028DDD001295C
:100180001DD14FF00203E3710225CB44B9F1000FFA
:1001900000F09380002D9FD00FA822F0FBFC494B6C
:1001A0001B781B0702D4069815F0C6FF002D82D0DD
:1001B00029464548FFF7DCFE7DE76169DAE7481C20
:1001C00002D10125E571E0E72369616103B921618D
:1001D000A3795A060CD52068A269039940780123B7
:1001E00015F0ACFD0028ECD1A37923F04003A371F6
:1001F000236861690193184617F035FE0028C0D0C6
:10020000029BB7F5007F00EB03082AD3019B029AFB
:100210009B7801987E0A32449A4288BF029A4078BD
:1002200088BF9E1A33464246514615F087FD002886
:10023000C7D1A169A1EB08018E420AD94FF400721F
:100240000AEB4121039818F002FAA37923F0400346
:10025000A3717602A3683344B244A360B144BF1BC8
:1002600069E7A36998450CD0D4E902329A4208D9CB
:100270000198039940780123424615F0E5FC0028D7
:100280009FD1C4F81880A068C0F30800C0F50076BC
:10029000BE4228BF3E46243032465146204418F024
:1002A000D6F9A37943F04003A371D3E71D464FF07D
:1002B00000096AE78146072567E701256CE7834661
:1002C000F9E600BFF7D10020F40B060037B504466D
:1002D000FFF7B8FE002841D021466846FFF71EFE12
:1002E00000283BD0019C94F82632012B36D12046C1
:1002F00015F022FF20B9204615F06CFE00B92060F1
:10030000019B1749022283F82622164B00225868C7
:1003100025F0E6FC054608B30122009927F02AFAE9
:10032000044678B10146284624F04CFEE389A3F543
:1003300000739BB2E381E38903F4F05313B92046C1
:1003400028F014F9EB89A3F500739BB2EB81EB89DC
:1003500003F4F05313B9284628F008F903B030BD70
:10036000ED0B0600682D002037B5214B2149586858
:10037000002225F0B5FC0446A0B1014601A822F0F8
:100380007EFC0198E8B9204624F018FFE389A3F524
:1003900000739BB2E381E38903F4F05313B9204661
:1003A00028F0E4F8144B1A782AB1002211461046BE
:1003B0001A7016F0C5F9FF21002015F01FFD03B0DB
:1003C00030BD25F0B2FB0546FFF780FF5DB1EB893C
:1003D000A3F500739BB2EB81EB8903F4F05313B9DF
:1003E000284628F0C3F801A822F034FCC9E700BF72
:1003F000682D0020ED0B0600F5D10020FFF7B4BFFB
:1004000038B504460D4627F0DFFE30B922460C49C8
:100410000120BDE8384025F0E1B928461DF0BEF8BE
:1004200028B908490120BDE8384025F0D7B9FFF7C1
:100430009BFF29462046BDE8384015F0DFBC00BFD1
:10044000710B06009C0B06002DE9F04FC1B004466D
:100450000F46FFF7F7FD68B3AE4BAF49586803226C
:1004600025F03EFC824628B300253C22294611A8EF
:100470001095EFF757F8A94B8DF80A501B88ADF887
:100480000830002C00F00A8110AE21463046FCF7FF
:1004900007F9814680B9BAF80E30A3F500739BB214
:1004A000AAF80E30BAF80E3003F4F05313B95046E0
:1004B00028F05CF80024E0E027B1032202A93846C6
:1004C00023F09AFF954902A82CF0BCFE002800F00A
:1004D000EC80934902A82CF0B5FE002800F00C81B6
:1004E000904902A82CF0AEFE002800F009818E4948
:1004F00002A82CF0A7FE002800F006810024ADE041
:1005000023F02EF85A4607468849204624F031FA4F
:10051000012387F824320023039687F8255287F8B1
:1005200026323B6008F01E0203A907A815F000FF61
:100530000646C8B904AB0D93039920AB07A80E93E8
:1005400017F02EFE0C9D064610B9002D08BF06269A
:1005500018F01C0F00F09580BEB1042E04D107A83E
:1005600018F080F80646C8B1E389A3F500739BB282
:10057000E381E38903F4F05313B9204627F0F6FF33
:1005800031466B48FFF7F4FCB8E7EB7A13F0110F34
:1005900040F0828018F0080F36D002E00C9D48F041
:1005A000080818F097F9C0F30723EB73030C002633
:1005B000A8732B74000E079B6874EE722E776E770B
:1005C000AE77EE7718780193294615F0F4FC019B7D
:1005D000AE760122EE762E756E7583461A7198B14D
:1005E0001A6B01920146184618F004F8019A064663
:1005F0000028B9D107980BF1FF33C360114617F0FB
:1006000093FC06460028AFD1079E336B18F0080F05
:1006100018BF48F02008C7E9073587F806804FF073
:10062000000887F807803078294615F0C4FC386147
:10063000EB69C7F81880C7E902833E60F388BB8086
:10064000B9F1000F03D0F968384615F0DDFC01233D
:1006500087F826322146504624F0ACF8BAF80E301E
:10066000A3F500739BB2AAF80E30BAF80E3003F46B
:10067000F05313B9504627F079FF204641B0BDE84A
:10068000F08F002E7FF470AFEB7ADA060BD418F0FF
:10069000020FB9D0DB07B7D5072665E7254901204A
:1006A00025F09CF8DAE704265EE74FF00108814662
:1006B0004546214900201DF02BFC044600283FF44C
:1006C0001DAF40F2272027F0FDFB834600287FF472
:1006D00017AF1A4A137843F008031370E389A3F5A0
:1006E00000739BB2E381E38913F4F0557FF406AF06
:1006F000204627F03BFF01E74FF012080225D8E71C
:1007000081464FF00A08F9E781464FF012080325A9
:10071000CFE700BF682D0020ED0B06009F09060003
:10072000044B0600282A0600BF0B0600360A060006
:10073000C20B0600D60B0600E80B0600F6D100201F
:1007400038B50446174828F041F9014605462046C9
:10075000FFF77AFE04465DB1EB89A3F500739BB207
:10076000EB81EB8903F4F05313B9284627F0FEFE22
:10077000B4B16FF000412046FAF7CAFB05462046A7
:10078000FFF7A4FDE389A3F500739BB2E381E3893E
:1007900003F4F05313B9204627F0E8FE284638BD8D
:1007A0002546FBE79F09060070B5C8B00446002146
:1007B0003C2219A81891EEF7B5FE34B9FFF742FCB8
:1007C00050B90024204648B070BD214618A8FBF758
:1007D00067FF0028F2D1F4E72022002107A8EEF7F6
:1007E000A1FE18AB002203A90FA8039315F0A0FDEA
:1007F0000028E6D104AB28AE039915930FA81696EE
:1008000017F0CEFC05460028DBD1149B002BD8D076
:1008100007A90FA817F0A6FAFBF739FF044600282E
:10082000D0D0079827F094FA21490246204624F0B8
:10083000A0F89DF82400C0F3001027F081FA1D49AC
:100840000246204624F095F8BDF820305A0A02F2FC
:10085000BC721292C3F34312013A03F01F030FA8B4
:100860001192109307F00AF8BDF822302890DA0AA6
:100870002C92C3F3451203F03F032B92CDE9295389
:1008800007F0A2F82D90304607F076F8CDE9000188
:10089000094928461DF03CFB9DED000B054602F082
:1008A0002FFA2A460549204624F063F88AE700BF5C
:1008B0000DD405003D0C0600410C0600460C060058
:1008C0002DE9F04FC7B0044600213C2217A816912D
:1008D000EEF728FE54BBFFF7B5FB002800F0C480FC
:1008E00016AB099317F0F6FF0122064609A90DA8D9
:1008F00015F01EFD044698B90AAB1393099926AB6F
:100900000DA8149317F04CFC0446002800F0D28088
:10091000042805D1139BD97A11F020010FD00624A9
:1009200065482146FFF724FB002005E0214616A874
:10093000FBF7B6FE0028CED147B0BDE8F08F0D988A
:1009400017F092FD0546002800F0AA80012D0D98B1
:1009500000F0AC806B1C00F0AB8017F08FFA0446FF
:10096000002840F09E80DDF834A02946504617F05C
:100970007AFA0AF1340807460AF50D73C14699451B
:1009800074D10AF13F0243462021934271D11023D2
:100990008AF83F30F3B201938AF84A30C6F307234E
:1009A00002938AF84B30C6F3074303938AF84C301E
:1009B000330E04938AF84D302E0CEBB22E2405939F
:1009C0008AF84E305FFA86FBC5F30723360A8AF8A9
:1009D0004F30202241468AF834408AF848B08AF8DD
:1009E00049600AF15400069317F031FE0D9A8AF817
:1009F000554011780F9B032903D1916A8B4208BFA0
:100A000000238AF86E30C3F307211B0C8AF8683084
:100A10001B0A8AF869308AF86F1092F802A0012345
:100A2000BA44574528D10DA817F01CFE04460028EB
:100A300037D1129B0D9883F814B01022DA72019A04
:100A40009A75029ADA75039A1A76049A5A76059A72
:100A50009A76069ADA765E750123037117F014FA16
:100A6000044600287FF45CAF012065E709F8014BDC
:100A700085E703F8011B88E70D98791C076303716C
:100A8000079115F075FA044658B9079940460123B5
:100A90000022814501D10F46C3E700F8012BF8E79A
:100AA000072429460D9817F0A5FD39E70224F8E739
:100AB0000124F6E7082433E7090C0600F0B5C7B0B7
:100AC000044600213C2217A81691EEF72BFDD4B95D
:100AD000FFF7B8FA00287BD016AB0122694604A8BC
:100AE000009315F025FCE8B901AB0A93009926ABF9
:100AF00004A80B9317F054FBA0B90A9BDB7A9A0663
:100B000009D506200EE0214616A8FBF7C9FD0028EE
:100B1000DED147B0F0BD09990029F2D0CC7AE307C5
:100B200006D5072001463248FFF722FA0020F0E7F9
:100B300014F010041ED0049B187815F03CFA0446FB
:100B400008B90220EEE704A90DA8242217F07FFDC2
:100B500002210DA80F9417F0E3FA0028E2D10DA8A6
:100B6000F0F732FC0028DCD0049B5B699C42D8D0B3
:100B70000428D7D1BDF81650BDF830104FF6FF73DA
:100B8000994208BF294604A817F0CAFA0028C9D11B
:100B90000646E5270899049817F0C6F918BB099B83
:100BA00003F12002934215D1099B1F700498012381
:100BB0000371BDF81630AB420FD324B1214617F0B4
:100BC00019FD0028AED1049817F05EF90028A9D1CC
:100BD00001209EE703F8016BE4E7002104A817F069
:100BE00093FC0028D6D0042808BF02209AE700BF53
:100BF0004C0C06002DE9F043D5B014AC054600219D
:100C00003C2215A82160EEF78DFC3DB9FFF71AFADA
:100C100058B90027384655B0BDE8F083294620462C
:100C2000FBF73EFD0028F1D1F3E70022694603A857
:100C3000009415F07DFB044690B9039B00990B933B
:100C400024AD34AE0BA81195129617F0A9FA0446FC
:100C5000002871D1109979B1CB7ADB0607D405242D
:100C60002546002729463648FFF782F9D2E7039B3D
:100C7000187815F0A0F90D90039B0021DB88ADF8E2
:100C800030300BA817F04CFA04280446E7D00028AF
:100C9000E6D1402309950A9327F0DCF8074600289F
:100CA0003CD00DF1150818E009980378002B08BF17
:100CB000404627F08BFE054678B10146384623F0C2
:100CC00079FDEB89A3F500739BB2EB81EB8903F40B
:100CD000F05313B9284627F049FC0BA815F07AF910
:100CE00005468146F0B90BA8CDF844D01296F0F72E
:100CF0006BFB0428054613D1CDF83C9003A90BA843
:100D000017F030F800210BA817F0FEFB0428054669
:100D10000FD10F949DF81530002BC5D1002501E0AF
:100D20000028EBD00BA815F055F9002D3FF472AF59
:100D300098E70028EED0F5E7042890D090E700BFB0
:100D4000280C060070B51B4B04461B48002A08BF40
:100D500018460E4627F03AFE014605462046FFF7A4
:100D600073FB04465DB1EB89A3F500739BB2EB8185
:100D7000EB8903F4F05313B9284627F0F7FBBCB115
:100D800031462046FFF786F905462046FFF79EFAD2
:100D9000E389A3F500739BB2E381E38903F4F05385
:100DA00013B9204627F0E2FB281C18BF012070BDB4
:100DB0002046FCE7282A0600044B060038B5164CEE
:100DC000164B1546002291420CBF2146194624F0CD
:100DD00087FF0446F0B15DB100232B7027F0D0F9F6
:100DE00030B1A38803F00F03022B04BF01232B7043
:100DF000204622F08DFBE389A3F500739BB2E381CB
:100E0000E38903F4F053054613B9204627F0AEFBFF
:100E1000284638BD0546FBE794170600DA1406009D
:100E20002DE9F04F8FB0CDE900230D4600229C49FB
:100E3000DDF860A09DF864B0044624F051FF24F072
:100E40002EFA30B19749012024F0C8FC0FB0BDE85C
:100E5000F08F28461CF0A2FB08B99349F3E7DDE9BF
:100E6000006323F000474FF0FF32904B3046394685
:100E70002BF046FF80B94FF0FF328C4B304639469D
:100E80002BF034FF40B984A3D3E90023DDE900014E
:100E90002BF00EFF074608B18549D4E710F01EFA83
:100EA000CDE90201504627F08FF90646002800F0F0
:100EB00087803A467F49504624F012FF25F098FE7D
:100EC00021F000490F464FF0FF32784B4946064665
:100ED0002BF016FF00BB4FF0FF32744B30464946F3
